:020000040800F2
:10000000000001208D050208DD050208DD0502085B
:10001000DD050208DD050208DD050208000000001C
:10002000000000000000000000000000DD050208E4
:10003000DD05020800000000DD05020893680008E5
:10004000DD050208DD050208DD050208DD05020800
:10005000DD050208DD050208DD6A0008E36A000824
:10006000E96A0008EF6A0008F56A0008DD05020881
:10007000DD050208DD050208DD050208DD050208D0
:10008000DD050208DD050208DD050208DD050208C0
:1000900000000000DD050208FB6A0008DD0502081B
:1000A000CD620008DD050208E1620008E562000893
:1000B000F96200080D630008751401088114010835
:1000C0008D14010899140108DD050208DD050208F8
:1000D000457700085D77000879770008DD0502089C
:1000E000DD050208116B0008DD050208DD050208C8
:1000F000DD0502080000000000000000DD05020828
:10010000A5140108B1140108CD110208DD0502088B
:10011000DD050208DD050208DD050208DD0502082F
:10012000DD050208DD050208DD050208DD0502081F
:08013000DD050208DD050208EF
:1001400081F0004102E000BF83F0004330B54FEA88
:1001500041044FEA430594EA050F08BF90EA020FF5
:100160001FBF54EA000C55EA020C7FEA645C7FEA88
:10017000655C00F0E2804FEA5454D4EB5555B8BFAB
:100180006D420CDD2C4480EA020281EA030382EA1C
:10019000000083EA010180EA020281EA0303362DAE
:1001A00088BF30BD11F0004F4FEA01314FF4801C81
:1001B0004CEA113102D0404261EB410113F0004F93
:1001C0004FEA03334CEA133302D0524263EB43034A
:1001D00094EA050F00F0A780A4F10104D5F1200EE8
:1001E0000DDB02FA0EFC22FA05F2801841F1000143
:1001F00003FA0EF2801843FA05F359410EE0A5F117
:1002000020050EF1200E012A03FA0EFC28BF4CF047
:10021000020C43FA05F3C01851EBE37101F00045FD
:1002200007D54FF0000EDCF1000C7EEB00006EEB0A
:100230000101B1F5801F1BD3B1F5001F0CD3490894
:100240005FEA30004FEA3C0C04F101044FEA4452EB
:1002500012F5800F80F09A80BCF1004F08BF5FEA72
:10026000500C50F1000041EB045141EA050130BD52
:100270005FEA4C0C404141EB0101013C28BFB1F564
:10028000801FE9D291F0000F04BF01460020B1FAAF
:1002900081F308BF2033A3F10B03B3F120020CDA82
:1002A0000C3208DD02F1140CC2F10C0201FA0CF060
:1002B00021FA02F10CE002F11402D8BFC2F1200CC5
:1002C00001FA02F120FA0CFCDCBF41EA0C0190407B
:1002D000E41AA2BF01EB0451294330BD6FEA0404C4
:1002E0001F3C1CDA0C340EDC04F11404C4F12002AF
:1002F00020FA04F001FA02F340EA030021FA04F3C1
:1003000045EA030130BDC4F10C04C4F1200220FA17
:1003100002F001FA04F340EA0300294630BD21FA55
:1003200004F0294630BD94F0000F83F4801306BF1B
:1003300081F480110134013D4EE77FEA645C18BF0F
:100340007FEA655C29D094EA050F08BF90EA020FA6
:1003500005D054EA000C04BF1946104630BD91EA9E
:10036000030F1EBF0021002030BD5FEA545C05D1A1
:100370004000494128BF41F0004130BD14F58004E0
:100380003CBF01F5801130BD01F0004545F0FE4154
:1003900041F470014FF0000030BD7FEA645C1ABF89
:1003A000194610467FEA655C1CBF0B46024650EAC0
:1003B000013406BF52EA033591EA030F41F40021EC
:1003C00030BD00BF90F0000F04BF0021704730B572
:1003D0004FF4806404F132044FF000054FF0000147
:1003E00050E700BF90F0000F04BF0021704730B508
:1003F0004FF4806404F1320410F0004548BF4042DD
:100400004FF000013EE700BF42004FEAE2014FEA31
:1004100031014FEA02701FBF12F07F4393F07F4F0C
:1004200081F06051704732F07F4208BF704793F00F
:100430007F4F04BF41F40021704730B54FF4607422
:1004400001F0004521F000411CE700BF50EA010225
:1004500008BF704730B54FF000050AE050EA0102CE
:1004600008BF704730B511F0004502D5404261EB3E
:1004700041014FF4806404F132045FEA915C3FF47F
:10048000D8AE4FF003025FEADC0C18BF03325FEA1C
:10049000DC0C18BF033202EBDC02C2F1200300FACD
:1004A00003FC20FA02F001FA03FE40EA0E0021FAF2
:1004B00002F11444BDE600BF70B54FF0FF0C4CF4E0
:1004C000E06C1CEA11541DBF1CEA135594EA0C0F92
:1004D00095EA0C0F00F0DEF82C4481EA030621EACD
:1004E0004C5123EA4C5350EA013518BF52EA033508
:1004F00041F4801143F4801338D0A0FB02CE4FF0BA
:100500000005E1FB02E506F00042E0FB03E54FF0E9
:100510000006E1FB03569CF0000F18BF4EF0010EE1
:10052000A4F1FF04B6F5007F64F5407404D25FEADD
:100530004E0E6D4146EB060642EAC62141EA555190
:100540004FEAC52040EA5E504FEACE2EB4F1FD0CD2
:1005500088BFBCF5E06F1ED8BEF1004F08BF5FEA50
:10056000500E50F1000041EB045170BD06F0004602
:1005700046EA010140EA020081EA0301B4EB5C04AF
:10058000C2BFD4EB0C0541EA045170BD41F48011A7
:100590004FF0000E013C00F3AB8014F1360FDEBFCC
:1005A000002001F0004170BDC4F10004203C35DAA8
:1005B0000C341BDC04F11404C4F1200500FA05F32B
:1005C00020FA04F001FA05F240EA020001F00042CC
:1005D00021F0004110EBD37021FA04F642EB060142
:1005E0005EEA430E08BF20EAD37070BDC4F10C046C
:1005F000C4F1200500FA04F320FA05F001FA04F230
:1006000040EA020001F0004110EBD37041F100011B
:100610005EEA430E08BF20EAD37070BDC4F1200526
:1006200000FA05F24EEA020E20FA04F301FA05F28E
:1006300043EA020321FA04F001F0004121FA04F236
:1006400020EA020000EBD3705EEA430E08BF20EA06
:10065000D37070BD94F0000F0FD101F00046400040
:1006600041EB010111F4801F08BF013CF7D041EAC2
:10067000060195F0000F18BF704703F000465200C6
:1006800043EB030313F4801F08BF013DF7D043EA97
:100690000603704794EA0C0F0CEA135518BF95EA4D
:1006A0000C0F0CD050EA410618BF52EA4306D1D1D4
:1006B00081EA030101F000414FF0000070BD50EAF3
:1006C000410606BF1046194652EA430619D094EA7D
:1006D0000C0F02D150EA013613D195EA0C0F05D167
:1006E00052EA03361CBF104619460AD181EA0301BB
:1006F00001F0004141F0FE4141F470014FF0000073
:1007000070BD41F0FE4141F4780170BD70B54FF00D
:10071000FF0C4CF4E06C1CEA11541DBF1CEA13558D
:1007200094EA0C0F95EA0C0F00F0A7F8A4EB05046F
:1007300081EA030E52EA03354FEA013100F0888066
:100740004FEA03334FF0805545EA131343EA12632F
:100750004FEA022245EA111545EA10654FEA0026E4
:100760000EF000419D4208BF964244F1FD0404F59D
:10077000407402D25B084FEA3202B61A65EB0305F9
:100780005B084FEA32024FF480104FF4002CB6EBB6
:10079000020E75EB030E22BFB61A754640EA0C0036
:1007A0005B084FEA3202B6EB020E75EB030E22BF76
:1007B000B61A754640EA5C005B084FEA3202B6EBB7
:1007C000020E75EB030E22BFB61A754640EA9C0076
:1007D0005B084FEA3202B6EB020E75EB030E22BF46
:1007E000B61A754640EADC0055EA060E18D04FEA04
:1007F000051545EA16754FEA06164FEAC30343EAA4
:1008000052734FEAC2025FEA1C1CC0D111F4801F70
:100810000BD141EA00014FF000004FF0004CB6E769
:1008200011F4801F04BF01430020B4F1FD0C88BF08
:10083000BCF5E06F3FF6AFAEB5EB030C04BFB6EB13
:10084000020C5FEA500C50F1000041EB045170BD06
:100850000EF0004E4EEA113114EB5C04C2BFD4EB33
:100860000C0541EA045170BD41F480114FF0000EB7
:10087000013C90E645EA060E8DE60CEA135594EA33
:100880000C0F08BF95EA0C0F3FF43BAF94EA0C0F36
:100890000AD150EA01347FF434AF95EA0C0F7FF4AB
:1008A00025AF104619462CE795EA0C0F06D152EAFF
:1008B00003353FF4FDAE1046194622E750EA4106E3
:1008C00018BF52EA43067FF4C5AE50EA41047FF4F4
:1008D0000DAF52EA43057FF4EBAE12E74FF0FF3C59
:1008E00006E000BF4FF0010C02E000BF4FF0010C2A
:1008F0004DF804CD4FEA410C7FEA6C5C4FEA430CA3
:1009000018BF7FEA6C5C1BD001B050EA410C0CBFF1
:1009100052EA430C91EA030F02BF90EA020F002053
:10092000704710F1000F91EA030F58BF994208BFBA
:1009300090422CBFD8176FEAE37040F00100704777
:100940004FEA410C7FEA6C5C02D150EA013C07D1CE
:100950004FEA430C7FEA6C5CD6D152EA033CD3D019
:100960005DF8040B704700BF8446104662468C4613
:100970001946634600E000BF01B5FFF7B7FF002846
:1009800048BF10F1000F01BD4DF808EDFFF7F4FF6F
:100990000CBF012000205DF808FB00BF4DF808EDFA
:1009A000FFF7EAFF34BF012000205DF808FB00BF1D
:1009B0004DF808EDFFF7E0FF94BF012000205DF83F
:1009C00008FB00BF4DF808EDFFF7CEFF94BF0120F4
:1009D00000205DF808FB00BF4DF808EDFFF7C4FFED
:1009E00034BF012000205DF808FB00BF4FEA410C36
:1009F0007FEA6C5C02D150EA013C0AD14FEA430C19
:100A00007FEA6C5C02D152EA033C02D14FF0000055
:100A100070474FF0010070474FEA410212F5001293
:100A200015D211D56FF47873B3EB625212D94FEA35
:100A3000C12343F0004343EA505311F0004F23FA1F
:100A400002F018BF404270474FF00000704750EA74
:100A5000013005D111F0004008BF6FF00040704731
:100A60004FF00000704700BF4A0011D212F500128B
:100A700011D20DD56FF47873B3EB62520ED44FEAF6
:100A8000C12343F0004343EA505323FA02F0704776
:100A90004FF00000704750EA013002D14FF0FF30B4
:100AA00070474FF0000070474FEA4102B2F1E04357
:100AB00024BFB3F5001CDCF1FE5C0DD901F0004C45
:100AC0004FEAC0024CEA5070B2F1004F40EB830095
:100AD00008BF20F00100704711F0804F21D113F1C1
:100AE0003872BCBF01F00040704741F480114FEAFA
:100AF0005252C2F11802C2F1200C10FA0CF320FA83
:100B000002F018BF40F001004FEAC1234FEAD3239F
:100B100003FA0CFC40EA0C0023FA02F34FEA430309
:100B2000CCE77FEA625307D150EA01331EBF4FF092
:100B3000FE4040F44000704701F0004040F0FE40AD
:100B400040F40000704700BF80F0004002E000BFAA
:100B500081F0004142001FBF5FEA410392EA030FA8
:100B60007FEA226C7FEA236C6AD04FEA1262D2EBF2
:100B70001363C1BFD218414048404140B8BF5B42F7
:100B8000192B88BF704710F0004F40F4000020F090
:100B90007F4018BF404211F0004F41F4000121F0A6
:100BA0007F4118BF494292EA030F3FD0A2F10102F0
:100BB00041FA03FC10EB0C00C3F1200301FA03F12E
:100BC00000F0004302D5494260EB4000B0F5000F51
:100BD00013D3B0F1807F06D340084FEA310102F110
:100BE0000102FE2A51D2B1F1004F40EBC25008BFC2
:100BF00020F0010040EA03007047490040EB00008C
:100C0000013A28BFB0F5000FEDD2B0FA80FCACF18C
:100C1000080CB2EB0C0200FA0CF0AABF00EBC250B9
:100C200052421843BCBFD0401843704792F0000FA7
:100C300081F4000106BF80F400000132013BB5E7FA
:100C40004FEA41037FEA226C18BF7FEA236C21D070
:100C500092EA030F04D092F0000F08BF08467047D5
:100C600090EA010F1CBF0020704712F07F4F04D1A3
:100C7000400028BF40F00040704712F100723CBFB6
:100C800000F50000704700F0004343F0FE4040F4E0
:100C9000000070477FEA226216BF08467FEA23639E
:100CA0000146420206BF5FEA412390EA010F40F489
:100CB000800070474FF0000304E000BF10F00043D5
:100CC00048BF40425FEA000C08BF704743F09643BC
:100CD00001464FF000001CE050EA010208BF7047D7
:100CE0004FF000030AE000BF50EA010208BF70475E
:100CF00011F0004302D5404261EB41015FEA010C73
:100D000002BF84460146002043F0B64308BFA3F16A
:100D10008053A3F50003BCFA8CF2083AA3EBC2534C
:100D200010DB01FA02FC634400FA02FCC2F120026B
:100D3000BCF1004F20FA02F243EB020008BF20F0A2
:100D40000100704702F1200201FA02FCC2F1200208
:100D500050EA4C0021FA02F243EB020008BF20EAFD
:100D6000DC7070474FF0FF0C1CEAD0521EBF1CEA2B
:100D7000D15392EA0C0F93EA0C0F6FD01A4480EA19
:100D8000010C400218BF5FEA41211ED04FF0006302
:100D900043EA501043EA5111A0FB01310CF000402E
:100DA000B1F5000F3EBF490041EAD3715B0040EA54
:100DB000010062F17F02FD2A1DD8B3F1004F40EB24
:100DC000C25008BF20F00100704790F0000F0CF0F7
:100DD000004C08BF49024CEA502040EA51207F3ABB
:100DE000C2BFD2F1FF0340EAC250704740F4000096
:100DF0004FF00003013A5DDC12F1190FDCBF00F087
:100E000000407047C2F10002410021FA02F1C2F134
:100E1000200200FA02FC5FEA310040F1000053EAD0
:100E20004C0308BF20EADC70704792F0000F00F01E
:100E3000004C02BF400010F4000F013AF9D040EA24
:100E40000C0093F0000F01F0004C02BF490011F4B8
:100E5000000F013BF9D041EA0C018FE70CEAD153B6
:100E600092EA0C0F18BF93EA0C0F0AD030F0004C36
:100E700018BF31F0004CD8D180EA010000F00040EA
:100E8000704790F0000F17BF90F0004F084691F0A8
:100E9000000F91F0004F14D092EA0C0F01D14202E2
:100EA0000FD193EA0C0F03D14B0218BF084608D1AB
:100EB00080EA010000F0004040F0FE4040F40000F5
:100EC000704740F0FE4040F4400070474FF0FF0C88
:100ED0001CEAD0521EBF1CEAD15392EA0C0F93EACF
:100EE0000C0F69D0A2EB030280EA010C49024FEA21
:100EF000402037D04FF0805343EA111143EA1013DA
:100F00000CF000408B4238BF5B0042F17D024FF491
:100F1000000C8B4224BF5B1A40EA0C00B3EB510F6C
:100F200024BFA3EB510340EA5C00B3EB910F24BF55
:100F3000A3EB910340EA9C00B3EBD10F24BFA3EBDA
:100F4000D10340EADC001B0118BF5FEA1C1CE0D1A2
:100F5000FD2A3FF650AF8B4240EBC25008BF20F055
:100F6000010070470CF0004C4CEA50207F32C2BFA9
:100F7000D2F1FF0340EAC250704740F400004FF046
:100F80000003013A37E792F0000F00F0004C02BF77
:100F9000400010F4000F013AF9D040EA0C0093F041
:100FA000000F01F0004C02BF490011F4000F013B9B
:100FB000F9D041EA0C0195E70CEAD15392EA0C0F03
:100FC00008D142027FF47DAF93EA0C0F7FF470AF3B
:100FD000084676E793EA0C0F04D14B023FF44CAF7E
:100FE00008466EE730F0004C18BF31F0004CCAD113
:100FF00030F000427FF45CAF31F000437FF43CAF4F
:101000005FE700BF4FF0FF3C06E000BF4FF0010C70
:1010100002E000BF4FF0010C4DF804CD4FEA400252
:101020004FEA41037FEA226C18BF7FEA236C11D09C
:1010300001B052EA530C18BF90EA010F58BFB2EB4F
:10104000030088BFC81738BF6FEAE17018BF40F0CF
:10105000010070477FEA226C02D15FEA402C05D183
:101060007FEA236CE4D15FEA412CE1D05DF8040B08
:10107000704700BF844608466146FFE70FB5FFF79B
:10108000C9FF002848BF10F1000F0FBD4DF808ED53
:10109000FFF7F4FF0CBF012000205DF808FB00BF44
:1010A0004DF808EDFFF7EAFF34BF012000205DF89E
:1010B00008FB00BF4DF808EDFFF7E0FF94BF0120EB
:1010C00000205DF808FB00BF4DF808EDFFF7D2FFE8
:1010D00094BF012000205DF808FB00BF4DF808ED2B
:1010E000FFF7C8FF34BF012000205DF808FB00BFF8
:1010F0004FEA40024FEA41037FEA226C02D15FEAE5
:10110000402C08D17FEA236C02D15FEA412C02D146
:101110004FF0000070474FF0010070474FEA400267
:10112000B2F1FE4F0FD34FF09E03B3EB12620DD915
:101130004FEA002343F0004310F0004F23FA02F07F
:1011400018BF404270474FF00000704712F1610F26
:1011500001D1420205D110F0004008BF6FF00040FD
:1011600070474FF00000704742000ED2B2F1FE4FC0
:101170000BD34FF09E03B3EB126209D44FEA002366
:1011800043F0004323FA02F070474FF0000070472D
:1011900012F1610F01D1420202D14FF0FF307047CE
:1011A0004FF00000704700BF7BB972B90029BEBF85
:1011B00000204FF0004106E008BF00281CBF6FF080
:1011C00000414FF0FF3000F057B8ADF1080C6DE969
:1011D00004CE002909DB002B1ADB1FF0C7FBDDF86A
:1011E00004E0DDE9022304B07047404261EB4101B5
:1011F000002B1BDB1FF0BAFBDDF804E0DDE9022366
:1012000004B0404261EB4101524263EB430370473B
:10121000524263EB43031FF0A9FBDDF804E0DDE974
:10122000022304B0404261EB41017047524263EB3C
:1012300043031FF09BFBDDF804E0DDE9022304B06B
:10124000524263EB4303704753B94AB9002908BFC0
:1012500000281CBF4FF0FF314FF0FF3000F00CB8FA
:10126000ADF1080C6DE904CE1FF080FBDDF804E061
:10127000DDE9022304B07047704700BF10F8012B6E
:1012800011F8013B012A28BF9A42F7D0D01A7047C3
:10129000034613F8012B002AFBD1181A01387047B6
:1012A00001F0FF01102A2BDB10F0070F08D010F817
:1012B000013B013A8B422DD010F0070F42B3F6D11B
:1012C000F0B441EA012141EA014122F007047FF034
:1012D00000070023F0E80256083C85EA010586EA8B
:1012E000010685FA47F5A3FA87F586FA47F6A5FAC7
:1012F00087F68EB9EED1F0BC01F0FF0102F00702D3
:1013000032B110F8013B013A83EA010313B1F8D17D
:101310000020704701387047002D06BF354603385E
:10132000073815F0010F07D1013015F4807F02BF97
:10133000013015F4C03F0130F0BC0138704700BFE8
:1013400010B5054C237833B9044B13B10448AFF3FF
:1013500000800123237010BDB003002000000000B6
:10136000BC62020808B5034B1BB103490348AFF345
:10137000008008BD00000000B4030020BC62020829
:1013800000B59BB04822002108A822F07EFF182259
:10139000002102A822F079FF02F086F94FF0B04256
:1013A0000120D2F8903023F01803C2F89030D2F820
:1013B000003423F4C06343F40073C2F80034D2F85D
:1013C000003403F4C0630193019B24230893812319
:1013D0000B930023CDE91003B02208A8CDE9122316
:1013E00002F08EFA00B1FEE74F23CDE90230CDE9DD
:1013F0000400CDE90600022102A802F01DFD00B1A3
:10140000FEE71BB05DF804FB7047000038B5104CD8
:10141000237805460BB9012038BD02F061FA227825
:101420004FF47A73B3FBF2F3B0FBF3F000F0C8FCB7
:1014300004460028EFD10F2DEDD8024629464FF083
:10144000FF3000F06BFC034B20461D60E4E700BF5B
:10145000000000200400002010B5032000F04CFC28
:1014600002F03EFA064B18600020FFF7CFFF04465B
:1014700018B9FFF7C9FF204610BD0124FBE700BFE4
:1014800040000020034A044B11681B780B44136092
:10149000704700BFCC03002000000020014B1868FB
:1014A000704700BFCC0300208068C0F38000704705
:1014B000F7B5002301930446002800F0E980856D0C
:1014C00025B905F05DF8E56584F8545023689A68FD
:1014D000D00040F1A1809A68D10000F1B480A26DE3
:1014E00042F01002A265E26D42F00102E2650125C0
:1014F0001846FFF7D9FFA26D02F01002024340F038
:10150000C980A26D206922F4817242F00202A265B4
:101510009A68D2075DD4226BA67E94F82CC0003A5C
:1015200018BF01221703D4E902120A43217E42EABE
:101530008132617E42EAC13242EA4632002842EA02
:101540004C02B4BF20F000414FF400113A430A436B
:1015500094F82010012903D1002E76D142F4803274
:10156000616A21B1A66A01F4E07131430A43D96886
:10157000E66C21F4FE3121F4FF711143D96094F837
:101580003C206168012A01F0404C4CEA060609D172
:10159000D4E910273A433243A66C324342EA0C02A4
:1015A00042F001061F693E4A3A4032431A6121F077
:1015B0000042B2F1804F0CD0B1F1004F09D0394E4A
:1015C000D6F8082701F4701122F470120A43C6F805
:1015D00008275A69666BA16B22F0070232435A61F1
:1015E0005A6922F0700242EA01125A61002835D18C
:1015F0009A6A62F00F029A625B6903F007039E42E7
:101600003CD10023E365A36D23F0030343F0010302
:10161000A365284603B0F0BD9A68234922F0104222
:1016200022F0170242F080529A60204A1268B2FB00
:10163000F1F2013252000192019A002A3FF44BAFBD
:10164000019A013AF7E7002552E7A16D41F0200128
:10165000A165E16D41F00101E16581E7B0F5001F91
:10166000CAD19A6AE269013A92006FF00F0102F062
:101670001C0201FA02F2216E0A43BCE7A36D23F0BB
:10168000120343F01003A365E36D43F00103E36528
:101690000125BEE7A36D43F01003A365F8E700BF83
:1016A00002FCFF1F00200140400D0300400000200D
:1016B000F8B54569082D04460E460AD00368DB6874
:1016C000D80705D5A36D43F02003A3650120F8BD1D
:1016D0000425FFF7E3FE074623681A682A4220D054
:1016E000A26D42F40072A265DA6812F4406F14D160
:1016F000A27E92B91A6812070FD51846FFF7D4FEDA
:1017000020BB5A6822F00C025A60A26D22F480724B
:1017100022F0010242F00102A265227EFAB100200D
:10172000D5E7711CD9D0FFF7B9FEC01BB04201D874
:10173000002ED1D123681B682B40CDD1A26D84F837
:10174000543042F00402A2650320C0E7A26D42F0CB
:101750002002A265E26D42F00102E265DDE70C22A3
:101760001A60DCE70368186C70470000F7B50023C7
:10177000019390F85430012B044600F0C0800568B6
:101780000269012380F854302846FFF78DFE0028B7
:1017900040F0AF8048680B68022822F004027ED037
:1017A000B2F1004FC3F3110E35D1AA6A42EA0E021C
:1017B000AA628A68686902EA032222F07C4222F067
:1017C000FF0220EA03210A43002B6A611DDA4D4A19
:1017D0004D4DD2F80817AB4201F0E07043D10D0235
:1017E00013D4D2F8083723F0E073034343F4000323
:1017F000C2F80837454B1A68454BB2FBF3F20C238D
:1018000002FB03330193019B53BB0020002384F8A8
:10181000543003B0F0BD226E00F01F074FF00F0CE4
:101820000CFA07FC6FEA0C0622EA0C0CBEF1000F62
:1018300011D1C3F38462BA4042EA0C0222668008E6
:10184000E26901309042B4D8A86AC3F38362BA4017
:1018500006403243ACE793FAA3F2B2FA82F2EAE727
:10186000019B013BCEE72B4DAB420BD1C901CCD440
:10187000D2F8083723F0E073034343F08073C2F8D3
:101880000837C2E7244DAB42BFD14B02BDD4D2F8DA
:10189000083723F0E073034343F48003EFE7B2F12A
:1018A000004F01BFAA6AC3F311018A43AA62002B49
:1018B000ABDA154813498342D1F8082709D1D1F88A
:1018C000083702F0A07223F0E0731A43C1F808272A
:1018D0009BE71048834204D1D1F8083702F4400254
:1018E000F1E70D48834290D1D1F8083702F0C07279
:1018F000E9E7A26D42F02002A265184686E70220C1
:1019000087E700BF00200140001000B04000002029
:10191000400D0300004000B8002000B4806D704707
:10192000026838B504461046FFF7BEFD08B900202E
:1019300038BD9368990707D4936823F0004323F0D8
:10194000170343F010039360FFF7A8FD05462368D3
:101950009B685B07EBD5FFF7A1FD401B0228F6D97A
:1019600023689B685A07F2D5A36D43F01003A36563
:10197000E36D43F00103E3650120D9E773B500236C
:10198000026801939368DD07044602D5002002B087
:1019900070BD9168214B194209D0A36D43F010032B
:1019A000A365E36D43F00103E3650120EFE793686E
:1019B00023F0004323F0170343F001039360184B17
:1019C000D3F8083718021CD4637E012BDED0FFF752
:1019D00065FD144E054622681368DB07D6D493686C
:1019E000D9075FBF9368334043F001039360FFF76B
:1019F00055FD401B0228EED923681B68DA07EAD49C
:101A0000CBE7094B094A1B68B3FBF2F3013301939F
:101A1000019B002BD8D0019B013BF8E71700008009
:101A200000200140E8FFFF7F40000020400D030040
:101A300038B504460068FFF737FD054620BB94F82B
:101A40005430012B20D0012384F854302046FFF776
:101A500095FFB0B9A36D226823F4706323F00103EE
:101A600043F48073A3651C23E065136084F854007D
:101A7000936823F0004323F0170343F004039360BB
:101A800038BD84F85450FBE70220F9E738B5036805
:101A90009A680446900704D49A68D10703D40020BA
:101AA00038BD9B68FBE79A6802F00502012A19D14C
:101AB0009A6822F0004222F0170242F002029A6075
:101AC00003221A60FFF7EAFC054623689B68DB07E0
:101AD000E5D5FFF7E3FC401B0228F6D923689B6895
:101AE000DA07F2D5A36D43F01003A365E36D43F06D
:101AF0000103E3650120D3E770B5044600284BD00D
:101B0000836D43F002038365FFF70AFF054668B95A
:101B10002046FFF7BBFF054608B90123A3652268ED
:101B2000936823F0104323F01703936023685A68E7
:101B300022F4677222F003025A6040F29F321A6068
:101B4000D968164A0A40DA605A6922F007025A61D7
:101B500000269A6A9E621A6A02F0F0221A625A6A93
:101B600002F0F0225A62DA6A02F0F022DA621A69AE
:101B700022F040421A610A4AD2F8083723F0FE7375
:101B8000C2F80837204604F01BFDE6652666A66508
:101B900084F85460284670BD0125FBE700023E83AF
:101BA0000020014010B590F85430012B044615D0A8
:101BB000012380F85430FFF7B3FE58B92046FFF7F1
:101BC00065FF38B9A36D23F4807323F0010343F05C
:101BD0000103A365002384F8543010BD0220FCE704
:101BE000F7B50023019390F85430012B04467FD0C1
:101BF000012380F85430FFF749FF23689A6812F0F8
:101C00000102054607D0A36D43F01003A36500232E
:101C100084F854302DE0A16D364F21F4817141F0EC
:101C20000201A165DE68D96826F4FF4626F07C062D
:101C300021F40041360421F00301360CD96008205C
:101C40009968394041F0004199609968002913DA98
:101C50000199013101910199B1F52E3FF5D3A36DA1
:101C600023F0120343F01003A365002384F85430DB
:101C70000125284603B0F0BDD3F8B410013801F0B7
:101C80007F010A44DCD199681A48014041F0010102
:101C90009960D3F8B41021F07F0141EAD202C3F871
:101CA000B4209A68024042F002029A60FFF7F6FB05
:101CB000074623689A68D20708D4DA683243DA60A4
:101CC000A36D23F0030343F001039FE7FFF7E6FB57
:101CD000C01B0228EDD923689B68D907E9D5A36DFD
:101CE00043F01003A365E36D43F00103E365BFE731
:101CF0000225BEE7E8FFFF7F0749CA6822F4E062D9
:101D00000302120403F4E063120C134343F0BF63B5
:101D100043F40033CB60704700ED00E0164B30B564
:101D2000DC68C4F30224C4F10703251D042B28BF7B
:101D30000423062D4FF0FF358CBF033C002405FA29
:101D400003F321EA0303A54022EA0502A340002889
:101D500043EA0203ACBF00F16040084A4FEA0313B4
:101D6000B8BF00F00F00DBB2AABF00F5614013540A
:101D700080F8003330BD00BF00ED00E014ED00E05E
:101D8000002807DB044A4109012300F01F008340BB
:101D900042F82130704700BF00E100E000280CDB72
:101DA0004309064900F01F0020330122824041F818
:101DB0002320BFF34F8FBFF36F8F704700E100E028
:101DC0000138B0F1807F0BD24FF0E023054A586113
:101DD000F02182F823100020072298611A617047D1
:101DE0000120704700ED00E00028A1BF4309403307
:101DF000054A52F82330A3BF00F01F0023FA00F079
:101E000000F001000020704700E100E0002808DB3E
:101E10004309044900F01F0001226033824041F869
:101E20002320704700E100E0704708B5FFF7FCFF92
:101E300008BD704710B5044608B9012010BD437FA6
:101E400003F0FF0213B90277FFF7F3FF0223637772
:101E50002379E3B92368134A5A619A6822F0180279
:101E60009A6062792368D2B94FF0FF321A619A689A
:101E7000616922F060020A439A609A68A16922F0BF
:101E800080020A439A60012363770020D6E7D4E9F1
:101E90000212204600F008F80028E2D0CDE72269BF
:101EA000E4E700BFB71DC104CB0710B50CD51F2355
:101EB000013B1CD321FA03F4E407F9D5102A12D010
:101EC00004D83AB1082A10D001200BE0182AFBD11F
:101ED000062BF9D800684161836823F01803134387
:101EE0008360002010BD072BF3E70F2BF1E7102ACA
:101EF000EAD0E9D8002AE7D1ECE710B5044640B1B2
:101F00000223037104F00EFB002020616071207138
:101F100010BD0120FCE710B504680122236801F020
:101F2000100102FA01F123EA01032360027100208B
:101F300010BD034640B190F82520022A06D00422A5
:101F4000C263002280F82420012070470268806C60
:101F5000116821F00E011160016821F480710160A7
:101F6000116821F001011160D3E9100202F01C0197
:101F700001228A404260D3E9132151605A6D32B187
:101F8000116821F480711160D3E91621516001229A
:101F9000002083F8252083F82400704708B590F8C6
:101FA0002530022B03D00423C363012008BD03683E
:101FB0001A6822F00E021A601A6822F001021A60F2
:101FC000826C136823F480731360D0E9101303F05C
:101FD0001C02012393404B60D0E913325A60436DD9
:101FE00033B11A6822F480721A60D0E916325A604E
:101FF000012380F82530002380F82430836B03B15F
:1020000098470020D2E790F8250070470A4A5369A4
:1020100043F4802330B55361EFF3108472B600238C
:10202000CD58C5500433B3F5807FF9D11369DB0374
:10203000FCD484F3108830BD00400058064B5A6928
:10204000002ABFBF054A9A6002F188329A60BABF7F
:102050005869C00F002070470040005823016745B1
:10206000044B5A6942F000425A615869C043C00F9C
:10207000704700BF0040005870B50546FFF70EFAE4
:10208000124E04463369D90313D43369DA0744BFC7
:10209000012232614CF2FA32134011D10B4E3069F9
:1020A00010F480200BD0FFF7F9F9001BA842F6D3FB
:1020B00004E0FFF7F3F9001BA842E3D3032070BD4F
:1020C000024A1361024A01205360F8E700400058B9
:1020D000D00300202DE9F041184D98462B78012BB4
:1020E00006460C46174626D001232B704FF47A7013
:1020F00000236B60FFF7C0FFA0B9012E16D1104A74
:10210000536943F0010353612760BFF36F8FC4F835
:1021100004804FF47A70FFF7AFFF094A536923EA4E
:102120000603536100232B70BDE8F0813946204639
:10213000FFF76CFFEDE70220F6E700BFD0030020B9
:1021400000400058054A536923F47E7343EAC000F7
:1021500040F4803040F00200506170470040005869
:102160002DE9F041234F3B78012B054688463FD0AF
:1021700001233B704FF47A7000237B60FFF77CFFF4
:10218000044688B92B68042B13D11B4A536943F4C6
:10219000803343F0040353614FF47A70FFF76CFF10
:1021A0000446154B1A681B6800233B702046BDE8A7
:1021B000F0814FF0FF33C8F800306E68D5E9013286
:1021C0001344B3420AD93046FFF7BCFF4FF47A708C
:1021D000FFF752FF50B1C8F800600446064A536941
:1021E00023F47E7323F002035361DAE70136E5E757
:1021F0000224DBE7D0030020004000582DE9F04F17
:10220000564C00234FF00F080A6832FA03F501D14B
:10221000BDE8F08F012505FA03F919EA020275D02D
:102220004E68032706F003054FEA430E07FA0EFC3B
:102230006F1E012F6FEA0C0C6AD8876807EA0C0A38
:10224000CF6807FA0EF747EA0A078760476827EA68
:102250000909C6F300179F4047EA09074760C768A6
:1022600007EA0C098F6807FA0EF747EA0907022DFB
:10227000C76059D0076805FA0EF507EA0C073D4319
:1022800016F4403F056041D023F0030707F1804773
:1022900007F5803703F0030CBD684FEA8C0C4FF054
:1022A000070E0EFA0CFEB0F1904F25EA0E0E51D03B
:1022B0002B4DA84250D005F58065A84214BF0725D4
:1022C000022505FA0CF545EA0E05BD602568D743E1
:1022D00016F4801F0CBF3D4015432560656816F459
:1022E000001F0CBF3D4015436560D4F8805016F4C4
:1022F000803F0CBF3D401543C4F88050D4F8845053
:10230000B60354BF3D401543C4F8845001337BE706
:10231000032DAFD0C76807EA0C098F6807FA0EF7DC
:1023200047EA0907C760A5E74FEAD30900EB890927
:1023300003F0070AD9F820704FEA8A0A08FA0AFB64
:1023400027EA0B0B0F6907FA0AF747EA0B07C9F8E8
:1023500020708FE70025B4E70125B2E70008005898
:1023600000040048044AD168014208B502D0D06098
:1023700004F09EFB08BD00BF0008005803689A697E
:10238000910744BF00229A629A69D2075EBF9A6998
:1023900042F001029A61704730B5039D04682B43F7
:1023A00043EA0243064A6068C1F309010B4342EA6B
:1023B000555223F0004320EA02000343636030BD1E
:1023C000FF63FF0370B5426B1F4CA2420BB201F0DA
:1023D000010501F002041DD01C4EB2421AD01C4E61
:1023E000B24217D0002BACBF0023B8230DB143F08D
:1023F000F2030CB143F0F403102902D143F090032F
:1024000003E0202901D143F0200301680A68134347
:102410000B6070BD002BACBF0023B8230DB143F09F
:10242000F2030CB143F0F4031029E7D0202902D1C4
:1024300043F06003E9E7064CA242E6D0402908BF1A
:1024400043F04003E1E700BF893100088134000810
:102450006530000811F0010307D090F8413003F017
:102460002803282B14BFF22342238A0709D590F8AA
:10247000412002F02802282A0CBF43F0440343F015
:10248000F4030A0401680A6848BF43F0B80322EA6B
:1024900003030B60704703682DE9F0419C6914F059
:1024A000100405460F4616466CD010220024DA614F
:1024B000A0462B689A69920660D4B8F1000F2ED01E
:1024C00044F0040401202E68B36913F4807F03F400
:1024D000806203F4007357D04FF4807144F001041C
:1024E000F161002A51D1002B56D12846FFF746FF53
:1024F000736823F0FF7323F48B3323F4FF7323F00B
:10250000010373606B6C23436B64202385F84130B7
:10251000002385F8423085F84030012044E07A1CE1
:1025200005D19A699606FCD52022DA61C8E7FEF744
:10253000B5FF801BB84201D8002FBAD12B6859686B
:1025400095F8422098690004D2B20AD5480408D40C
:10255000202A06D05A6842F480425A60FEF79EFF55
:1025600006462B689B699906A3D4FEF797FF801B4C
:102570001928F6D920244FF001089AE7B8F1000F86
:102580009ED1D1E720469EE72AB14FF4806244F005
:102590000804F261A7E72BB14FF4007344F0020482
:1025A000F361A2E70028A0D1BDE8F0812DE9F04158
:1025B000DDF8188004460F4616461D4623689B69C1
:1025C00037EA03030CBF01230023B34201D00020EC
:1025D00025E0424629462046FFF75DFFF0B96B1C17
:1025E000ECD0FEF75BFFA0EB0800A84201D8002D5D
:1025F000E4D123689B6937EA03030CBF012300235E
:10260000B342DBD1636C43F020036364202384F87E
:102610004130002384F8423084F840300120BDE886
:10262000F081C36AAA2B02D10023C3627047C36A38
:10263000B3F52A4FFAD14FF00073F6E7704710B5A3
:10264000044600284ED090F8413003F0FF021BB939
:1026500080F84020FFF7F2FF242384F841302368FC
:102660001A6822F001021A60626822F070621A6130
:102670009A6822F400429A60D4E90221012906D125
:1026800042F400429A605A6822F4006207E042F481
:10269000044202299A60F6D15A6842F400625A60F4
:1026A0005A6842F0007242F400425A60DA6822F43A
:1026B0000042DA60D4E904210A43A16942EA012216
:1026C000DA60D4E907210A431A601A6842F001026D
:1026D0001A6000202023606484F84130206384F86D
:1026E000420010BD0120FCE7704710B5044698B1C8
:1026F0000268242380F84130136823F0010313603B
:10270000FFF7F2FF0020606484F8400084F8410085
:10271000206384F8420010BD0120FCE72DE9F0435E
:1027200085B01D460023039390F84130202B0446CA
:10273000174672D103689B6913F400436DD190F87A
:102740004020012A69D00122C1F3090680F8402007
:1027500046F00078242280F8412048F42058436451
:10276000E3682268012B06BF46F0007343F4005370
:1027700043465360FEF792FE814622689369926950
:10278000C3F34013C2F30012134316D023689A69AF
:10279000CDF8009012F010022B4624D120212046C3
:1027A000FFF704FFE8B922682023D36184F84130A1
:1027B00084F8400005B0BDE8F0836B1CDDD0FEF767
:1027C0006DFEA0EB0900A84201D8002DD5D1202331
:1027D00084F84130636C43F020036364002384F881
:1027E00040300120E6E7002220212046FFF7DEFEF0
:1027F0000028F6D123681022DA612022DA61039BD7
:1028000001330393039BBB42AAD384F84120636C3A
:1028100084F8400013436364E3E70220CAE7000042
:10282000F7B50446104694F84120089E202A65D149
:1028300094F84020012A61D0012284F8402021220E
:1028400084F84120102284F84220002262646385CB
:10285000E6622B4B6363638D60629BB2FF2B99BF73
:10286000638D2385FF232385228D94BFE56A4FF076
:1028700080756AB136F000731DD1236810F8017BB2
:102880009F62638D6062013B9BB26385531E23850B
:10289000236B112B16D1AA2E0FD12046FFF7C1FEB4
:1028A000638D9BB2FF2B00D8E56A1648009094F820
:1028B00028202B4615E00022EAE7B6F52A4FECD097
:1028C000002008E02046FFF7ACFE638D9BB2FF2B93
:1028D00000D8E56A0B4836F00073E7D100902B462C
:1028E000D2B220460025FFF757FD204684F840501D
:1028F0000121FFF767FD284603B0F0BD0220FBE78A
:102900002D2F00080020008037B50446069894F863
:102910004150202D44D194F84050012D40D0012544
:1029200084F84050222584F84150102584F8425004
:10293000002565646385E0621A4B6363638D6262A0
:102940009BB2FF2B9BBF638D2385FF23E26A88BF69
:102950002385236B88BF4FF08072122B04D1AA28E5
:1029600002D0B0F52A4F09D12046FFF75AFE638DF9
:102970009BB2FF2B00D8E26A0B4B00E000230093D0
:1029800020461346002594F82820FFF705FD204631
:1029900084F840500221FFF715FD284603B030BDF2
:1029A0000220FBE72D2F000800240080F8B51F4609
:1029B00090F8413003F02803282B04460E461546B4
:1029C00001D00120F8BD01B11AB94FF4007363645E
:1029D000F7E748F20101FFF73DFD90F84030012B89
:1029E00040D0012380F8403090F841302A2B14D198
:1029F0000221FFF72FFD03681A6810040DD51A682D
:102A0000E06B22F400421A6038B1174B8363FFF782
:102A1000C5FA10B1E06B836B9847292384F84130E5
:102A200020682023002284F842306264436823F443
:102A3000004343606585638D2385E7620B4B6363C9
:102A4000836981696662C90303D51B0744BF0823F4
:102A5000C361204684F8402048F20101FFF7B2FC30
:102A60000020AFE70220ADE789360008773500087F
:102A7000F8B51F4690F8413003F02803282B044690
:102A80000E46154601D00120F8BD01B11AB94FF428
:102A900000736364F7E748F20201FFF7DBFC90F88C
:102AA0004030012B3FD090F841300121292B80F894
:102AB000401013D1FFF7CEFC03681A6850040DD5FF
:102AC0001A68A06B22F480421A6038B1174B8363F6
:102AD000FFF764FA10B1A06B836B98472A2384F840
:102AE000413020682023002284F842306264436829
:102AF00023F4004343606585638D2385E7620C4BB7
:102B00006363836981696662C90303D41B0744BF99
:102B10000823C361204684F8402048F20201FFF7F1
:102B200051FC0020B0E70220AEE700BF8936000864
:102B30007735000808B590F84120202A0AD12822CC
:102B400080F84120044A42634FF40041FFF73AFC09
:102B5000002008BD0220FCE7773500080268436BBF
:102B60009169126803B1184770477047704738B5CC
:102B7000002580F8425090F84130212B4FF020037F
:102B800080F841300AD11123036345630121FFF727
:102B900061FC80F84050FFF7E8FF38BD1223036363
:102BA00045630221FFF756FC80F84050FFF7DEFF37
:102BB000F3E708B503681A68002180F84210510451
:102BC00015D51A6822F480421A6090F84130292BFA
:102BD00013D1282380F84130212303630121FFF71B
:102BE00039FC002380F840300EF03AFC08BD120496
:102BF000EBD51A6822F40042E6E790F841302A2B20
:102C0000F4D1282380F84130222303630221FFF707
:102C100021FC002380F840300EF00FFCE6E790F82E
:102C2000412002F02802282AF8B5036834D19E69B1
:102C3000C2689D699968DF682D0C022AC6F30046B8
:102C400005F0FE051FD185EAD11515F00605C1F383
:102C500009020ED1816C01318164816C022907D196
:102C600008218564D96180F8405031460EF098FB08
:102C7000F8BD4FF40041FFF7EDFB002380F8403032
:102C800007F0FE02F1E74FF40041FFF7E3FB0023FA
:102C900080F840302A46E8E70822DA61002380F80D
:102CA0004030E5E708B5164BC362202200230363DA
:102CB000436380F8412080F842304B0712D5036807
:102CC0005A6A436A1A70436A01334362038D4BB1F7
:102CD000013B0385438D013B9BB24385436C43F02D
:102CE0000403436448F20301FFF7B4FB03681022B6
:102CF000DA61002380F840300EF08AFB08BD00BF87
:102D00000000FFFF70477047704790F84120602A2D
:102D100008B54FF0000208D1202180F8411080F85A
:102D200040200263FFF7F0FF08BD026380F84020F7
:102D30000EF09AFBF8E7000070B500223D4D90F8C8
:102D4000413080F84220C5624285426C283B0A43EC
:102D5000022B044642642AD80321FFF77BFB282379
:102D600080F84130344BA06B6363236B002841D063
:102D7000112B01D0212B3DD123681A68510442BF89
:102D80001A6822F480421A60FFF73DF901282CD01E
:102D9000A06B2A4B8363002384F84030FFF7FEF8D2
:102DA000002845D0A06B836BBDE87040184748F2FF
:102DB0000301FFF74FFBFFF7E1FA90F84130602B7A
:102DC00011D0202380F8413003689A6995060AD50E
:102DD0009A69D00605D51022DA61626C42F00402CD
:102DE00062642022DA610023BDE72046BDE870401E
:102DF000FFF78BBFE06B0028F7D0122B01D0222BFE
:102E0000F3D123681A68120442BF1A6822F4004200
:102E10001A60FFF7F8F80128E7D0E06B074B8363EF
:102E2000002384F84030FFF7B9F808B1E06BBAE747
:102E300070BD00BF0000FFFF77350008893600082D
:102E400073B505682023EB6190F84130212B0446CF
:102E50000E4635D10121FFF7FDFA112323636B687C
:102E600023F0FF7323F48B3323F4FF7323F0010368
:102E70006B6000236363F206A3F58033E36205D53C
:102E80001023EB61636C43F00403636494F84130F6
:102E9000602B05D1730741BF6B6ADBB20193019BC5
:102EA0002046FFF76BFA636C94F84120602A00D04B
:102EB0007BB1616C204602B0BDE87040FFF73CBFBB
:102EC00090F84130222BCAD10221FFF7C3FA122316
:102ED000C4E794F84120212A12D1202284F841200D
:102EE000236394F8422084F84030402A84F842302A
:102EF00003D1FFF707FF02B070BDFFF736FEFAE718
:102F000094F84120222AF6D1202284F8412023631C
:102F100094F8422084F84030402A84F8423002D1AC
:102F2000FFF7F1FEE7E7FFF721FEE4E773B590F85E
:102F30004030012B04460D46164600F091800123D7
:102F4000CA0680F8403017D5F30615D5036810225D
:102F5000DA61436C43F004034364FFF70FFAAA06F7
:102F600005D5B30603D529462046FFF769FF0020A3
:102F700084F8400002B070BD680712D5710710D503
:102F800023685A6A636A1A70636A25F0040501337C
:102F90006362238D013B2385638D013B9BB2638577
:102FA000DDE76A060DD4AB0727D5B00725D5638DBD
:102FB0009BB2002BD3D0636A226813F8011B916285
:102FC000E6E7290606F0400337D5002BC7D0638D0E
:102FD00022689BB22BB3208D18BB5168638D9BB2C6
:102FE000FF2BC1F309010DD9FF2222854FF0807319
:102FF00000902046FFF7D0F9B1E72A06AFD5730657
:10300000E5D4ACE7628DE36A92B213F5803F228586
:10301000D2B202D0E36A0090EBE700904FF0007369
:10302000E7E75368980103D42046FFF7A0FD96E731
:1030300040212046FFF780FE91E7002B8FD0638D63
:103040009BB2002BF4D123685A68910187D4E26ABD
:1030500012F5803FE8D15A6842F480425A607EE718
:10306000022087E713B590F84030012B044600F0AA
:103070008580012380F84030CB0612D5D30610D5C9
:1030800003681022DA61436C43F004034364202197
:10309000FFF798F9FFF772F9002084F8400002B0BA
:1030A00010BD880708D5930706D52368226D9A625C
:1030B0004FF0FF332365EFE7080633D5530631D5CC
:1030C00010212046FFF77EF9638D9BB233B3638DE9
:1030D0009BB2FF2B18D90023FF22E16C22850093BD
:1030E0004FF0807389B2FFF757F9638D228D9B1AD9
:1030F0009BB2638594F841202368222A1A6832D152
:1031000042F400421A60C7E7628DE16C92B200237C
:1031100022850093D2B24FF00073E3E74021FFF71E
:103120000BFEB9E7480621D553061FD594F8411088
:10313000134A144B222918BF1346628D92B2FF2AFC
:1031400008D9FF22E16C228500934FF0807389B289
:103150002046C8E7628DE16C92B222850093D2B21C
:103160004FF00073F3E742F48042CBE7880693D533
:10317000930691D52046FFF763FE8DE702208EE788
:10318000002000800024008073B590F84030012BAF
:10319000044678D0012380F84030CB0612D5D606FD
:1031A00010D503681022DA61436C43F004034364D2
:1031B0002021FFF707F9FFF7E1F8002084F840002D
:1031C00002B070BD0D0641D550063FD525682B686D
:1031D00023F040032B60638D9BB25BB36968638D02
:1031E0009BB2FF2BC1F309011AD9FF2323854FF0AE
:1031F00080730022268D009294F828202046FFF745
:10320000CBF8638D9B1B9BB2638594F84130222BD6
:103210002B680CBF43F4004343F480432B60CCE79E
:10322000638D2385E36A13F5803F14BFE36A4FF093
:103230000073DEE76B689A0103D42046FFF797FC22
:10324000BBE740212046FFF777FDB6E74B0612D5D6
:10325000560610D5638D9BB2002BF2D123685A68B5
:103260009501AAD4E26A12F5803FE6D15A6842F489
:1032700080425A60A1E788069FD593069DD52046D7
:10328000FFF7DEFD99E702209AE7036899691A685B
:1032900010B4CC0508D5140606D5446C44F00104DE
:1032A00044644FF48074DC614C0508D5140606D5DF
:1032B000446C44F0080444644FF48064DC61890584
:1032C00008D5120606D5426C42F0020242644FF461
:1032D0000072DA61416C11F00B0F02D010BCFFF7E5
:1032E0002BBD10BC704700002DE9F8430568D5F8E8
:1032F0000090D0F82C8090F8417007F0F707202359
:10330000212F04460E46EB6164D148F20101FFF71C
:10331000A1F827636B6843F400436B606B6823F08C
:10332000FF7323F48B3323F4FF7323F001036B60EB
:103330002046FFF723F819F4804F50D02B6823F470
:1033400080432B60A36B1BB11B685B689BB26385DA
:1033500072070FD5636A6A6A1A70636A013363621F
:10336000238D2BB1013B2385638D013B9BB263858C
:1033700026F00406638D9BB21BB1636C43F004031B
:103380006364F30611D519F0100F0ED0638D9BB254
:10339000002B3ED194F84130282B29D1B8F1007F81
:1033A00026D131462046FFF77DFC002384F84230C9
:1033B000656C6363002D3BD0616C2046FFF7BCFC5D
:1033C00094F84130282B45D131462046BDE8F843DA
:1033D000FFF768BC222F9DD148F2020197E719F44C
:1033E000004FB5D02B6823F400432B60E36BAAE7B2
:1033F00094F841202368292A4FF01002DA61D4D1D1
:1034000018F5803FD1D02046FEF7B8FFFFF7D1FB7B
:10341000CBE723681022DA61636C43F00403636432
:1034200038F08073C1D1616C2046FFF785FCBCE7A2
:10343000E36A13F5803F0FD02046FFF7BAFB0F4B2E
:10344000E362202384F8413084F84050256320460D
:103450000DF0DEFFBDE8F88394F8413084F8405069
:10346000222B4FF0200384F841302046256302D1FF
:103470000DF0E3FFEEE70DF0F3FFEBE70000FFFFD9
:1034800070B590F84060C56A012E04460B4670D0B6
:10349000012680F840608E0607D5960605D5FFF711
:1034A00023FF002084F8400070BDD80659D5D1060E
:1034B00057D512F4404F50D0D4E90E10E0B921B1E5
:1034C000520402D50A6852680AB323681022DA61EE
:1034D000636C43F00403636494F8413035F0807208
:1034E000DBB2DED1213B092B30D8DFE803F02D34ED
:1034F0002F2F2F2F2F2F2D341604E0D50068406872
:103500000028DCD119B1500444BF0A68526894F80D
:103510004120282A07D1B5F1007F04D11946204661
:10352000FFF7C0FBBDE794F841202368292A4FF03C
:103530001002DA61B5D115F5803FB2D02046FEF712
:103540001DFFFFF736FBACE721232363616C2046A8
:10355000FFF7F2FBA5E72223F7E723681022DA61E1
:103560009FE719079DD513079BD52046FFF757FB0B
:1035700097E7022098E770B590F84060C56A012E81
:1035800004460B467ED0012680F840608E0607D5A3
:10359000960605D5FFF7A8FE002084F8400070BD10
:1035A000D90630D5D6062ED5628D92B2E2B994F8FE
:1035B0004120282A07D1B5F1007F04D119462046C1
:1035C000FFF770FBE8E794F841202368292A4FF0C1
:1035D0001002DA61E0D115F5803FDDD02046FEF71C
:1035E000CDFEFFF7E6FAD7E723681022DA61636CB5
:1035F00043F00403636435F08073CDD1616C2046E1
:10360000FFF79AFBC8E758071BD5510719D5638DFB
:103610009BB26BB123685A6A636A1A70636A01339A
:103620006362238D013B2385638D013B9BB26385E0
:10363000638D9BB2002BAFD115F5803FACD02046F7
:10364000CFE71E0705D5100703D52046FFF7E7FA99
:10365000A2E79907A0D593079ED5638D9BB26BB166
:10366000636A226813F8011B91626362638D013BF8
:103670009BB26385238D013B23858DE735F08073F5
:103680008AD1DCE702208AE7806A836B0BB10022D3
:103690009A63C36B0BB100229A63FFF736BB90F8B5
:1036A00041007047406C7047024A136843F48073CE
:1036B0001360704700040058024B186800F4C060A3
:1036C000704700BF00040058024A936823F4004387
:1036D0009360704700040058054A136843F00703DD
:1036E0001360044A136943F00403136130BF704749
:1036F0000004005800ED00E04FF0B0431868C0F33C
:10370000404070474FF0B0431868C0F34000704726
:103710004FF0B042536823F47F4343EA00235360E1
:1037200070474FF0B0431868C0F340607047000026
:103730007FB54FF0B0432C4AD3F80831C0F30310E3
:1037400003F00F0352F82040284A52F82330B4FB0C
:10375000F3F4FFF7B1FF264B054693E80700B5F5F4
:10376000007F04AB03E9070010D0224B9C4218D322
:1037700003F5B70303F67F539C4229D903F574136D
:1037800003F510639C4225D802230BE01A4B9C42A0
:1037900007D91A4B9C421BD903F5370303F5D853BD
:1037A000F0E7002304AA02EB830353F80C4C144DFA
:1037B0002B6823F0070323432B60FDF76FFE0646BB
:1037C0002B6803F007039C4206D1002004B070BDB3
:1037D0000123E7E70024EAE7FDF760FE801B0228EB
:1037E000EED90320F2E700BFF4680208546902082A
:1037F000D8620208C0CF6A00BFEA21013F933402B9
:10380000004000584FF0B04310B59A68D96812F0E4
:103810000C0205D00C2A4AD101F00303012B51D12F
:103820004FF0B0412B480B6813F0080306D00B682B
:1038300013F0080337D1D1F8941007E00C6824077F
:1038400056BFD1F894300968C3F3032350F82330EE
:10385000002A0CBF184600204FF0B0418A6802F0E1
:103860000C020C2A1ED1CA6802F00302022A2ED0D2
:10387000032A06D10B68184A13F4801F174B18BF90
:1038800013464FF0B042D068D168D268C0F306202A
:103890005843C1F302130133B0FBF3F0530F01336C
:1038A000B0FBF3F010BD0B68C3F30313CEE7042A9B
:1038B00005D0082A06D11B6813F4801305D00648EA
:1038C0000023C9E700231846C6E70448C4E7024BB3
:1038D000D7E700BFF46802080024F4000048E801BC
:1038E00008B5FFF78FFF4FF0B043044A9B68C3F35E
:1038F000031352F82330B0FBF3F008BD54690208FB
:103900002DE9F0410446002853D04FF0B0439D68A4
:10391000DE680368990605F00C0506F0030668D515
:10392000026A1DB10C2D46D1012E44D1002A40D08F
:103930004FF0B043A16A1A68120756BFD3F894300B
:103940001B681B0903F0F00399421FD90846FFF7D3
:10395000EFFE00282DD14FF0B042136843F008036A
:1039600013601368A16A23F0F0030B431360606ACD
:10397000FFF7CEFEFFF7B4FFAC4B1860AC4B1868F6
:10398000FDF744FD002834D0BDE8F0814FF0B0428F
:10399000136843F008031360136823F0F0030B432C
:1039A0001360606AFFF7B4FE0846FFF7C1FE002807
:1039B000E0D00120E8E74FF0B043002A54D01A6865
:1039C00042F001021A60FDF769FD0746FFF79AFE13
:1039D000002842D04FF0B042136843F00803136050
:1039E0001368A16A23F0F0030B431360606AFFF7CA
:1039F0008FFE2368DF0748D42368980700F1A18071
:103A000023681E0740F1FC80A3694FF0B046002BED
:103A100000F0E380D6F89430E16903F0100291429F
:103A200000F0C68003F00302022AC2D0D80740F19A
:103A3000B580D6F8943023F00103C6F89430FDF732
:103A40002DFD0746D6F89430990740F1A780FDF781
:103A500025FDC31B112BF5D904E0FDF71FFDC01B8D
:103A60000228B3D903208FE71A6822F001021A60F6
:103A7000FDF714FD0746FFF745FE0028B9D0FDF716
:103A80000DFDC01B0228F6D9ECE7082D626803D0B3
:103A90000C2D1AD1032E18D1002A8AD09907AFD540
:103AA00023694FF0B046002B67D0336843F480732E
:103AB0003360FDF7F3FC074633685A0555D4FDF72C
:103AC000EDFCC31B022BF7D9CCE74FF0B043A06845
:103AD000196821F480110143B2F5803F196010D1BB
:103AE0001A6842F480321A60FDF7D8FC0746FFF7E7
:103AF00003FE002880D1FDF7D1FCC01B6428F6D955
:103B0000B0E7B2F5041F04D11A6842F400121A603B
:103B1000E6E7196821F480311960196821F4001171
:103B20001960002AE0D1FDF7B9FC0746FFF7E4FD74
:103B300000283FF461AFFDF7B1FCC01B6428F5D944
:103B400090E7042D03D00C2DAAD1022EA8D1236911
:103B5000002B3FF42EAF4FF0B0426169536823F061
:103B6000FE4343EA016353604AE77368626923F0E6
:103B7000FE4343EA0263736042E7336823F48073D1
:103B80003360FDF78BFC074633685B057FF538AF84
:103B9000FDF784FCC31B022BF6D963E74FF0B0425C
:103BA000E169D2F8943023F010030B43C2F894304B
:103BB0004FF0B047D7F8943043F00103C7F8943082
:103BC000FDF76CFC0646D7F894309A0718D4FDF739
:103BD00065FC831B112BF6D944E7D6F8943023F00B
:103BE0000103C6F89430FDF759FC0746D6F8943027
:103BF0009B0705D5FDF752FCC31B112BF6D931E706
:103C00002368580754D50B4F3B68D90514D4FFF7E8
:103C10004BFDFDF743FC06463B68DA050CD4FDF787
:103C20003DFC831B022BF7D91CE700BF400000209E
:103C30000400002000040058E3684FF0B046002B59
:103C400058D023F08003052B02BFD6F8903043F004
:103C50000403C6F890304FF0B046FDF71FFCD6F8CD
:103C6000903043F001030746C6F8903041F288389F
:103C7000D6F890309B0705D4FDF710FCC31B4345D5
:103C8000F6D9EFE6E36823F00403812B1BD1FDF79F
:103C900005FCD6F8903043F08003C6F89030074614
:103CA0004FF0B04641F28838D6F89030180504D568
:103CB000E36A002B4AD1002066E6FDF7EFFBC01B4C
:103CC0004045F1D9CEE6FDF7E9FBD6F8903023F078
:103CD0008003C6F8903007464FF0B04641F288386E
:103CE000D6F890301905E3D5FDF7D8FBC01B404549
:103CF000F6D9B7E6FDF7D2FBD6F8903023F0800373
:103D00000746C6F8903041F28838D6F890301A0548
:103D100016D4FDF7C3FBD6F8903023F00103C6F8A4
:103D2000903007464FF0B04841F28836D8F89030CE
:103D30009B07BDD5FDF7B2FBC31BB342F6D991E695
:103D4000FDF7ACFBC01B4045DFD98BE60C2D4ED0F8
:103D5000022B4FF0B0431A6822F080721A6033D100
:103D6000FDF79CFB0546FFF7DCFC38BBD4E90C31C2
:103D70004FF0B0420B43D0682D4901400B43E16B3B
:103D80000B43216C0B43616C0B43A16B43EA012392
:103D9000D360136843F080731360D36843F080539B
:103DA000D360FDF77BFB0446FFF7BBFC002882D104
:103DB000FDF774FB001B0A28F6D953E6FDF76EFBEE
:103DC000401B0A28CFD94DE6FDF768FB0446FFF7F4
:103DD000A8FC30B94FF0B042164BD1680B40D3600D
:103DE00069E7FDF75BFB001B0A28F0D93AE6012BD7
:103DF0003FF4DFAD4FF0B043D868236B00F003020F
:103E00009A427FF4D6AD626B00F0700393427FF468
:103E1000D0ADA26B00F4FE43B3EB022F7FF4C9AD2B
:103E2000636C00F06040C01A18BF0120ACE500BF11
:103E30008C80C111FCFFFEEE2DE9F0410D460446D9
:103E400010B90120BDE8F081684E336803F0070324
:103E50008B4216D323689A0727D54FF0B047A26844
:103E6000BB6823F0F0031343BB60FDF717FB064666
:103E7000BB68DB0319D4FDF711FB831B022BF7D9B9
:103E800011E0336823F007030B433360FDF706FBB3
:103E90000746336803F00703AB42DBD0FDF7FEFAB9
:103EA000C01B0228F5D90320CCE72368580617D594
:103EB0004FF0B0476269D7F8083123F00F0343EAA7
:103EC0001213C7F80831FDF7E9FA0646D7F80831AA
:103ED000D90305D4FDF7E2FA831B022BF6D9E2E7FA
:103EE00023685A0713D54FF0B047E268BB6823F444
:103EF000E0631343BB60FDF7D1FA0646BB689B0342
:103F000005D4FDF7CBFA831B022BF7D9CBE7236847
:103F1000180714D54FF0B0472269BB6823F46053EB
:103F200043EAC203BB60FDF7B9FA0646BB68590312
:103F300005D4FDF7B3FA831B022BF7D9B3E7236847
:103F4000DA070FD4294C236803F00703AB4239D8B2
:103F5000FFF7C6FC264B1860264BBDE8F0411868F9
:103F6000FDF754BA6268022A1DD1FFF7C5FB00288D
:103F70003FF467AF4FF0B04641F28838B36823F0A2
:103F800003031343B360FDF789FA0746B368626819
:103F900003F00C03B3EB820FD4D0FDF77FFAC01B04
:103FA0004045F3D97FE7032A02D1FFF7BAFBDEE7EA
:103FB00012B9FFF7A7FBDAE74FF0B0431B685B05C8
:103FC000D8D43EE7236823F007032B432360FDF793
:103FD00065FA0646236803F00703AB42B8D0FDF745
:103FE0005DFA801B0228F5D95DE700BF004000584C
:103FF000400000200400002008B5FFF703FC4FF04C
:10400000B043054AD3F8083103F00F0352F82330C8
:10401000B0FBF3F008BD00BF5469020808B5FFF714
:104020005FFC4FF0B043044A9B68C3F3022352F88D
:104030002330D84008BD00BF3469020808B5FFF737
:104040004FFC4FF0B043044A9B68C3F3C22352F8BD
:104050002330D84008BD00BF3469020810B5D8B17C
:10406000D1B14F234FF0B0420360936803F00C04CA
:10407000446003F0F004846003F4E06403F46053EC
:10408000C4600361D2F808311B01DBB24361034B0A
:104090001B6803F007030B6010BD00BF0040005811
:1040A0004FF0B0431868C0F3802070474FF0B04322
:1040B000D3F89000C0F3400070474FF0B043D3F8FE
:1040C0009400C0F3400070474FF0B0431868C0F34D
:1040D000C00070474FF0B04210B5D36803F003033F
:1040E000022B39D0032B10D0FFF7EEFF1B4C0146FB
:1040F00028BBFFF7E9FF012816BFD2F89410136818
:10410000C1F3032154F8213006E01368144A13F474
:10411000801F144B18BF13464FF0B042D068D168CF
:10412000D268C0F306204343C1F30211C2F34260D8
:1041300001310130B3FBF1F3B3FBF0F010BDFFF739
:10414000C3FF01280BBF1368D2F89430C3F30313E5
:10415000002354F82330DFE7014BDDE7F468020861
:104160000024F4000048E801B0F5807F10B500F0AD
:104170008F8123D8202800F0FA800AD8022800F086
:10418000D680102800F09481012800F0A78000203C
:1041900010BD402800F057818028F8D14FF0B0447E
:1041A000B24AD4F888301B0903F4406343F4402337
:1041B000934200F0A48002F5806253E1B0F5804F95
:1041C00000F0E58027D8B0F5806F00F08981B0F568
:1041D000006F00F0A281B0F5007FD8D14FF0B0435E
:1041E000A34AD3F888301B0C03F00C0343F440239C
:1041F000934200F0DC80B3F10C1F22D0043A9342CA
:1042000040F06781FFF759FF0128C0D14FF0B0435C
:10421000D3F8943022E0B0F5004F25D0B0F5803FC0
:10422000B5D14FF0B042D2F8903003F44073B3F5FB
:10423000007F0DD0B3F5407F00F08581B3F5807F1E
:10424000A5D1FFF733FF441E60426041C0039FE7E2
:10425000FFF733FF01289AD1D2F89430D80654BF23
:104260004FF4FA40FA2093E74FF0B042D2F888308A
:1042700003F04043B3F1804FEAD0B3F1004FE0D0F8
:1042800033B91368990182D5BDE81040FFF722BF0A
:1042900013689A077FF57BAFFFF716FF7549024653
:1042A00068B9FFF711FF4FF0B043012816BFD3F8EC
:1042B00094201B68C2F3032251F8220068E7FFF73D
:1042C00003FF4FF0B04301280BBF1B68D3F89430B5
:1042D000C3F30313002351F8230059E74FF0B04311
:1042E000654AD3F8883003F0030343F44033934224
:1042F0005DD0B3F1031FA4D0013A934203D1BDE8CE
:104300001040FFF77FBAFFF77DFA4FF0B0435B49EB
:104310009A689B68C2F30312C3F3C22351F82220A8
:10432000B0FBF2F0564A52F82330D84030E74FF055
:10433000B0444F4AD4F8883003F00C0343F44023D0
:10434000934234D0B3F10C1F3FF47BAF043A934255
:10435000D5D0FFF757FAA268A3684849C2F3031201
:10436000C3F3022351F82220B0FBF2F0DAE74FF05A
:10437000B044D4F8883003F44063B3F5006F16D02E
:10438000B3F5406F3FF45DAFB3F5806FE0E74FF0FA
:10439000B042D2F8883003F04053B3F1005F0DD043
:1043A000B3F1405FABD0B3F1805F7FF4F0AEFFF7C5
:1043B00077FE01287FF4EBAE3248E9E613689B01F3
:1043C0007FF5E5AED36803F00303022B39D0032B4E
:1043D00010D0FFF779FE274C014628BBFFF774FE8B
:1043E000012816BFD2F894101368C1F3032154F8C2
:1043F000213006E01368234A13F4801F224B18BFB4
:1044000013464FF0B042D068D168D268C0F306209E
:104410005843C1F302130133B0FBF3F0C2F344433A
:104420000133B0FBF3F0B3E6FFF74EFE01280BBFFC
:104430001368D2F89430C3F30313002354F82330E5
:10444000DFE7104BDDE74FF0B044104AD4F8883076
:104450001B0903F4407343F4403393423FF44FAFDE
:1044600002F580729342A2D073E700BF00040C00F3
:1044700008000C00F46802080200030054690208F6
:10448000346902080024F4000048E8010001030038
:104490004FF0B0442D4AD4F888301B0903F4405340
:1044A00043F4401393423FF42AAF02F58052D9E718
:1044B0004FF0B043D3F8883003F44073B3F5007F76
:1044C0003FF475AFB3F5407F7FF4DEAE4BF680303E
:1044D0005EE6FFF797F94FF0B0439A689B683CE7B8
:1044E0004FF0B0441A4AD4F888301B0C03F0300364
:1044F00043F4401393423FF45AAFB3F1301F3FF4FB
:10450000A0AE103A93427FF424AFFFF7D6FD012806
:104510007FF43DAED4F89430A0E64FF0B0440D4A9D
:10452000D4F888301B0C03F0C00343F440039342DB
:104530003FF43DAFB3F1C01F3FF483AE403A934226
:104540007FF407AF5EE6044822E600BF00103000AB
:10455000200030008000C00040420F00704770B55E
:104560000446002866D0436A002B5FD14268B2F54A
:10457000827F00D0C3610023A36294F85D3003F012
:10458000FF0223B984F85C202046FFF7E7FF22688A
:10459000E068A668A169022384F85D30136823F0FF
:1045A00040031360B0F5E06F4FF000038ABF1D4673
:1045B0004FF48055B0F5706F18BFA362636806F4BE
:1045C000044603F482733343266906F0020633433C
:1045D000666906F00106334301F400763343E66969
:1045E00006F038063343266A06F080063343A66A8F
:1045F00006F4005633431360666B636A06F00806E0
:1046000003F0100300F470603343090C034301F01E
:1046100004010B432B435360D36923F40063D3613C
:1046200000200123206684F85D3070BD0023C0E9BE
:104630000433A0E70120F8E7704710B5044680B1C5
:104640000268022380F85D30136823F04003136092
:10465000FFF7F2FF0020206684F85C0084F85D001C
:1046600010BD0120FCE7022310B580F83D3003683F
:10467000196A41F211121142044608D1196A40F236
:104680004442114202BF1A6822F001021A60204619
:1046900002F0FFFC002084F8480084F83C0084F815
:1046A0003E0084F83F0084F8400084F8410084F81C
:1046B000420084F8430084F8440084F8450084F8FC
:1046C000460084F8470084F83D0010BD90F83D3066
:1046D000012B17D102230C4A80F83D300368934226
:1046E00002D0B3F1804F07D19968084A0A40062AE0
:1046F00006D0B2F5803F03D01A6842F001021A607A
:104700000020704701207047002C01400700010085
:104710000368196A41F21112114208D1196A40F274
:104720004442114202BF1A6822F001021A600123BA
:1047300080F83D30002070470368DA6822F00102FB
:10474000DA60196A41F21112114208D1196A40F275
:104750004442114202BF1A6822F001021A6001238A
:1047600080F83D300020704790F83C20012A034635
:104770004FF0020009D01A6883F83D005161002013
:10478000012283F83D2083F83C0070477047704752
:10479000036870B5DD681E69B20704460DD5A90728
:1047A0000BD56FF002021A61012202779B699A070A
:1047B00074D001F052FE00232377730710D56807E9
:1047C0000ED523686FF004021A61022222779B69DA
:1047D00013F4407F204667D001F03FFE002323778B
:1047E00031070FD52A070DD523686FF008021A612B
:1047F00004222277DB699B0720465BD001F02DFE67
:1048000000232377F00610D5E9060ED523686FF054
:1048100010021A6108222277DB6913F4407F2046D8
:104820004ED001F01AFE00232377F20708D5EB07DC
:1048300006D523686FF001021A61204601F0EAFDF7
:10484000300608D5290606D523686FF080021A6164
:10485000204600F002FAF20508D52B0606D523689B
:104860006FF480721A61204600F0F8F9700608D5DE
:10487000690606D523686FF040021A612046FFF7EB
:1048800086FFB20622D5AB0620D523686FF0200242
:1048900020461A61BDE8704000F0DEB901F0DBFD92
:1048A0002046FFF773FF86E701F0D5FD2046FFF7AE
:1048B0006DFF93E701F0CFFD2046FFF767FF9FE70D
:1048C00001F0C9FD2046FFF761FFACE770BD0000B5
:1048D0001B4A0368904202D0B0F1804F08D14A6869
:1048E00023F070031343CA6823F44073134306E0B4
:1048F000144A9042F7D002F580629042F3D04A69A0
:1049000023F08003134303608B68C3620B688362E8
:104910000B4B984207D003F5C053984203D003F5E0
:104920008063984201D10B690363012343610369EA
:10493000DB0742BF036923F001030361704700BF37
:10494000002C01400044014010B5044650B390F8DB
:104950003D3003F0FF021BB980F83C2002F072FBEF
:104960000223206884F83D30211DFFF7B1FF0123A9
:1049700084F84830002084F83E3084F83F3084F8D2
:10498000403084F8413084F8423084F8433084F871
:10499000443084F8453084F8463084F8473084F851
:1049A0003D3010BD0120FCE7036A01F01F0110B586
:1049B00001248C4023EA04030362036A8A401A43F9
:1049C000026210BD082908B525D00AD8A9B104296A
:1049D00019D090F84330012B13D1022380F84330D3
:1049E0002CE00C291FD01029F3D190F84230012B74
:1049F00007D1022380F8423020E090F83E30012BAE
:104A000019D0012043E090F83F30012BF9D1022367
:104A100080F83F3012E090F84030012BF1D10223B2
:104A200080F840300AE090F84130012BE9D10223B0
:104A300080F8413002E0022380F83E300068012215
:104A4000FFF7B2FF124B984214D003F5C0539842BF
:104A50000BD003F58063984207D0B0F1804F0DD0A2
:104A6000036843F00103036010E0436C43F4004328
:104A70004364F5E7436C43F4004343648268054BA9
:104A80001340062B02D0B3F5803FE9D1002008BDCA
:104A9000002C014007000100FFF794BF082910B562
:104AA00003465AD010D809B3042946D093F843409E
:104AB00093F84720012CE0B2D2B26FD1012A3BD14A
:104AC000022283F8432065E00C2956D01029EDD14D
:104AD00090F8424093F84720012CE0B2D2B25DD169
:104AE000012A29D1022283F8422053E090F83E4067
:104AF00093F84420012CE0B2D2B24FD1012A1BD14D
:104B0000022283F83E2083F8442018680122FFF730
:104B10004BFF234B984202D0B0F1804F07D18268FF
:104B2000204B1340062B06D0B3F5803F03D003681B
:104B300043F001030360002010BD90F83F4093F85C
:104B40004520012CE0B2D2B228D1012AF4D10222B0
:104B500083F83F2083F84520D7E790F8404093F84A
:104B60004620012CE0B2D2B218D1012AE4D10222AF
:104B700083F8402083F84620C7E790F8414093F837
:104B80004720012CE0B2D2B208D1012AD4D10222AE
:104B900083F84120022283F84720B6E70120CBE7C3
:104BA000002C014007000100036A01F01F0110B54D
:104BB00004248C4023EA04030362036A8A401A43F4
:104BC000026210BD08B529B990F84430012B1DD000
:104BD000012039E0042907D190F84530012BF7D1A5
:104BE000022380F8453014E0082907D090F84730B8
:104BF000012BEDD1022380F847300AE090F84630CF
:104C0000012BE5D1022380F8463002E0022380F830
:104C1000443000680422FFF7C7FF436C43F40043AD
:104C200043640A4B984202D0B0F1804F07D18268AA
:104C3000074B1340062B06D0B3F5803F03D0036823
:104C400043F001030360002008BD00BF002C0140B9
:104C500007000100FFF7B6BF7047704770470000BC
:104C600010B5026852E8003F23F4907342E8003127
:104C700002680029F5D10F4C02F1080353E8003F08
:104C8000234002F1080C4CE800310029F4D1C36E36
:104C9000012B07D152E8003F23F0100342E8003116
:104CA0000029F7D12023C0F88C300023C366436766
:104CB00010BD00BFFEFFFFEF026852E8003F23F087
:104CC000800342E8003102680029F5D152E8003F34
:104CD00043F0400342E800310029F7D17047D0F893
:104CE0008820212A034611D1B0F8562092B20AB981
:104CF000FFF7E2BF026D016812F8010B88621A65C6
:104D0000B3F85620013A92B2A3F856207047D0F873
:104D10008820212A034613D1B0F8562092B20AB94E
:104D2000FFF7CABF1A6D006832F8021BC1F3080111
:104D300081621A65B3F85620013A92B2A3F8562060
:104D40007047D0F88830212B10B51BD1B0F86A20FD
:104D5000C2B1B0F85610036889B2A1B903F10802D4
:104D600052E8002F22F4000203F1080040E800217D
:104D70000029F3D153E8002F42F0400243E800211C
:104D80000029F7D110BDD96909060AD5016D11F8BE
:104D9000014B9C62B0F856300165013B9BB2A0F814
:104DA0005630013A92B2D3E7D0F88830212B10B5B3
:104DB0001BD1B0F86A20C2B1B0F85610036889B2AE
:104DC000A1B903F1080252E8002F22F4000203F116
:104DD000080040E800210029F3D153E8002F42F0F9
:104DE000400243E800210029F7D110BDD969090626
:104DF0000CD5016D31F8024BC4F308049C62B0F885
:104E000056300165013B9BB2A0F85630013A92B290
:104E1000D1E77047D0F88830202B10B544D1002955
:104E200044D0002A42D0A0F85620A0F85420426E68
:104E300001650023C0F89030B2F1005F4FF021030C
:104E4000C0F888300268836819D1B3F5805F14D147
:104E50000469174B1749002C08BF0B46836702F102
:104E6000080353E8003F43F4000302F1080040E860
:104E700000310029F3D1002010BD0D4BEEE7B3F552
:104E8000805F0FD104690C4B0C49002C08BF0B4606
:104E9000836752E8003F43F0800342E80031002975
:104EA000F7D1E8E7044BF3E70220E5E70120E3E769
:104EB000434D0008A94D0008DF4C00080F4D0008C5
:104EC00008B5806A0023A0F85E30A0F8563002F0E2
:104ED00015FC08BD704700000368D9691A682DE900
:104EE000F04140F60F0631429D68044610D18E060F
:104EF00040F1978002F0200605F080573E4300F015
:104F00009080436F002B00F08580BDE8F04118478A
:104F1000AB4EAC482E401040304300F08280CF07AB
:104F200009D5D00507D501201862D4F8900040F0CB
:104F30000100C4F890008F0709D5E80707D50220C3
:104F40001862D4F8900040F00400C4F890004F07B5
:104F500009D5E80707D504201862D4F8900040F07E
:104F60000200C4F890000F070BD502F02000304378
:104F700007D008201862D4F8900040F00800C4F868
:104F800090000E050AD5500108D54FF40060186254
:104F9000D4F8903043F02003C4F89030D4F8903027
:104FA000002B37D08B0609D502F0200205F0805582
:104FB0002A4303D0636F0BB1204698472668D4F884
:104FC0009020B36802F0280203F0400353EA020580
:104FD000204621D0FFF744FEB3685F0617D522684C
:104FE00002F1080353E8003F23F04003083242E88F
:104FF00000310029F3D1D4F8800040B1724B8363B3
:10500000FCF7CCFF30B1D4F88000836B7DE72046FD
:1050100002F074FBBDE8F08102F070FBC4F8905020
:10502000F8E7E06E012840F08980CE0640F18680E6
:10503000D00640F1838010221A629A6851064BD53F
:10504000D4F8802011684A6892B2002AE2D0B4F8FD
:105050005C009042DED9A4F85E200A6892062FD444
:1050600053E8002F22F4807243E800210029F7D191
:1050700003F1080252E8002F22F0010203F10800B8
:1050800040E800210029F3D103F1080252E8002F83
:1050900022F0400203F1080040E800210029F3D18A
:1050A0002022C4F88C20E16653E8002F22F0100281
:1050B00043E800210029F7D1D4F88000FCF739FF3C
:1050C00002232367B4F85E30B4F85C10C91A89B2C1
:1050D0002046FFF7FFFE9DE7B4F85E20B4F85E00BF
:1050E000B4F85C1080B292B2002893D0891A89B2C9
:1050F00000298FD053E8002F22F4907243E800205B
:105100000028F7D1314D03F1080252E8002F2A4060
:1051100003F1080646E800200028F4D12022C4F854
:105120008C206067E06653E8002F22F0100243E80D
:1051300000200028F7D102232367C9E7CF0209D551
:105140006E0207D54FF4801220461A62BDE8F04186
:1051500002F01EBB08060BD502F0800005F4000526
:10516000284305D0A36F002B3FF454AF2046CCE674
:105170004F0611D556060FD553E8002F22F04002F6
:1051800043E800210029F7D12023C4F88830A16723
:10519000204602F0AFFA3DE70D0206D5500004D5D7
:1051A0002046BDE8F04100F032BECB017FF532AFC2
:1051B000002ABFF62FAF2046BDE8F04100F026BE22
:1051C0000100001020010004C14E0008FEFFFFEFA7
:1051D000D0F88C20B0F86010222A08B5036855D1A9
:1051E0005B6A826D0B401370836D01338365B0F889
:1051F0005E30013B9BB2A0F85E30B0F85E309BB2EF
:10520000002B42D1026852E8003F23F4907342E839
:10521000003103680029F5D103F1080252E8002F9C
:1052200022F0010203F1080C4CE800210029F3D11F
:105230002022C0F88C20184A41679342016705D1AB
:10524000C26E012A0ED002F051FA1EE05A68110215
:10525000F6D553E8002F22F0806243E800210029B0
:10526000F7D1EDE70022C26653E8002F22F01002CA
:1052700043E800210029F7D1DA69B0F85C10D206C2
:1052800044BF10221A62FFF725FE08BD9A6942F05A
:1052900008029A61F9E700BF00800040D0F88C2036
:1052A000B0F86010222A08B5036852D15A6A11403A
:1052B000826D22F8021B8265B0F85E20013A92B23C
:1052C000A0F85E20B0F85E2092B2002A40D153E8E8
:1052D000002F22F4907243E800210029F7D103F156
:1052E000080252E8002F22F0010203F1080C4CE8FA
:1052F00000210029F3D12022C0F88C20174A4167F1
:105300009342016705D1C26E012A0ED002F0EEF978
:105310001EE05A681102F6D553E8002F22F0806291
:1053200043E800210029F7D1EDE70022C26653E8E7
:10533000002F22F0100243E800210029F7D1DA699A
:10534000B0F85C10D20644BF10221A62FFF7C2FD0B
:1053500008BD9A6942F008029A61F9E700800040AE
:105360002DE9F84F0368B0F86060D3F81CB01F68EF
:105370009D68D0F88C20222A044640F0B980B0F80D
:10538000683043B1DFF87491DFF874A14FF0000882
:105390001BF0200F20D1B4F85E309BB2D3B1B4F82B
:1053A00068209A4216D9226802F1080353E8003FA8
:1053B00023F08053083242E8003122680029F2D1FC
:1053C000504B636752E8003F43F0200342E800314E
:1053D0000029F7D1BDE8F88F2368A26D5B6A3340DE
:1053E0001370A36D0133A365B4F85E30013B9BB22B
:1053F000A4F85E302368D3F81CB01BF0070F2ED042
:105400001BF0010F09D0F90507D501221A62D4F863
:10541000902042F00102C4F890201BF0020F09D046
:10542000EA0707D502221A62D4F8902042F004025B
:10543000C4F890201BF0040F09D0E80707D5042218
:105440001A62D4F8903043F00203C4F89030D4F8D4
:10545000903023B1204602F051F9C4F89080B4F89E
:105460005E309BB2002B93D1226852E8003F23F4B8
:10547000807342E8003123680029F5D103F1080266
:1054800052E8002F02EA090203F1080040E8002177
:105490000029F3D120225345C4F88C20616721678D
:1054A0000AD05A68110207D553E8002F22F0806213
:1054B00043E800210029F7D1E26E012A14D100222D
:1054C000E26653E8002F22F0100243E80021002991
:1054D000F7D1DA69B4F85C10D20644BF10221A6220
:1054E0002046FFF7F7FC53E7204602F0FFF84FE7AE
:1054F0009A6942F008029A616CE700BFFEFFFFEF75
:1055000000800040D15100082DE9F84F0368B0F841
:105510006060D3F81CB01F689D68D0F88C20222AE8
:10552000044640F0B780B0F8683043B1DFF87091BE
:10553000DFF870A14FF000081BF0200F20D1B4F865
:105540005E309BB2D3B1B4F868209A4216D9226873
:1055500002F1080353E8003F23F08053083242E889
:10556000003122680029F2D14F4B636752E8003FB7
:1055700043F0200342E800310029F7D1BDE8F88F5D
:105580002368A26D596A314022F8021BA265B4F863
:105590005E20013A92B2A4F85E20D3F81CB01BF052
:1055A000070F2ED01BF0010F09D0F90507D50122F6
:1055B0001A62D4F8902042F00102C4F890201BF047
:1055C000020F09D0EA0707D502221A62D4F8902008
:1055D00042F00402C4F890201BF0040F09D0E80741
:1055E00007D504221A62D4F8903043F00203C4F8BD
:1055F0009030D4F8903023B1204602F07FF8C4F800
:105600009080B4F85E309BB2002B95D1226852E8AE
:10561000003F23F4807342E8003123680029F5D16C
:1056200003F1080252E8002F02EA090203F1080020
:1056300040E800210029F3D120225345C4F88C20F2
:10564000616721670AD05A68110207D553E8002F15
:1056500022F0806243E800210029F7D1E26E012A9E
:1056600014D10022E26653E8002F22F0100243E832
:1056700000210029F7D1DA69B4F85C10D20644BFE2
:1056800010221A622046FFF725FC55E7204602F05B
:105690002DF851E79A6942F008029A616EE700BF5F
:1056A000FEFFFFEF008000409D52000810B590F80B
:1056B0008430012B1ED0012380F884302423C0F8CD
:1056C0008830026852E8003F23F00C0342E80034BF
:1056D0000168002CF5D151E8002F42F0080241E8A2
:1056E0000023002BF7D12022C0F8882080F88430D6
:1056F000184610BD0220FCE710B590F88430012B4D
:105700001ED0012380F884302423C0F8883002683A
:1057100052E8003F23F00C0342E800340168002CFB
:10572000F5D151E8002F42F0040241E80023002B9C
:10573000F7D12022C0F8882080F88430184610BDA8
:105740000220FCE7D0F88820D0F88C001043704786
:1057500038B5044603682169A2681D68C0690A4318
:1057600061690A437549024329400A431A605A682D
:10577000E16822F440520A435A60714AA169934297
:105780001CBF226A11439A6822F06E4222F43062F2
:105790000A439A60DA6A616A22F00F020A43DA6207
:1057A000684A934217D14FF0B043674AD3F8883024
:1057B00003F0030343F4403393425BD0B3F1031F80
:1057C00021D0013A934274D0B0F5004F40F0B08040
:1057D000FEF734FC31E05D4A934231D14FF0B043E3
:1057E0005B49D3F8883003F00C0343F440228A422B
:1057F00040D005D8E3B1574B9A425AD0012062E01D
:10580000B2F10C1FFAD1B0F5004F37D04FF4004081
:105810006368616A504A32F81120B0FBF2F000EB85
:105820005300B0FBF3F04FF6EF73A0F1100274E0F9
:10583000B0F5004F77D1FEF7F1FB002842D01DE014
:105840003F4A9342DAD14FF0B043D3F8883003F4A3
:105850004063B3F5006F3DD006D883B3B3F5806FD6
:10586000CCD1FDF7CFFF2CE0B3F5406FC6D14FF49C
:10587000004030E0B0F5004F3848C9D16268616A35
:10588000354B33F81130B0FBF3F0530803EB400312
:10589000B3FBF2F34FF6EF72A3F110019142ADD8D2
:1058A00023F00F02216892B2C3F342031343CB608B
:1058B00008E0B0F5004F3ED1FDF7A4FFBDE7FEF7CD
:1058C000ADFB40B900204FF00113A3660023C4E9EB
:1058D0001D3338BD214865681F4B626A05EB4501E1
:1058E00033F81220B0FBF2F3994287D8B3EB053FAF
:1058F00084D800231946FBF7A7FC090241EA10618E
:105900006B080002C0182A464FF0000341F1000165
:10591000FBF79AFC124BA0F540729A423FF66EAF2D
:105920002368D860CEE7FEF779FB0028CAD06FE77E
:10593000FEF784FBF9E7FDF765FFF6E7F369FFCFB4
:105940000080004000380140020003000044004095
:1059500008000C0004000C00F86702080024F400A2
:10596000FFFC0F00836A1A0710B506D50168846B27
:105970004A6822F4004222434A60DC0706D50168E7
:10598000C46A4A6822F4003222434A60990706D565
:105990000168046B4A6822F4803222434A605A0745
:1059A00006D50168446B4A6822F4802222434A608B
:1059B000DC0606D50168C46B8A6822F48052224353
:1059C0008A60990606D50168046C8A6822F4005240
:1059D00022438A605A060FD50168446C4A6822F453
:1059E00080122243B4F5801F4A6005D14A68846C56
:1059F00022F4C00222434A601B0606D50268C16C2D
:105A0000536823F400230B43536010BD2DE9F84382
:105A1000DDF8209005460E46174698462A68D36959
:105A200036EA03030CBF01230023BB4201D0002050
:105A300029E0B9F1FF3FF2D0FBF730FDA0EB080001
:105A400048452C6802D8B9F1000F1ED154E8003F38
:105A500023F4D07344E80032002AF7D104F108039C
:105A600053E8003F23F0010304F1080141E800324C
:105A7000002AF3D12023C5F88830C5F88C300023E4
:105A800085F884300320BDE8F88323685A07C5D51C
:105A9000802EC3D0402EC1D0E3691B05BED54FF484
:105AA0000063236254E8003F23F4D07344E80032DB
:105AB000002AF7D104F1080353E8003F23F0010363
:105AC00004F1080141E80032002AF3D12023C5F88F
:105AD0008830C5F88C30C5F89030D0E72DE9F74311
:105AE0009846D0F88830202B04460E46174643D1FE
:105AF000002943D0002A41D021230025C0F890502E
:105B0000C0F88830FBF7CAFCA368A4F85470B3F55A
:105B1000805F8146A4F8567003D123690BB93546DE
:105B20001E46B4F85620CDF8008092B24B4642B9DA
:105B300040212046FFF76AFF48B92023C4F8883087
:105B400006E0002280212046FFF760FF18B1032005
:105B500003B0BDE8F08322685EB935F8023BC3F3B9
:105B600008039362B4F85620013A92B2A4F8562082
:105B7000D7E716F8013BF4E70220E9E70120E7E761
:105B800073B504460026C0F89060FBF787FC2368D5
:105B90001B681A07054619D423681B685B070AD5DA
:105BA0006FF07E43009300222B464FF48001204685
:105BB000FFF72CFFB0B900202023C4F8883084F808
:105BC0008400C4F88C30E06620670CE06FF07E4300
:105BD0000093324603464FF400112046FFF716FFAC
:105BE0000028D9D0032002B070BD10B5044650B3D0
:105BF000D0F888301BB980F88430FFF70AF92268A2
:105C00002423C4F88830136823F001031360A36AC7
:105C100013B12046FFF7A6FE2046FFF799FD0128A5
:105C200011D023685A6822F490425A609A6822F090
:105C30002A029A601A6842F0010220461A60BDE802
:105C40001040FFF79DBF012010BD10B5044670B392
:105C5000D0F888301BB980F88430FFF7DAF8226872
:105C60002423C4F88830136823F001031360A36A67
:105C700013B12046FFF776FE2046FFF769FD0128A5
:105C800015D023685A6822F490425A609A6822F02C
:105C900022029A609A6842F008029A601A6842F0FA
:105CA000010220461A60BDE81040FFF769BF0120DD
:105CB00010BD000030B581658168A0F85C2000232C
:105CC000B1F5805FA0F85E20436731D10369002BF6
:105CD00040F2FF1318BFFF23A0F860300023C0F884
:105CE00090302223C0F88C30016801F1080353E89A
:105CF000003F43F00103083141E800340368002C01
:105D0000F2D1456E84680169B5F1005F35D1B0F814
:105D10006850954231D8B4F5805F29D1C1B1264A87
:105D2000426753E8002F42F4807243E8002121E0EB
:105D300029B90369002B14BF7F23FF23CCE7B1F1FE
:105D4000805FC9D10369002B14BF3F237F23C3E7C2
:105D50001A4A426703F1080252E8002F42F08052CB
:105D600003F1080040E800210029F3D1002030BDF4
:105D7000114A42670029D4D1ECE7B4F5805F16D10F
:105D800051B10F4A426753E8002F42F4907243E842
:105D900000210029F7D1E9E70A4A426753E8002FBA
:105DA00042F0200243E800210029F7D1DEE7044A4F
:105DB00042670029F2D0E6E7615300080955000860
:105DC000D15100089D520008D0F88C30202B30B4FF
:105DD00015D1B9B1B2B100230468C3660A4B9C4225
:105DE0000AD063681B0207D554E8003F43F0806384
:105DF00044E80035002DF7D130BCFFF75BBF02202F
:105E000030BC70470120FBE70080004070477047BE
:105E100090F88430012B0FD0012380F88430016882
:105E200051E8002F42F0020241E80023002BF6D196
:105E300080F88430184670470220704790F884300C
:105E4000012B0FD0012380F88430016851E8002F26
:105E500022F0020241E80023002BF6D180F88430C2
:105E60001846704702207047836810B504462BB16E
:105E70000322014698470023C4E9023310BD83681A
:105E800010B5044613B1032201469847204610BDC1
:105E900010B5044650F8103FDA6822F00102DA60CB
:105EA000DA6822F00202DA60DA6822F00402DA60CC
:105EB000DA6822F00802DA60DA6822F01002DA60AA
:105EC000FEF726FC2269136823F001031360012307
:105ED00084F84E3084F84F3084F8503084F85130D4
:105EE00084F8523084F8533084F8543084F85530B4
:105EF00084F8563084F8573010BD4B1E032B00D960
:105F0000FEE78900081F70470139435C13F0100059
:105F100004D0022916D80C4A32F81100DB0712D53A
:105F200003290FD8DFE801F00205080B40F001005B
:105F3000704740F01000704740F48070704740F4A4
:105F400080507047FEE7704718680208013903293E
:105F500000D9FEE7014B585C704700BF1468020887
:105F60000139032900D9FEE7014B585C704700BF97
:105F7000106802082DE9F04104460E46FFF7BDFF08
:105F800004EB061808F16408054631462046FFF781
:105F9000DDFFD8F808302BB12369C2431A61DA68F3
:105FA0000243DA60771E04EB47039B880B2B49D82A
:105FB000DFE803F051181818060618184A4A4A2A4A
:105FC000E35DDE0604D5294604F11000FEF742FE2B
:105FD000E35DD80736D5294604F11000BDE8F0414D
:105FE000FEF75ABDE35DD90604D5294604F1100039
:105FF000FEF7E8FDE35DDA0724D5294604F1100039
:10600000BDE8F041FEF7DEBC294604F11000FEF7C2
:1060100045FD31462046FFF7A3FF256901460646A8
:106020002046FFF771FF2B6A1843D8F80830286222
:1060300043B131462046FFF789FFC3432B61EB682C
:106040001843E860BDE8F081294604F11000BDE87E
:10605000F041FEF723BD23691B68DB07F2D404F18E
:106060001000BDE8F041FEF731BB70B501250446D4
:10607000861C294636F8023F23B129462046FFF701
:1060800079FF00210135052DF4D1E36E3BB1236981
:106090006FF001021A61DA6842F00102DA6049B178
:1060A00023691B68DB0705D404F11000BDE87040CC
:1060B000FEF70CBB70BD01211030FEF755BB036924
:1060C000186800F00100704710B502460C46FFF753
:1060D000F6FF80B9CB68DB070ED5CB6823F0010350
:1060E000CB601046FFF7E7FF6FF001032361E36821
:1060F00043F00103E36010BDBDE810401046FFF718
:10610000DABF00000B4B98420BD0B0F1804F0AD0A1
:1061100003F5C053984208D003F58063984206D037
:10612000FEE70020704701207047022070470320DF
:10613000704700BF002C0140024670B5044652F87B
:10614000100FFFF7DFFF0546104600F00DFF094A6C
:10615000002342F8253004F16406E36004F1B4053D
:10616000B54204D0103D2846FFF789FEF8E72046E7
:1061700070BD00BFE803002070B504460846FFF775
:10618000C1FF256905B1FEE7204B216104F10C0236
:1061900043F8202004F110060E23C4E917353046D9
:1061A000C4E90C55C4E90E55C4E9105584F82C50C7
:1061B000A56484F84C5084F84D50E46000F0A8FECB
:1061C00004F16400FFF750FE04F17400FFF74CFE89
:1061D00004F18400FFF748FE04F19400FFF744FE49
:1061E00004F1A400FFF740FEC4E900554FF6FF7329
:1061F000C4E906538023C4E90855A5606561A3621C
:106200003046BDE87040FEF79FBB00BFE8030020AA
:1062100010B588B018220446002102A81EF035F8F7
:10622000002301A902A80193FDF718FF206900F0DF
:1062300041FF012802D002280FD0FEE7059CFDF7A0
:10624000EDFEB4F5C06F05D00BD824F48074B4F51E
:10625000806F00D1400008B010BD069CFDF7EEFE37
:10626000EFE7B4F5E06FF4E7012A38B505460C46D0
:106270000BD0022A16D004B1013C29692846CC6211
:10628000EC61BDE83840FFF71FBFFFF7C1FF084BC7
:10629000B0FBF3F044432A69230C93620133B4FB4F
:1062A000F3F4E8E7FFF7B4FFB0FBF4F4F3E700BF63
:1062B00040420F0010B500F110042046FEF73CFAF2
:1062C0002046BDE81040FEF7CEB90000034B186829
:1062D00010B10430FEF75CBA704700BFE80300203D
:1062E000FFF7F4BF034B586810B10430FEF750BA03
:1062F000704700BFE8030020034B986810B10430DA
:10630000FEF746BA704700BFE8030020034BD86889
:1063100010B10430FEF73CBA704700BFE80300201C
:106320000022C0E90022C0E902227047F8B5044605
:106330000E4600F1640500F1B40728461035FFF75A
:10634000EFFFBD42F9D10023204623613146FFF71C
:1063500013FF2046F8BD38B50023C0E90033C0E97B
:1063600002338B6804460D462BB102229847EB6836
:10637000E360AB68A360204638BD30B587B002AD9E
:1063800004462846FFF7E7FF95E803006B4683E8DD
:10639000030094E8030085E8030093E80300049BEE
:1063A000A268A360059B049284E80300E268E360AE
:1063B00028460592FFF763FD07B030BD38B50446A7
:1063C0000D46E36E64301BB1BDE83840FFF7D5BF22
:1063D000FFF7D3FFAB683BB123696FF001021A618D
:1063E000DA6842F00102DA6038BD826810B50AB995
:1063F0001AF01AFCBDE81040C368184708B500B988
:10640000FEE700F083FD0068C36E13B16430FFF750
:10641000ECFF08BDFFF7F2BF10B500B9FEE7037F40
:10642000013B072B10D8DFE803F004140F100F0F07
:106430000F12012400F06AFD240100686434204436
:1064400083680BB1FFF7D1FF10BD0324F2E70424EA
:10645000F0E70224EEE7FFF7DFBFFFF7DDBF1CF038
:10646000C7BC1CF0C5BC1CF0CBBC4FF0B04382B025
:10647000DA6C0243DA64DB6C03400193019B02B0E7
:106480007047000008B5032818D8DFE800F00208BC
:106490000D120120FFF7E9FF4FF0904008BD0220E8
:1064A000FFF7E3FF0648F9E70420FFF7DEFF0548A2
:1064B000F4E78020FFF7D9FF0348EFE70020EDE77E
:1064C0000004004800080048001C004808B50649C0
:1064D00000F0E4FCC0F3C430112800D9FEE7034B00
:1064E00053F8200008BD00BF006702082C680208AE
:1064F000A0F580500138022800D9FEE7014B53F87F
:10650000200070472068020808B5054900F0C6FC65
:10651000C0F3C430012800D0FEE7002008BD00BF52
:10652000E86602080268094B9A420DD14FF0B04369
:106530009A6B42F000529A639A6B22F000529A636F
:106540009A6D22F000529A65704700BF00740040B7
:1065500010B50A4986B0044600F07EFC019050B1A7
:106560002046FFF7D1FF014628B901A8FBF7D3FC6D
:1065700001A8FBF7C2FC06B010BD00BFE866020828
:106580004FF0B04382B01A6E42F400721A661A6E6F
:1065900002F400720192019AD3F8882042F040522E
:1065A000C3F88820044B1868C30403D4034902B01D
:1065B00000F03ABC02B070471800002000670208E3
:1065C0004FF0B0431A6C42F400721A641A6C22F451
:1065D00000721A641A6C42F400721A641A6C22F483
:1065E00000721A641A6E22F400721A667047000074
:1065F000F0B59FB0054664220E4605A800211DF0A7
:1066000044FE0023EA04CDE902330493ADF80230DE
:10661000019340F1AC8041F203039D4200F2A78058
:106620005D4B05932846FFF763FF07270446082EB6
:1066300000F0AE800A2E00F0AD80062E0CBF1823AD
:1066400000234FF00042CDE906230023CDE90832B4
:106650000422CDE90E330A92ADF82C3001228DF8D8
:106660002E308DF834308DF840308DF8503018933E
:106670001B9319938DF86830484B0C9205A84FF482
:106680008052CDE9112713971D60FAF711FF0028FA
:1066900079D1012C029435D0414B9C4232D0414BF0
:1066A0009C422FD0404B9C422CD0404B9C4229D046
:1066B0003F4B9C4226D03F4B9C4223D03E4B9C42BA
:1066C00020D03E4B9C421DD03D4B9C421AD03D4BAE
:1066D0009C4217D003F104239C4213D03A4A24F081
:1066E000004393420ED0394A93420BD0384A93422A
:1066F00008D0384A944205D0374A944202D0374AEB
:10670000934240D1012302A905A8CDE90337FBF745
:106710002DF8002837D105A8FBF762FA002832D1FE
:1067200005A8FBF785F970BB0A2105A8FAF7C0FF99
:1067300048BB05A8FBF7F2F8830505D505A8FBF7CC
:1067400011F880B2ADF8020005A8FBF72BFAD0B91A
:1067500005A8FBF7D1F9B0B9214AD2F8083723F0E0
:10676000E073C2F80837BDF8020080B20CE01D49A2
:10677000284600F071FB01A905902846FFF7A6FE08
:10678000059B044613B900201FB0F0BD03274EE758
:10679000102356E7082354E7002401401800002086
:1067A00002000004040000080800000C10000010A3
:1067B00020000014400000188000001C0001002090
:1067C00000020024000400280010003000200034E3
:1067D000004000380080003C0000014000000244FE
:1067E0000020014000670208F8B51449144E07461E
:1067F00000F032FBFFF786FC56F82030044673B9F0
:10680000B420FFF72CFE0D490546384600F024FB66
:1068100001462846FFF78AFD56F824301D6056F8D9
:1068200024301C6844B12046FFF786FC2046B42182
:10683000BDE8F840FFF717BEF8BD00BF7465020859
:10684000E803002037B5FAF729FE4FF0E0250446AB
:10685000AB690093FAF722FEAB6901936969844240
:1068600001F101014FF47A7308D0019A8A1A5A4350
:10687000B2FBF1F203FB002003B030BD009A8A1A8C
:106880005A43B2FBF1F203FB0420F5E7FAF706BE28
:10689000704708B5FAF7F6FDFBF7C7FAFFF7F8FF00
:1068A00008BD10B594B048220021044602A81DF08E
:1068B000ECFCFCF7F9FE4FF0B0439A6D42F48062B5
:1068C0009A659A6D02F480620192019A032C11D8A4
:1068D000DFE804F00219283DD3F8942042F00102C9
:1068E000C3F89420D3F894309C0703D40823029370
:1068F00001230893029B002B3AD002A8FDF700F871
:10690000002835D0FEE71A6842F480721A601B68CE
:106910005905EFD4022302934FF480724023CDE94E
:106920000623E7E7D3F8902042F00102C3F8902055
:10693000D3F890209407DDD4D3F8902022F01802E9
:10694000C3F890200423029381230593D2E71A68A9
:1069500042F400121A601A6842F480321A601B680E
:1069600099035EBF01224FF40413CDE90223C1E76E
:1069700014B010BD70474FF0B04382B01A6D42F4AE
:1069800000221A651A6D02F400220192019A9A6C93
:1069900042F480529A649B6C03F480530093009BF2
:1069A00002B070470C4BD3F8FC20D2015EBFD3F885
:1069B000FC2042F08072C3F8FC20084B00225A6091
:1069C0001A6842F001021A6000BF00BF00BF586899
:1069D000B0FA80F04009704700ED00E0001000E0E0
:1069E00008B5FFF7C8FFFFF7DDFFFAF735FDFFF742
:1069F000C1FFFAF7C5FCBDE808400148FBF71ABA29
:106A00001C000020012A02D1016000207047022AE8
:106A100005D0032AF9D0002AF7D10260F5E70B6808
:106A20000360F2E7036818470023C0E90033C0E9B8
:106A30000233704770B50024012904F101032CD101
:106A4000184DE4B2142161436E18F3683BB1043170
:106A500029440322084698470023C6E90333142338
:106A600063430022E8560F4B93F90010814201D195
:106A7000D968A9B90132102A03F11403F4D10A4AE2
:106A80000A49D2F8803051F8241023EA0103BDE806
:106A90007040C2F88030FBF781B949081C46CBE74B
:106AA00070BD00BFF8030020000800587468020899
:106AB0000023012803F101020AD11422DBB253435F
:106AC000054A181D1044816829B11A4413691847F2
:106AD00040081346EDE77047F80300200120FBF75C
:106AE00041BC0220FBF73EBC0420FBF73BBC082066
:106AF000FBF738BC1020FBF735BC38B50524202542
:106B0000A8B2FBF72FFC013C4FEA4505F8D138BD90
:106B100038B506244FF48065A8B2FBF723FC013C8E
:106B20004FEA4505F8D138BD2DE9F04116468CB045
:106B30000A460024012A04F1010543D1E4B26200AF
:106B4000CDE90713C168DFF88480032393400B402D
:106B5000D34003F0030303AD099307A902230A936B
:106B6000FBF74CFB1423314628465C43FFF7F3FB4D
:106B700095E8030008EB040301AA043382E803004C
:106B800093E8030085E8030092E80300271D83E8EB
:106B900003004744059BBA68BB60069B05922846E4
:106BA000FA68FB600692FFF76AF918F90400002200
:106BB0000621FBF7B3F818F90400FBF7E1F80CB075
:106BC000BDE8F08152082C46B4E700BFF80300206E
:106BD000344A104608B5062300F8043BFFF724FFAB
:106BE000072302F118001375FFF71EFF082302F1B7
:106BF0002C0082F82830FFF717FF092302F140002C
:106C000082F83C30FFF710FF0A2302F1540082F8AB
:106C100050301621FFF708FF02F1680082F8641077
:106C2000FFF702FF02F17C0082F87810FFF7FCFE0C
:106C300002F1900082F88C10FFF7F6FE02F1A4003A
:106C400082F8A010FFF7F0FE02F1B80082F8B4104D
:106C50002921FFF7E9FE02F1CC0082F8C810FFF706
:106C6000E3FE02F1E00082F8DC10FFF7DDFE02F146
:106C7000F40082F8F010FFF7D7FE02F5847082F876
:106C80000411FFF7D1FE02F58E7082F81811FFF79C
:106C9000CBFEBDE8084002F5987082F82C11FFF792
:106CA000C3BE00BFF803002038B5054CA4F5A0759D
:106CB000143C201DFFF7E3F8AC42F9D138BD00BF0A
:106CC0003805002030B591FAA1F391FAA1F1B3FA99
:106CD00083F3C4685B000325B1FA81F105FA03F37D
:106CE000490024EA03038A401A43C26030BD431CB2
:106CF00004D00C3151F80C3C5A1C01D100207047D3
:106D0000834201F10C01F5D101207047F8B5471C11
:106D100006460D4600D1FEE700F00F02414BC0F3DE
:106D2000031053F82240FFF7ADFB94FAA4F3B3FA33
:106D300083F3876803225B0002FA03F394FAA4F258
:106D4000B2FA82F227EA03075200032393403B433F
:106D500005F007018360032903D8DFE801F05F0332
:106D60002C61FEE7012394FAA4F2B2FA82F20668DB
:106D70005200032707FA02F226EA020694FAA4F266
:106D8000B2FA82F252009340013933430129036081
:106D900005D843682A074CBF2343A3434360C5F388
:106DA0000112012A02D0022A18BF00222146BDE8A2
:106DB000F840FFF787BFC5F306227F2A01D10223DF
:106DC000D1E7360716D5230A93FAA3F6B6FA86F664
:106DD000476A93FAA3F3B6004FF00F0CB3FA83F3AC
:106DE0000CFA06F69B0027EA060602FA03F3334381
:106DF0004362E4E794FAA4F3B3FA83F3066A9B00D0
:106E00000F2707FA03F326EA030694FAA4F3B3FA6A
:106E100083F39B009A4032430262D0E70023A2E74B
:106E20000323A0E7B4680208431C06D170478342DD
:106E300002D18968FFF76ABF0C310B685A1CF6D182
:106E4000FEE70B685A1C01D100207047834201D134
:106E5000486870470C31F4E7431C01D0FFF7F1BFDD
:106E6000002070474B6813B94FF0FF3070478342E2
:106E700001D1086870470C31F4E708B1FFF7F2BFA1
:106E80004FF0FF30704703460868421C00D170473E
:106E9000984201D1886870470C31F5E7431C01D056
:106EA000FFF7F1BF704703468B42084604D01BB181
:106EB00000290CBF18460020704700004FF0B04377
:106EC0001A6842F061021A604FF4E0229A6061226F
:106ED0001A60064ADA6000229A6140F23F321A6272
:106EE000034B4FF000629A60704700BF000104221C
:106EF00000ED00E04FF0B04382B01A6E02431A6614
:106F00001B6E03400193019B02B070470438704729
:106F10000368124A934282B004D14FF4006002B079
:106F2000FFF7E8BFB3F1804F0CD14FF0B0439A6D3B
:106F300042F001029A659B6D03F001030193019BEE
:106F400002B07047064A934202D14FF40030E6E7A0
:106F5000044A9342F4D14FF48020E0E7002C014032
:106F600000440140004801400368134A934206D19F
:106F70004FF0B042136E23F4006313667047B3F111
:106F8000804F06D14FF0B042936D23F0010393651B
:106F900070470A4A934205D14FF0B042136E23F472
:106FA0000033EAE7064A9342E8D14FF0B042136E4D
:106FB00023F48023E1E700BF002C0140004401409E
:106FC00000480140431C10D00C4B984210D007D809
:106FD000B0F1804F0ED0A3F5C05398420CD0FEE71D
:106FE000074B9842FBD11D2070476FF00D00704792
:106FF0001C2070471B207047182070470044014038
:1070000000480140431C10D00C4B984210D007D8C8
:10701000B0F1804F0ED0A3F5C05398420CD0FEE7DC
:10702000074B9842FBD11D2070476FF00D00704751
:107030001C2070471B2070471A20704700440140F5
:107040000048014038B50446FFF762FF2068FFF7AB
:10705000B9FFD4E91312FAF761FE2068FFF7B2FF17
:10706000FAF78EFE22681046FFF7CCFF0546104661
:10707000FFF7A8FF85420BD02846D4E91312FAF790
:107080004DFE2068FFF7BEFFBDE83840FAF778BE36
:1070900038BD10B5FFF768FF04460068FFF792FFA0
:1070A000FAF77CFE2068FFF7ADFFBDE81040FAF765
:1070B00075BE0000431C10D00A4B98420BD003D879
:1070C000B0F1804F0BD0FEE7074B984203D003F599
:1070D00080639842F7D1022070470020704701205A
:1070E000704700BF002C0140004401404FF0B04207
:1070F000D2F8883023F440630343C2F888307047E5
:107100002DE9F04F89B0CDE901230446129BD0F858
:10711000A00003938B46B449FFF79EFEB349824615
:10712000D4F8A400FFF798FEB1490646D4F8A800A9
:10713000FFF792FEAF490746D4F8AC00FFF78CFE8C
:10714000AA498046D4F8A000FFF786FEA6498146EA
:10715000D4F8A400FFF780FE0546BAF1000F03D172
:10716000B9F1000F00F03A81D4F8A430013303D014
:1071700016B9002D00F03281D4F8A830013302D0C6
:10718000002F00F02B81D4F8AC30013303D0B8F1DC
:10719000000F00F0238131465046FFF784FE206047
:1071A00020B929464846FFF77EFE20603946206810
:1071B000FFF779FE41462060FFF775FE206000284A
:1071C00000F00C818C4B984240F0A1804FF0B0430E
:1071D0001A6C42F480421A641A6C22F480421A64D7
:1071E0001A6E42F480421A661B6E03F480430593C4
:1071F000059B2423A4F8B030BAF1000F00F0BA8048
:107200007949D4F8A000FFF70FFE26B17749D4F8EA
:10721000A400FFF709FE4FF00009002F00F0BC802A
:107220007349D4F8A800FFF7FFFD4FF4807AB8F156
:10723000000F06D06F49D4F8AC004AF4007AFFF78B
:10724000F3FD94F8B1206D4B94F9B000C4F83C9074
:10725000271D43F822702368C4E9013B019BE360CA
:10726000039B2361029B63610C230022C4E9063A5D
:107270000823E362226262620121FAF74FFDD4F82B
:1072800000805F4B984538D1BBF5165F384600F259
:107290008580FEF7BDFD3846002E00F09380FEF796
:1072A000A4FC002800F09A800220FFF7FAFA4FF0C1
:1072B000B043D3F890309B0700F1A6804FF0B04365
:1072C00022681B68590500F1D58022684C4B9A4210
:1072D00002D10020FFF70AFF16B9002D00F0BB8095
:1072E0003846FEF782FC002878D02268444B9A4248
:1072F00003D14FF48060FFF7F9FE16B9002D00F0BE
:10730000B380384609B0BDE8F04FFEF76EBC3D4B88
:10731000984215D14FF0B0439A6B42F400329A6311
:107320009A6B22F400329A639A6D42F400329A65A5
:107330009B6D03F400330693069B40F2251359E737
:107340002F4B98427FF458AF4FF0B043DA6B42F0C6
:107350000102DA63DA6B22F00102DA63DA6D42F0DD
:107360000102DA65DB6D03F001030793079B40F22E
:1073700026233FE7B9F1000F3FF44DAF1B49D4F886
:10738000A000FFF751FD25B11749D4F8A400FFF77D
:107390004BFD4FF4004940E7BA4648E7FEF74EFD83
:1073A0003846AEB1FEF721FCC0B14FF0B0431A68C9
:1073B0002368500589D5434562D14FF40060FFF73B
:1073C00095FE5AE0002D7FF46AAFFEF73EFC68E7B9
:1073D0003DB9FEF73AFC00287FF470AF09B0BDE874
:1073E000F08FFEF702FCF6E72C650208D86402086D
:1073F000C0640208A8640208003801403805002073
:1074000000800040004400402268234B9A4203D190
:107410004FF44060FFF76AFE3846002EE1D1002DA0
:10742000DFD1FEF712FC0028D8D04FF0B04322681D
:107430001B685B057FF549AF174B9A42BDD03846B4
:10744000FEF703FC0028C9D02268134B9A4202D1F0
:107450000020FFF74BFE3846FEF7F7FB0028BDD0B3
:1074600022680D4B9A4212D0384609B0BDE8F04F61
:10747000FEF7EBBB084B9A429FD00EB9002DDED031
:107480003846FEF7B2FB00287FF41FAFA6E74FF4A3
:107490008060FFF72BFEE7E70080004010B4019CFE
:1074A00018B1019410BCFFF72BBE10BC7047000050
:1074B000094B13B55C6909492046FFF7CDFC48B17B
:1074C00007480023C0F8A0401A4600934FF4165115
:1074D000FFF716FE02B010BD8C6702082C6502088B
:1074E0004400002008B5074B90F8B12053F8220063
:1074F000FEF728F900F02200A0F12203584258417B
:1075000008BD00BF3805002008B5074B90F8B12032
:1075100053F82200FEF716F900F02100A0F1210334
:107520005842584108BD00BF380500202DE9F047FA
:107530002B4C06460D46F9F7B1FF94F8B130022BFB
:10754000074613D894F8B120264B53F82240A4F1F3
:1075500004084046FFF7D8FFD0BB4FF47A73AAB2B5
:1075600031462046FEF7BAFA40B908E01E4B1F49E3
:10757000D3F814804046FFF76FFC18BB002528465F
:10758000BDE8F0875AF8233043B994F8B13001339D
:10759000DBB2022B84F8B130F4D90CE04946404606
:1075A000FFF75AFC94F8B1205AF822301B68834246
:1075B000EBD1022AC6D9FFF77BFF94F8B130022B3A
:1075C000C0D9DBE7DFF81CA0DFF820900023E0E75C
:1075D000F9F764FFC01BB0F57A7FBAD3CEE700BFDE
:1075E00044000020380500208C6702082C65020842
:1075F00070B50E46054610B94FF0FF3070BDFFF76D
:1076000071FF04460028F7D12946012211F8B23F44
:10761000337095F8B100034B53F82000FEF7D4FB0C
:107620002046EBE73805002038B50D460446C0B1CA
:10763000FFF758FFA8B994F9B000C4F89850FAF7CA
:10764000ADFB94F8B100074B04F1B20153F82000F0
:107650000122FEF7B9FB94F9B000BDE83840FAF713
:107660008FBB38BD3805002038B515460446C8B173
:10767000C0F89C1090F9B000FAF790FBD4F8B8303D
:10768000B4F8C21094F8B10013FA81F1064BAAB213
:1076900053F82000FDF7BEFB94F9B000BDE8384078
:1076A000FAF76EBB38BD00BF3805002050B1D0F8E6
:1076B000A430013306D190F8B120034B53F82200D7
:1076C000FDF7F4BF704700BF3805002050B1D0F877
:1076D000A430013306D190F8B120034B53F82200B7
:1076E000FEF70AB8704700BF38050020D0F8943084
:1076F00004381847D0F898300438184710B50446B5
:1077000050F80439DA69D1070CD501221A62FFF763
:10771000E9FEB0B904F1AE0120460122BDE81040F7
:10772000FEF752BBDA69920701D50222EEE7DA6969
:10773000510701D50422E9E7DA691207E7D50822E3
:10774000E4E710BD08B52420FAF760FB024B186887
:10775000BDE80840FDF7C0BB3805002008B525206E
:10776000FAF754FB034B586818B1BDE80840FDF721
:10777000B3BB08BD3805002008B52620FAF746FB44
:10778000024B9868BDE80840FDF7A6BB380500200D
:10779000012200F1AE01FEF717BB00000A490346C3
:1077A000086810B50344EFF30882934205D9074BEC
:1077B0000C221A604FF0FF3010BD054A054C121B19
:1077C0009342F4D20B60F7E70C010020F43F002055
:1077D00000000120000400004FF0FF3070474FF41C
:1077E00000534B6000207047012070470020704715
:1077F00000207047FEE70000024B16221A604FF08F
:10780000FF307047F43F0020012070470048704768
:1078100080EE360000207047704770477047704711
:10782000704770477047D0F8FC00704790F87601B9
:10783000704790F82502003818BF0120704790F873
:1078400077314FF47A605843704790F86B01704776
:10785000004870479469020800487047946902081C
:1078600000487047A669020800487047A6690208E8
:1078700000487047B269020800487047B2690208C0
:1078800080F8E810704780F8201070476830704723
:1078900060387047704700F58053F0B50246D3F862
:1078A00094560023184602F52576A027AB4200DB4C
:1078B000F0BD07FB03F491F800C0345DA44502BF9E
:1078C00000F6F224013042F824300133EEE70020C4
:1078D00070470000084A0023C2E90433D360426EB7
:1078E000A0F85830C0E90E33C0E90C33C2F80C35AB
:1078F000C2F80835704700BFE0370020A0F1C8008B
:10790000FFF7E8BF02F6F22250F82230002B12DB1C
:1079100000F58052D2F8942693420CDAA02202FBA2
:10792000030000F2F62300F2163053F8042B41F85E
:10793000042B8342F9D170472DE9F041054605F546
:10794000005488464FF4FA6117461E4603F064FB64
:107950009DF81830079984F8C53B4EF660235943CB
:10796000C4F8B40BC4F8BC8BC4F8C07B84F8C46BF7
:1079700001F5FA61284603F04FFBC4F8B80BBDE8E7
:10798000F081A0F1C800FFF7D7BF000010B590F854
:107990004611044621B1044B594303F03DFB014617
:1079A000C4F8E01010BD00BFC0D40100A0F1C800B1
:1079B000FFF7ECBF10B590F84711044621B1044B16
:1079C000594303F029FB0146C4F8E41010BD00BF81
:1079D00080EE3600A0F1C800FFF7ECBF7FB50A4A81
:1079E0000346084651690491D96B0391996B029142
:1079F000596B01911B6B0093D2E9032303491CF0DF
:107A000059FB07B05DF804FBE0370020BB690208B2
:107A1000A0F1C800FFF7E2BF10B5C06D104C0368BD
:107A200086B01B689847014604A80FF025FF9DF813
:107A300010309DF813200B4903F5FA6303939DF86A
:107A4000113002939DF8123001939DF81530009388
:107A500020469DF814301CF02DFB204606B010BDCA
:107A6000440500201C6A020870B5D0F848510C4645
:107A7000284600211646F9F71DFBD8B921460E48C5
:107A8000F9F766F80146284619F0CAFCF8F7BCFC7D
:107A90000A4B0022F8F758FB044630460D46F8F72B
:107AA00091FC02460B4620462946F8F705FDF8F7FB
:107AB000B3FF70BD0020FCE79A99593F0000F03FEA
:107AC00038B50B7813F0030304460D460FD100F5CB
:107AD000CA500122183007F003FE04F5005329466E
:107AE000C3F8D8022046BDE8384004F033B9012B72
:107AF00009D100F5805393F8E83DDB0703D400F586
:107B0000EF500430E9E70020E7E702F6F22238B54B
:107B100050F82240002C054618DB00F58052D2F8C0
:107B20009426944212DAA022544304F2B6209DF81F
:107B300014200499284404F03AFC2C4484F8B5023B
:107B4000E86D03681B689847C4F81C03002038BD23
:107B500000F5805310B5B3F85C29A3F80C2E044649
:107B6000002100F50A50A3F8121E1C223C301CF024
:107B70008CFB04F5005304F50A5414340122C3F8B5
:107B8000B84283F80C2310BDA0F1C800FFF7E0BF96
:107B9000C268104910B50446553207F027FBE26869
:107BA0000D492046803207F021FBE2680B49204650
:107BB000813207F01BFBE26809492046823207F058
:107BC00015FBE2680749204602F59A72BDE81040AD
:107BD00007F00CBB386A0208406A0208466A0208CD
:107BE000506A02085A6A0208C26802497A3207F0EB
:107BF000FDBA00BF5F6A020810B500F1100204462A
:107C00002B49202307F03AFA04F140022046294983
:107C1000102307F033FA04F16002204626491023AE
:107C200007F02CFA782304F1B8022046234907F024
:107C300025FA04F156022046214907F0D7FA04F14B
:107C4000570220461F4907F0D1FA04F130022046BE
:107C50001D4907F027FB04F1380220461B4907F0B5
:107C600021FB04F59E722046194907F09DFB04F59F
:107C7000A6722046174907F097FB04F5AE7220461E
:107C8000154907F091FB04F5BE722046134907F031
:107C90008BFB04F5C6722046114907F085FB04F5FD
:107CA000B67220460F49BDE8104007F07DBB00BF0B
:107CB0003F7B0208676A02086C6A0208726A02085F
:107CC0007A6A0208786A0208826A0208866A0208EA
:107CD0009C7F02088A6A0208916A0208956A020873
:107CE0009C6A0208A16A020810B5C26806490446E7
:107CF000B43207F01BFBE26804492046A532BDE818
:107D0000104007F073BA00BFA76A0208B06A020801
:107D1000C268364910B50446503207F007FBE268E6
:107D2000334920467C3207F001FBE26831492046A6
:107D3000783207F05BFAE2682F492046793207F083
:107D400055FAE2682D49204602F2351207F04EFA44
:107D5000E2682B492046863207F048FAE268294952
:107D6000204602F5987207F041FAE268264920465B
:107D700002F2311207F03AFAE2682449204602F58D
:107D8000997207F033FAE26821492046543207F02D
:107D90005BFAE2681F4920460C3207F0C7FAE26836
:107DA0001D492046583207F0C1FAE2681B492046B7
:107DB0005C3207F0BBFAE26819492046703207F0DE
:107DC000B5FAE26817492046873207F00FFAE268F1
:107DD0001549204602F2331207F008FAE268134907
:107DE00020467B32BDE8104007F000BABB6A0208AB
:107DF000C06A0208DC7A0208C36A0208C66A02087E
:107E0000CA6A02081C790208D26A0208DD6A0208FE
:107E1000E86A0208EB6A0208EE6A0208F66A0208DB
:107E2000006B02080A6B0208126B02081C6B020846
:107E3000C268134910B50446883207F0D7F9E268E2
:107E4000104920468A3207F0A3F9E2680E4920461D
:107E50008C3207F0CBF9E2680C492046903207F0EB
:107E600069F9E2680A492046943207F0BFF9E268EE
:107E7000084920461023BDE81040953207F0FEB8AF
:107E8000B86A0208F06A0208266B02082A6B020828
:107E90002F6B0208326B0208C2680A4910B504460B
:107EA000A63207F0A3F9E26807492046A83207F096
:107EB00041F9E26805492046AC32BDE8104007F0C0
:107EC00095B900BFB86A02080E6B0208396B020848
:107ED0002DE9F04307468DB08846914642F21435AD
:107EE0007C1941464A4620461CF0A5F90146A0B936
:107EF0002C2201A81CF0C9F901A803F046FB01AE31
:107F000023460BAA344603CC944218605960264697
:107F100003F10803F6D122781A702C3542F6AC33FF
:107F20009D42DDD10DB0BDE8F083A0F1C800FFF7A0
:107F3000CFBF0000014808F040BA00BFE037002082
:107F4000A0F1C800FFF7F6BF01480FF0E2BD00BF87
:107F5000143A0020A0F1C800FFF7F6BFD0F8CC100B
:107F600000F5CA500022183007F0C6BDA0F1C800C5
:107F7000FFF7F4BF07B5D0F8CC3000930A46044BA6
:107F800004490193684607F07BFA03B05DF804FBEF
:107F9000CB850208416B0208A0F1C800FFF7EABFD9
:107FA0000249D0F8CC000FF0EEBD00BF476B0208CD
:107FB000A0F1C800F4E700BFD0F8CC1000F5B45031
:107FC000183005F0A9B8A0F1C800F5E710B40446D0
:107FD00000F50B501C3039B1024604F5CA5001239C
:107FE00010BC183007F056BB10BC10221CF04DB965
:107FF000A0F1C800FFF7EABF036810B55C6A50F84B
:10800000042C516A8C4201D8036010BD40F8042949
:10801000F5E7F0B54C1E04EBD474641091424FEABE
:1080200081050CDD50F824105E6A4F6AB74206D90C
:108030004151611E01EBD17521466C10EEE74351B1
:10804000F0BDF0B5541E04EBD4740E4665106FF00D
:10805000404CA94215DBD4070ED4023A02EBD2728F
:10806000B1EB620F08D14C1C620000EBC40454F861
:10807000044C40F82140511E3246BDE8F040FFF765
:10808000C8BF4C1C640004EB0C0E50F82E7050F866
:1080900024E07F6ADEF824E0BE4588BF04F1FF34A7
:1080A00050F8247040F821702146D2E7F0B5541EF4
:1080B00004EBD4740E4665106FF0404CA94215DBFA
:1080C000D4070ED4023A02EBD272B1EB620F08D1A0
:1080D0004C1C620000EBC40454F8044C40F82140EE
:1080E000511E3246BDE8F040FFF793BF4C1C6400C0
:1080F00004EB0C0E50F82E7050F824E07F6ADEF886
:1081000024E0BE4588BF04F1FF3450F8247040F8E5
:1081100021702146D2E7036810B55C6A50F8042C40
:10812000516A8C4201D8036010BD40F80429F5E77C
:10813000F0B5541E04EBD47466106FF0404C0C463E
:10814000B44225DBD5070ED4023A02EBD272B4EB6F
:10815000620F08D1621C550000EBC20252F8042CD9
:1081600040F824206C1E621E02EBD2725210A14213
:108170004FEA840521DA50F822405E6A676AB74206
:108180001BD24451541E04EBD47514466A10EEE71A
:10819000651C6D0005EB0C0E50F82E7050F825E0B4
:1081A0007F6ADEF824E0BE4538BF05F1FF3550F8A0
:1081B000257040F824702C46C2E74351F0BD036897
:1081C00010B55C6A50F8042C516A8C4201D30360EC
:1081D00010BD40F80429F5E7F0B5541E04EBD47443
:1081E00066106FF0404C0C46B44227DBD5070ED426
:1081F000023A02EBD272B4EB620F08D1621C550056
:1082000000EBC20252F8042C40F824206C1E621EBF
:1082100002EBD2725210A1424FEA840524DA50F8E0
:10822000224093F9286094F92870B7421CDD44512C
:10823000541E04EBD47514466A10ECE7651C6D00FF
:1082400005EB0C0E50F82E7050F825E097F92870C9
:108250009EF928E0BE45C8BF05F1FF3550F82570EE
:1082600040F824702C46BFE74351F0BD10B50368B9
:1082700050F8042C93F9284092F928108C4201DC24
:10828000036010BD40F80429F2E7F0B5541E04EB7A
:10829000D47466106FF0404C0C46B44227DBD5070F
:1082A0000ED4023A02EBD272B4EB620F08D1621C18
:1082B000550000EBC20252F8042C40F824206C1E3A
:1082C000621E02EBD2725210A1424FEA840524DAF8
:1082D00050F8224093F9286094F92870B7421CDACC
:1082E0004451541E04EBD47514466A10ECE7651C27
:1082F0006D0005EB0C0E50F82E7050F825E097F944
:1083000028709EF928E0BE45B8BF05F1FF3550F84A
:10831000257040F824702C46BFE74351F0BD10B5DE
:10832000036850F8042C93F9284092F928108C42E5
:1083300001DB036010BD40F80429F2E788421346D0
:1083400004D00A1A0146981A1BF085BF704788426C
:10835000F8B504460D4602D00430854200D1F8BD80
:108360000646236856F8047B93F9283097F92820AD
:108370009A4207DA014632462046FFF7DFFF2760C0
:108380003046EAE7FFF7CBFFFAE78842F8B5044644
:108390000D4602D00430854200D1F8BD0646236860
:1083A00056F8047B93F9283097F928209A4207DD84
:1083B000014632462046FFF7C1FF27603046EAE714
:1083C000FFF754FFFAE78842F8B504460D4602D09D
:1083D0000430854200D1F8BD0646236856F8047B78
:1083E0005B6A7A6A9A4207D2014632462046FFF714
:1083F000A5FF27603046ECE7FFF7E1FEFAE7884289
:10840000F8B504460D4602D00430854200D1F8BDCF
:108410000646236856F8047B5B6A7A6A9A4207D953
:10842000014632462046FFF789FF27603046ECE7D9
:10843000FFF771FEFAE78842F8B504460D4602D010
:108440000430854200D1F8BD0646236856F8047B07
:108450005B6A7A6A9A4207D9014632462046FFF79C
:108460006DFF27603046ECE7FFF7C6FDFAE78B8823
:108470009A0903F03F0310B502FB033304464A8810
:10848000006D52FA83F1036802319B689847F8F750
:1084900011FCD4F86011F8F765FCF8F765FE00EB05
:1084A0008000421C0021206EBDE8104003F0DABFBE
:1084B00000F00300023801288CBF00200120704723
:1084C00080F00200C0F340007047002070478B88A6
:1084D0009A0903F03F0310B502FB033304464A88B0
:1084E000006D52FA83F1036802319B689847F8F7F0
:1084F000E1FBD4F84C11F8F735FCF8F735FE00EB4A
:108500008000421C0021206EBDE8104003F0AABF8D
:108510002DE9F84F04460D461746994600F1040828
:10852000291B40291CDD4FEAA10ADFB9AAF1020686
:10853000761054F82630524631462046FFF781FD2A
:108540005EB1013EF5E755F8043D22682A602A1B1A
:10855000921000212046FFF774FD2B1B042BF2DC48
:10856000BDE8F88FC910D4F804A054F82100DAF857
:1085700024B0D0F824E055F804CC2368DCF824209B
:10858000F34546462AD9964521D9206044F8213042
:108590002B462268D2F824E031460868426A7245C8
:1085A0000E4601F10401F8D8191F0B4651F80429B1
:1085B000D2F824C0E645F8D89E4217D3013F294699
:1085C0004B463A463046FFF7A3FF3546A8E79345AA
:1085D00006D9C4F800C045F8043CD9E7934502D950
:1085E000C4E900A3D4E79645CFD9F2E746F8042BB7
:1085F0001860CEE72DE9F84F04460D461746994618
:1086000000F10408291B402919DD8E10CFB9B11ED5
:10861000491054F8213032462046FFF789FD59B100
:108620000139F6E755F8043D22682A602A1B9210AA
:1086300000212046FFF77CFD2B1B042BF2DCBDE85C
:10864000F88FC910D4F804A054F82100DAF824B047
:10865000D0F824E055F804CC2368DCF82420F34556
:1086600046462AD2964521D2206044F821302B4636
:108670002268D2F824E031460868426A72450E4604
:1086800001F10401F8D3191F0B4651F80429D2F85F
:1086900024C0E645F8D39E4217D3013F29464B46F6
:1086A0003A463046FFF7A6FF3546ABE7934506D27C
:1086B000C4F800C045F8043CD9E7934502D2C4E9A8
:1086C00000A3D4E79645CFD2F2E746F8042B186012
:1086D000CEE72DE9F84F04460D461746994600F1BE
:1086E0000408291B402919DD8E10CFB9B11E49108D
:1086F00054F8213032462046FFF76EFD59B101395A
:10870000F6E755F8043D22682A602A1B92100021E2
:108710002046FFF761FD2B1B042BF2DCBDE8F88F30
:10872000C910D4F804A054F821009AF928B090F99F
:1087300028E055F804CC23689CF92820F3454646E8
:108740002BDD964522DD206044F821302B4622683F
:1087500092F928C03246116891F928006045164602
:1087600002F10402F7DC1A1F134652F8040990F9CB
:1087700028E0E645F8DB9E4217D3013F29464B46E9
:108780003A463046FFF7A5FF3546AAE7934506DD92
:10879000C4F800C045F8043CD8E7934502DDC4E9BD
:1087A00000A3D3E79645CEDDF2E746F8040B196047
:1087B000CDE72DE9F84F04460D461746994600F1DE
:1087C0000408291B402919DD8E10CFB9B11E4910AC
:1087D00054F8213032462046FFF757FD59B1013990
:1087E000F6E755F8043D22682A602A1B9210002102
:1087F0002046FFF74AFD2B1B042BF2DCBDE8F88F67
:10880000C910D4F804A054F821009AF928B090F9BE
:1088100028E055F804CC23689CF92820F345464607
:108820002BDA964522DA206044F821302B46226864
:1088300092F928C03246116891F928006045164621
:1088400002F10402F7DB1A1F134652F8040990F9EB
:1088500028E0E645F8DC9E4217D3013F29464B4607
:108860003A463046FFF7A5FF3546AAE7934506DAB4
:10887000C4F800C045F8043CD8E7934502DAC4E9DF
:1088800000A3D3E79645CEDAF2E746F8040B196069
:10889000CDE72DE9F84F04460D461746994600F1FD
:1088A0000408291B40291CDD4FEAA10ADFB9AAF1FF
:1088B0000206761054F82630524631462046FFF71D
:1088C000F5FB5EB1013EF5E755F8043D22682A60EC
:1088D0002A1B921000212046FFF7E8FB2B1B042BDC
:1088E000F2DCBDE8F88FC910D4F804A054F82100D8
:1088F000DAF824B0D0F824E055F804CC2368DCF88A
:108900002420F34546462AD9964521D9206044F8CB
:1089100021302B462268D2F824E031460868426AAA
:1089200072450E4601F10401F8D8191F0B4651F8A3
:108930000429D2F824C0E645F8D89E4217D3013F57
:1089400029464B463A463046FFF7A3FF3546A8E78F
:10895000934506D9C4F800C045F8043CD9E79345CF
:1089600002D9C4E900A3D4E79645CFD9F2E746F887
:10897000042B1860CEE700002DE9F04F00F50C53F2
:1089800000F52E52BBB081460F4614332C32002521
:10899000596A31B13AA901EB8501013541F8C83C6A
:1089A0002DB22C339342F3D108AE06EB8508B045C7
:1089B0004FEA850414D0A210B2FA82F2C2F11F026B
:1089C0004FF00003520041463046FFF762FF402C53
:1089D00023DD18A93046FFF72EFD18ACA04517D1AE
:1089E000DFF88CB03C464FF000084FF00A0A4545CE
:1089F00002DDE31B852B15DDBC4204D120461D4959
:108A00001BF07BFD0634002323703BB0BDE8F08FE4
:108A10002046FFF7F1FA0434E0E741463046FFF71D
:108A20000AFDDDE756F82810B8F1000F01D004F870
:108A300001AB042205A8039103F026FDD9F85C00E0
:108A400003681B68984703994B6A91F928200092A4
:108A5000C31A05AA594620461BF02CFB23461C4688
:108A600013F8012B002AFAD108F10108BFE700BF73
:108A7000536B02085C6B0208A0F1C800FFF77CBFD3
:108A8000036810B51B68044698476368834228BF93
:108A9000581C606010BD2DE9FF41044640689DF8F8
:108AA00028701D460368DB6B1646984760680368AC
:108AB0002946D3F8F0309847606803683146D3F808
:108AC000EC3098470022394660680BF0DAFF6068A6
:108AD00084F82450092D036834BF4FF020084FF06C
:108AE000100841461B6E984733462A46CDE9007868
:108AF000214602A807F0D6FC6368029AC3F8CC218D
:108B0000039AC3F8D02104B0BDE8F081406803683F
:108B10001B6F1847406803685B6F18472DE9F043E7
:108B20000346006DDFF85880D3E90495036885B0EB
:108B30001B6A0E46984704464046FFF7E7FF074684
:108B40004046FFF7E7FF80463846F8F7E7FA07B2F6
:108B500040464FF47A73B5FBF3F5B9FBF3F3039595
:108B60000293F7F751FC24B2CDE900013B460549D9
:108B7000224630461BF09EFA05B0BDE8F08300BFE8
:108B8000E0370020636B0208A0F1C800FFF7C6BF02
:108B900038B50C2017F036FD08250024C32017F047
:108BA0004FFD013D0444F9D12046F7F70BFC0EA31D
:108BB000D3E90023F7F780FC0D4B0022F7F77CFC8C
:108BC0000C4B0022F7F778FC00224FF07F53F7F7A9
:108BD00073FC094B0022F7F76FFCF7F745FF80B2F3
:108BE00038BD00BFAFF30080AE47E17A14AEFB3F63
:108BF0000000144000408F400000303F2DE9F34159
:108C0000466DC76CB0F858800D480C46FFF7C0FFA2
:108C1000336805461B68304698473B6806465B69E3
:108C2000384698470749CDE900802A4620464FF448
:108C30007A73B6FBF3F31BF03DFA02B0BDE8F081A6
:108C4000E4390020B76B0208A0F1C800FFF7D6BFD7
:108C5000D0E9003213448B4209D9438901339BB2D6
:108C600043810089984234BF0020012070470123CE
:108C700001604381184670472DE9F84F00F50C5507
:108C8000143500F52E5A07460C46914698462E4656
:108C90000AF12C0A4FF0FF3B2022314620461BF000
:108CA000CAFA30B3736A5B4538BF354606F12C0605
:108CB00038BF9B465645EFD12B4604F12002206871
:108CC00061681E4603C6083494423346F7D1F86DF6
:108CD000C5F8209003681B6898474FF0814168628F
:108CE0004046F8F73FF8F8F719FA85F82800BDE88C
:108CF000F88F3546E0E7F0B51F468B8816469A0692
:108D00008DB005460C4627D10A78092302F00302EC
:108D1000D340DB0703D5CB880BB90B89E3B19DF8B2
:108D20004C201299684603F083FD9DF801309BB1F9
:108D30009DF8003003F00F03022B0DD194F90201CE
:108D4000F7F7BCFF4FF07A51F8F70CF83A460346B4
:108D500031462846FFF790FF0DB0F0BDF0B591F811
:108D60004A3003F0F002802A8BB005460C4621D130
:108D70004B88052B1CD990F84531CBB9504E4FF498
:108D80007A72D6E904010023F8F75EFAB16801446B
:108D900005F50B502C30FFF75BFF48B1618894F864
:108DA0004B30E26C092903F004034ED8002B53D159
:108DB0000BB0F0BD902AFBD14A88052AF8D903F000
:108DC0000F03022BF4D1252AF2D900F50056D6F86C
:108DD0000433002B6FD0D6F8081302F011F90028E5
:108DE00069D1E36CD6F804239A42E1D16A4604F1D2
:108DF000500304F1700C174618685968164603C6EC
:108E0000083363453246F7D1202205F16801384620
:108E10001BF011FA0028CBD094F90201284EF7F785
:108E20004DFF4FF07A51F7F79DFF4FF47A720446E9
:108E30000023D6E90401F8F707FAB2682346024492
:108E400039462846FFF718FFB2E7216D002BAFD057
:108E5000D5F8A0318B42ABD3922194F84A308DF8EB
:108E6000001094F802118DF80110CDF8022003F0E3
:108E7000010305F168020DF1060105F1880052F8C1
:108E8000044B41F8044B8242F9D1002B0CBF26223F
:108E90000E226946284602F0B2FE0446002887D01A
:108EA0002B6801461B6C28469847214682002846BD
:108EB00003F040FA7CE70023C6F8043378E700BFEC
:108EC000C03700202DE9F047089E9DF82480994680
:108ED000337805468A461746BBB305F59871304688
:108EE000F8F7CCF9002861D103260022514605F598
:108EF000247003F07DFDD0F884304B4504465DD2EC
:108F0000C0F88490E86D03681B68984794F8203097
:108F1000C4F8880023F00303334384F820303A4632
:108F200004F1620307F1200152F8040B43F8040B2B
:108F30008A42F9D18EB141F28831284602F06CF8AC
:108F400005F50053C3F8100307E0202200F5247054
:108F500003F032FD04460028BFD0B8F1000F02D064
:108F6000FF2384F82130E86DFFF78AFD05F5805670
:108F70000023C6F83807A6F83C3794F8203003F0F1
:108F80000303DA1E5342534186F83E3794F82030EB
:108F900086F83F37286E036804221B6805F5BA512E
:108FA0009847022386F844370D2008E0304605F53F
:108FB000A871F8F763F90646002896D00020BDE8AE
:108FC000F0870000F7B51E4D04461746D5E90401A9
:108FD0001E464FF47A720023F8F736F9A968014467
:108FE00004F50B503830FFF733FE10B9002003B002
:108FF000F0BD04F58055307885F8300803F0B8F9F5
:109000000028F3D004F5BF5095F83028711C1030BB
:1090100003F0BEF9C5F83877E06D03681B68984720
:109020000023C5F83C0704F5CA500093AC22012385
:1090300004F5BA51183006F007FD0830C0B2D6E783
:10904000C0370020F8B51F4D04461746D5E9040186
:109050001E464FF47A720023F8F7F6F8A968014427
:1090600004F50B503830FFF7F3FD08B90020F8BDC8
:1090700004F58055307885F8300803F079F9002838
:10908000F4D004F5BF5095F83028711C103003F06F
:109090007FF9C5F83877E06D03681B689847C5F815
:1090A0003C0704F5BA55084904F5D47304F58072F9
:1090B00028461AF0FFFF2846F8F7EAF80830C0B251
:1090C000D5E700BFC0370020976D0208F8B51C4DEA
:1090D00004461746D5E904011E464FF47A72002370
:1090E000F8F7B2F8A968014404F50B503830FFF7DF
:1090F000AFFD08B90020F8BD04F58055307885F83B
:10910000300803F035F90028F4D004F5BF5095F885
:109110003028711C103003F03BF9C5F83877E06D4A
:1091200003681B6898470023C5F83C0785F840375B
:1091300094F8453113B1802385F840370920DAE7E8
:10914000C037002010B5044688B000F5B4506A4618
:109150000221183004F040F86A46034604F1680121
:10916000204602F0A7FB08B010BD10B5D1F8CC1016
:10917000044601230EF0F1FC204610BD2DE9F04F0E
:10918000CFB005460C46164601462D4A06A899461C
:10919000FFF7EBFF06A80EF048FE002847D02B682B
:1091A000284F5B6928469847014606A816F098FDA7
:1091B0002078254BC0F3830AFFF77AF9002818BFFF
:1091C0001F46286DB4F802B00368DB6B98478046F1
:1091D000286D03689B6B98471C4905464846F7F77E
:1091E000C1FDF7F79BFF04902846F7F797FF039020
:1091F0004046F7F793FF5346CDE901B03246144994
:10920000009706A816F099FD227840F20713C2F3E2
:109210008302D340DB070DD594F84A3094F84B20F5
:109220000C4906A816F089FD06A80EF0B6FD4FB051
:10923000BDE8F08F084906A816F07FFDF4E700BFEF
:10924000476B020820110308F56B020800007A44FE
:10925000F76B0208406C0208C10C030810B490F8C8
:10926000E84014B110BCFFF789BF10BC7047000084
:1092700070B5CAB005460C46164601461D4A02A8FE
:10928000FFF773FF02A80EF0D0FD60B32B682846ED
:109290005B699847014602A816F022FD207816491E
:1092A000164AC0F38303FFF703F9002818BF0A46E4
:1092B000618802A8CDE900213246114916F03DFD32
:1092C000227840F20713C2F38302D340DB070CD5A8
:1092D00094F84A3094F84B200A4902A816F02DFD64
:1092E00002A80EF05AFD4AB070BD074902A816F058
:1092F00024FDF5E7476B0208F56B0208201103080F
:10930000516C0208406C0208C10C030890F8E83068
:109310000BB1FFF7ADBF704770B5CAB004460D463C
:1093200016460146134A02A8FFF71FFF02A80EF0D7
:109330007CFDE0B1236820465B699847014602A89E
:1093400016F0CEFC28780C490C4AC0F38303FFF7D3
:10935000AFF8002818BF0A46698802A8CDE90021A5
:109360000749324616F0E9FC02A80EF016FD4AB095
:1093700070BD00BF476B0208F56B0208201103089F
:10938000826C020890F8E8300BB1FFF7C5BF704758
:109390002DE9F8438C88A309013390465FFA83F9DD
:1093A00004F03F0401F10A05002600F168073CB90A
:1093B00018F80900B0428CBF00200120BDE8F883F6
:1093C0004A46394628461AF036FF08B90136F6B241
:1093D000013CE4B24D44EAE770B590F845410546DA
:1093E000002C3CD10B781846FFF76AF8A8B38A889E
:1093F00095F8706102F03F02964230D903F00306FF
:10940000012E0AD195F87161964228D9C3F38306DB
:109410006FF083043441E40707D5C3F38303042BBF
:1094200003D195F87231934219D905F50053D3F859
:10943000D832B3B195F8243263B1012B0BD00A4A6C
:109440000A48022B08BF02462846FFF7A1FF80F01A
:109450000100C0B270BD064AF6E70120FAE700201D
:10946000F8E71846F6E700BF1001002014010020BD
:109470001801002030B585B004464FF49063006EAB
:10948000ADF804300368042204F500551B680DF1A3
:1094900006019847DDF80630C5F804334EF6602122
:1094A000204601F0B9FD01A9C5F808030A220025EC
:1094B0002046CDF80A5002F0A2FB014618B12A4618
:1094C000204602F037FF05B030BD00002DE9F74F10
:1094D0000446402015461E460091FCF7C0FF20219F
:1094E000074606F059FCBE4B236033686665C4E945
:1094F00013750025C4E904551B686560304698471C
:10950000012384F82C30B74BA364B74B23600D9B29
:10951000E3650C9B23660E9BA4F85850C4E906052E
:10952000C4E90955C4E910552562636604F1680071
:1095300002F03AF8AD4B2360EC33C4F8C830AC4BC2
:10954000C4F8F030AB4BC4F82C32AB4BC4F83C320F
:10955000AA4BC4F84C324FF0000904F1F008A84BB4
:10956000C4F8F85000260027C4E95C55C4F86851D7
:1095700084F87851A4F87A5184F87C5184F8955194
:1095800084F89651C4F8985184F89C51C4F8A051BD
:10959000C4F82052A4F82452C4F83452C4F84452F7
:1095A000C4F85452C4E94867C4E94A67C4F8FC9057
:1095B000C4F86091C4F86C91C4F8A491C4F83882DE
:1095C000C4F84882C4F85882C4F86452C4F85C32C3
:1095D0008C4BC4F86C3204F5257B8B4BC4F8745269
:1095E00004F5B45AC4F8845284F8005184F8305118
:1095F000C4F8445184F85051C4F88051A4F88451FF
:1096000084F8A851C4F86882C4F87882C4F87C321F
:10961000C4F88882C4F84091C4F84891C4F84C91C9
:1096200004F524755A460AF1140A1046019201F015
:10963000ACFF019AA0325245F7D14FF4A05200215D
:1096400058461AF022FE04F580520D9BC2F8B0561F
:1096500004F1C80104F5CA5004F5C1554FF0000BE0
:10966000C2F89836C2F8A016009B6849C2F894B6B2
:1096700014351830C2F89C86C2F8A436C2F8A81671
:10968000C2F854B9C2F8AC06294605F04DFF04F5FE
:10969000F0502946083005F047FF04F500587823BC
:1096A0000422C8E9BC32B42304F50C5AC8E9BF321D
:1096B000C8F8ECB2C8F8F8B20AF1140A04F52E5B47
:1096C00055460BF12C0B28462C3501F05EFF5D450D
:1096D000F9D1B42128460EF01AF900250023002202
:1096E000C4E93623C4E93855C4F8D0502946C8F82F
:1096F0001053C8F8B85BC8F8B45B40F6980284F819
:10970000E850504688F80C53C8F8D8521AF0BDFDFE
:109710004FF07E53C4F8FC304FF07C53C4F84C310A
:109720003B4BC4F8603104F580703A49C4F8489165
:10973000202206F023FCC4E94867C4E94A6704F51F
:1097400098703549102206F019FC344BC4F84031AA
:109750004FF4A163A4F86831162384F8443142F62B
:109760000173A4F846312E4BC4F86C312D4BC4F86C
:10977000703144F24003A4F874314FF4FA730126B7
:10978000A4F87A314FF4E133C4F8803104F2851043
:10979000254984F87651A4F8246284F8786184F825
:1097A0007C5184F88461102206F0E8FB022304F562
:1097B0000B5084F89651C4F8985184F89C31C4F841
:1097C000A49184F8216284F822521022C8E9C1557C
:1097D00029461C301AF059FD204603B0BDE8F08F31
:1097E000A472020880EE360048730208FC6D02087D
:1097F000F06D0208A86D0208B46D0208C06D020881
:10980000CC6D0208D86D0208E46D020860370020B4
:109810009A99993EBA6C0208F47802088D67594407
:1098200000007A4240400840CF6C020837B5044639
:109830000D4601F0E5FF04F5B4502946C4F8CC50BC
:10984000183004F5CA5503F087FC1835D4F8CC104D
:1098500004F1680204F5247003F022F8D4F8CC1067
:109860000022284605F088FE284606F044F8014606
:1098700030B104F50B5201231C32284605F00AFFD3
:1098800094F86931009394F86831D4F86C21D4F8D5
:1098900040110A48FFF7FFF894F94411074806F011
:1098A0008CFD23682046D3F89C3098472368D3F872
:1098B000A030204603B0BDE830401847E037002014
:1098C0002DE9F04385B0054608469DF8309088465E
:1098D00014461E4606F08CFA074640B14B46324607
:1098E0002146284605B0BDE8F04302F09DB9214667
:1098F000404606F0C9FACDF80090ADF80C003346AA
:1099000003AA21462846ADF80E7002F0BAF905B058
:10991000BDE8F0832DE9F041984600F500530E466E
:10992000D3F8D81200F50B5586B0044617461C35FF
:1099300011B30B88B3B100F5CA50012302AA183045
:1099400005F0A8FE0028284617DD06F051FACDF8EC
:1099500000803B46324602A92046FFF7B1FF06B021
:10996000BDE8F081284606F043FA43463A463146C0
:10997000204602F059F9F2E7284606F039FA0028A5
:10998000F3D1CDF800803B4632462946E4E72DE985
:10999000F04F0E460978C1F3830185B007290446CC
:1099A00098469146DDE90E3068D1002504F5805ACD
:1099B00019681D54FF208AF830081879451E1E2D9D
:1099C00040D93078FEF77CFD0433019000932046A7
:1099D0000B464146FFF776FA054600284ED0202276
:1099E000414604F5247002F0E7FF8346002854D076
:1099F00090F82170FF3F18BF01273078FEF760FD17
:109A000004F5B9539AF830281833002847D0CDE927
:109A100002350123019333790093414606F10A038D
:109A20004A46204601F0ECFF014638B3B3889B0953
:109A30000133DBB24FF49672204605B0BDE8F04F1B
:109A4000FFF768BF01280AD13078FEF731FDA8B1D1
:109A50000A46053341462046FFF7B4FABCE7022820
:109A60000AD13078FEF724FD40B10A46053341465D
:109A70002046FFF7E7FAAFE7032802D005B0BDE8BC
:109A8000F08F3078FEF714FD0028F7D00A46053332
:109A900041462046FFF71AFB9EE70746ADE7FF2A3F
:109AA000CDE9003508BFC7F103074FF001014B4670
:109AB000424620460CBFFFB2012701F0B5FF014628
:109AC0000028DBD0012F0DD14FF496730E9304F5CF
:109AD000BF529AF830381032204605B0BDE8F04F3A
:109AE00002F000B9022FA1D14FF496729BF82130F9
:109AF0000E920BF12202EFE773B50D4604461646AF
:109B0000FFF720FB014668B176B194F823020130DB
:109B1000C0B20A4604F50B5100902B461C3120467A
:109B2000FFF7CEFE02B070BD2A46204602B0BDE867
:109B3000704002F0FFBBA0F1C800FFF7DDBF0000DE
:109B40002DE9F04700F500571E4697F80C338AB010
:109B50000446884615464BBB154612F8013B202BA0
:109B6000FAD02846F7F794FB042808D9AB787C2B69
:109B700005D12B883380AB78B370033503367D492C
:109B8000082228461AF057FB8146002840F0A5809D
:109B90000835202128461AF080FB002870D176492C
:109BA00030460AB0BDE8F0471AF0A7BC104606F0F0
:109BB000F4F9F8B92B469846994613F8012B202A58
:109BC000F9D0A8EB05054F4619F8010B05F0C0FCCC
:109BD0000028F8D13B780BB138704F46B94617F8DA
:109BE000013BEBB96B1E062B1DD9002333700AB065
:109BF000BDE8F08704F5805404F608614FF49662DE
:109C000004F658101AF081FCB4F862295B4900236D
:109C1000304687F80C330AB0BDE8F0471AF04ABA6C
:109C2000462BDBD1DEE798F80030002BDDD004EBCB
:109C3000850505F50055D5F8B472002FD5D004F58B
:109C4000CA504146183005F07BFD04F5F0543A88BF
:109C50000834074660B103884146204605F0A0FD60
:109C60000028C2D037B13B790371C5F8B802BCE710
:109C70000346F1E799F80030463B18BF0123F3E7AC
:109C800082462A460AF8019BAAEB0503402BA8BF8F
:109C9000402303EBD3734FEA6308414602A802F066
:109CA0002BFCC0B1504619F09BF8C0B2009043465F
:109CB00002AA04F1680104F5247002F0EBFE40B141
:109CC00041F28831204601F0A7F92D49C7F8100369
:109CD00066E72C4964E72C4962E7B8F1000F2BD105
:109CE0002A492846F7F7CAFA074628BB28492948CF
:109CF000DFF8A490DFF89C80DFF8A0A016F00AF847
:109D000004F5257504F58053D3F894369F42BFF6C9
:109D10006CAF95F8202062B14946404616F00DF828
:109D200029464046202202F0C9FB5146404616F023
:109D300004F80137A035E5E71949122228461AF040
:109D40007AFA60B9113515F8013F202BFBD00BB121
:109D5000144925E72046FFF78DFB134920E704F55A
:109D6000B45033462A46414618300AB0BDE8F047A1
:109D700004F080BCF06C0208F96C0208D96C02088F
:109D80000A6D02080D6D0208226D0208336D02088B
:109D90003B6D0208283C0020406D0208C10C0308FE
:109DA000466D0208596D0208816D020837B50446F8
:109DB00001F028FDD4F8E410002963D0204601F01A
:109DC0001FF900285ED02046FFF7BCF902460028A4
:109DD0006CD123682046D3F8A030984723682046EA
:109DE000D3F89C30984704F50055D5F8B41B91B1D1
:109DF000204601F005F970B10023C5F8B43B95F891
:109E0000C53B009395F8C43BD5F8C02BD5F8BC1BD7
:109E10002D48FEF740FED5F8B81B91B1204601F061
:109E2000EFF870B10023C5F8B83B94F8693100939E
:109E300094F86831D4F86C21D4F840112248FEF728
:109E40002AFED5F8101369B1204601F0D9F848B1BF
:109E5000D4F8CC10002204F5247002F06BFE00232D
:109E6000C5F8103316F04CFDD4E93631D4F8D020C3
:109E7000C4F8D000821A9B1841F10001C4E93631C0
:109E800003B030BDD4F8E0100029ACD0204601F07A
:109E9000B7F80028A7D02046FFF754F9014600285C
:109EA0009CD00022204602F045FA97E794F823322E
:109EB0000133DBB204F50B5100931C310023204623
:109EC000FFF7FEFC85E700BFE0370020C06C08B557
:109ED00003685B6998470028D4BF0020012008BDB3
:109EE0002DE9F04F00F58056DBB0C6F838271A7818
:109EF000012A04460D4662D1C048C14DFEF748FE16
:109F0000ADF8A000E06C03685B699847ADF8A2006B
:109F1000206D03681B6A9847ADF8A4002846FEF739
:109F2000F5FDF7F7FBF8EB682A932B69ADF8A6006F
:109F30004FF47A72D4E936012B934FF47A76236981
:109F4000B3FBF6F32C930023F7F77EF9236B2E93E4
:109F5000636B2F93A36B3093E36B2D903193284663
:109F6000B4F85830ADF8C830FEF7D4FD4FF0814159
:109F7000F6F7F8FEF7F7D2F8636EADF8CA00D3F83B
:109F80000825D3F80C35ADF8CE306369B3FBF6F392
:109F900004F5B95434936B69ADF8CC20359328AAF5
:109FA0001C3436AD134603CBAB42206061601A46C9
:109FB00004F10804F6D13C205BB0BDE8F08F032A21
:109FC0002ED100F52E562C3630465F780DF0B2FCBF
:109FD0008A48FEF7DDFDF6F76DFE8A49F6F776FF53
:109FE0000121024630460DF05BFD95F820108648B1
:109FF00011F003011CBFFF43F9B2324600F0D0FD5F
:10A0000030460DF09AFC054630460DF098FC0146AE
:10A0100004F5B9502A461C301AF077FA281DCBE710
:10A02000052A2DD191F8202002F00302032A40F0E6
:10A0300056815A789B781A4340F0518100F5257576
:10A04000042341F23877D6F894168A421846B3DAD8
:10A05000AD2BB1D895F8201079B1D919D5F800C039
:10A0600044F801C06018A9888180991D54FA81F1D3
:10A0700095F82000C8550733DBB20132A035E2E77E
:10A08000062A40F018815D78002D40F0288193F871
:10A0900006809A78B3F803700492B8F1200F5A79C9
:10A0A00000F52E5100F50C5328BF4FF02008143353
:10A0B0002C31586A30B15AA800EB8500013540F8C0
:10A0C000C83C2DB22C338B42F3D1002A46D128AEA6
:10A0D00006EB8509B1454FEA850A16D04FEAAA0278
:10A0E000B2FA82F2C2F11F024FF000035200494659
:10A0F0003046FEF70DFABAF1400F2ADD304638A996
:10A10000FEF77DF938AEB1451ED108F1050A07AB5F
:10A110004FF0000B5FFA8AFA03EB0806D946049B5E
:10A120004B4502DDBD4200F3A38004F580535A463F
:10A13000A3F83C57A3F83E9707A904F5BA501AF0C4
:10A14000E4F90BF1080037E73046FDF7E4FF043689
:10A15000D9E749463046FEF752F9D6E7012A27D11A
:10A1600028AE06EB8509B1454FEA850ACDD04FEA06
:10A17000AA02B2FA82F2C2F11F024FF000035200AB
:10A1800049463046FEF736FABAF1400F0BDD30464D
:10A1900038A9FEF718F938AEB145B6D03046FEF70B
:10A1A0000EF80436F8E749463046FEF70CF9ACE7FE
:10A1B000022A30D128AE06EB8509B1454FEA850A5F
:10A1C000A3D04FEAAA02B2FA82F2C2F11F024FF004
:10A1D0000003520049463046FEF77BFABAF1400FC1
:10A1E00014DD304638A9FEF7D0F838AEB1458CD032
:10A1F0003046FEF73BF80436F8E700BFE4390020AC
:10A20000E037002000007A4460370020494630469D
:10A21000FEF7BBF879E7032A7FF477AF28AE06EBA9
:10A220008509B1454FEA850A3FF46FAF4FEAAA02AC
:10A23000B2FA82F2C2F11F024FF000035200494607
:10A240003046FEF7B6FABAF1400F0CDD304638A9B9
:10A25000FEF77DF838AEB1453FF457AF3046FEF714
:10A260005EF80436F7E749463046FEF770F84CE7EB
:10A270000BEB0A03822B05933FF757AFE06D28AB3A
:10A28000026853F827B012689047DBF8242059463B
:10A29000831A4246A6EB080003931AF036F9039B93
:10A2A0003360059B9BF82820327109F1010956445F
:10A2B00001379B4633E7072A11D100F5B95500F560
:10A2C000D4731C35074A0849009300F5807328466B
:10A2D00019F0F0FE2846F6F7DBFF04306CE60020AC
:10A2E0006AE600BF94690208946D02082DE9F04FF8
:10A2F00003F6F223B5B050F823700E46002F3E99B6
:10A300000491DDE93F9B0446C0F2F38000F58053E1
:10A31000D3F894369F4280F2EC80A0257D4300F56F
:10A32000247305F1040805939844002A5FD1471966
:10A33000D9F800A0D7F81833534580F0DA80ABF194
:10A3400004030093524609F104034146FFF7C8FD98
:10A350008146002800F0CD80C7F818A3E06D03689F
:10A360001B689847C7F81C033078FEF7A9F804F576
:10A37000B9531833E0B1CDE90239012301933379A0
:10A3800000934146049A06F10A03204601F038FB87
:10A390000146002800F0AD80B3889B090133DBB291
:10A3A0004FF49672204635B0BDE8F04FFFF7B2BAD1
:10A3B000CDE900390121049B4246204601F034FBDF
:10A3C0000146002800F0958097F8B532FF2BE3D0C6
:10A3D0004FF4967005F126023E9004F52470104467
:10A3E0000246204635B0BDE8F04F01F07BBC022AA2
:10A3F0007FD1BBF1050F7CD9431993F8B42202F049
:10A400000302032A75D199F80420D9F800A0910815
:10A41000072A07916DD8D3F818230592524568D8BA
:10A42000C3F818A3C06D0693026812689047069B94
:10A430000799C3F81C03002309F80B3009F1050B39
:10A4400019BB5846F6F724FF2023CDE900834A467E
:10A45000431D042109A802F091F8099B0A930AA957
:10A460000422204601F00BFB014670B1A02303FB40
:10A47000074393F8B532FF2B3ED1B3889B090133D4
:10A48000DBB2C8222046FFF745FA059B53453ED173
:10A4900000238DF82D300DF12D00F6F7F9FE8146E1
:10A4A00038B3E06DFEF7ECFA042350458DF82C30FC
:10A4B00009F1050308BF0AF1010001930AAB0A90F4
:10A4C00000930221049B4246204601F0ADFA01466A
:10A4D00078B1A02303FB074797F8B532FF2B1ED1B5
:10A4E000B3889B090133DBB24FF416722046FFF7A5
:10A4F00011FA35B0BDE8F08FC82005F126020090B2
:10A5000004F524700244204601F0ECFBBDE70DF198
:10A510002D035A4651462046FFF712FBBBE74FF486
:10A52000167005F12602009004F5247010440246CE
:10A53000204601F0D7FBDCE710B5C8B0D0F8CC104E
:10A540000E4A684600230DF008FB68460DF06DFCCE
:10A5500060B10B4C68460DF064FB20B168460DF00D
:10A56000F1FB011E04DA68460DF017FC48B010BD7F
:10A57000C9B2204615F0B8FBECE700BF476B0208F4
:10A58000283C0020A0F1C800FFF7D6BF38B50C4624
:10A590008D18AC4200D138BD4FF48071002015F009
:10A5A00042FF04F8010BF4E716F0AAB913B504460C
:10A5B0000846694601F017FFD4F804256B4603CB23
:10A5C00004EBC20291605060D4F80435A02201333C
:10A5D00093FBF2F102FB1133C4F8043502B010BD55
:10A5E00037B504460846694601F0FDFE251D04F214
:10A5F000045408222946684619F01DFE18B928603F
:10A60000686003B030BD0835A542F2D1F9E7F7B56F
:10A610000E4604466946304601F0E5FE251D04F26B
:10A62000045708222946684619F005FE98B9337880
:10A6300003F00303023B012B07D9D4F80C35013397
:10A64000C4F80C35012003B0F0BDD4F8083501334F
:10A65000C4F80835F6E70835BD42E2D10020F2E73C
:10A660001FB5114C114B20464FF4A062002140F859
:10A67000043B19F00AFE00230420C4F80435C4F892
:10A680000C35C4F80835FBF7EAFE094A0260094AAE
:10A690000192094A00920346084A0949029409486E
:10A6A000FEF714FF04B010BD50320020886F02087E
:10A6B000706F0208C037002020010020E037002022
:10A6C000E439002008060020044A054B13600548C1
:10A6D000EC33C2F8C8300DF026B900BF08060020E0
:10A6E000FC6D0208B431002070B506229AB04FF418
:10A6F000E131354815F084FA4FF47A7016F004F918
:10A70000324B0022012113201A7115F0AFFF0121F5
:10A71000132016F015F80221C12015F0A7FF00F054
:10A72000A9FA00B9FEE72A4C2A4805F041FE15F0C7
:10A730006BFE204605F0CAFF274B284A284918948B
:10A7400018A8199304F074FE00BB684600F0E0FA04
:10A750002248244D6022694619F0D7FE0A2405F1EB
:10A76000680695F86830013BDBB2FD2B09D96846D5
:10A7700000F0CEFA60226946304619F0C6FE013C70
:10A78000EFD1164A164918A804F07AFE16490E4869
:10A7900015F0A6FA202211490B4801F08FFE0A4855
:10A7A00015F0A6FA114B124800241C7000F033F982
:10A7B00007490C48FFF73AF80A4822464FF47A5105
:10A7C000FFF79AF91AB070BD283C0020E439002048
:10A7D000143A0020E0370020CB85020870060020E4
:10A7E000416B020808060020546F0208640500202F
:10A7F000603700202DE9F0433B483C4E3A4FA9B06A
:10A80000F6F746FD4FF000090446304615F070F8A3
:10A8100068B19F2C0DD0A046304615F02FFAC5B276
:10A820000A2D2BD1304615F063F80028F4D19F2C67
:10A8300032D12D4B0D2283F89F209F242A4D013CBD
:10A840002B5D0D2B2AD10A21284815F04DFA002145
:10A850006B46274829552A468DF80010FFF770F9F6
:10A860009DF800303BB12349204815F039FA1F48C4
:10A87000694615F04FFA00232B700FE0013429468A
:10A88000304607F8085007F8049015F02DFA0D2D02
:10A89000BBD19F2CD2D1CCE7002CCFD1144C204679
:10A8A000FFF784FA16F02CF8134BD3E904259969C5
:10A8B0009861411A521845F10005C3E9042594F83E
:10A8C000953173B12046FFF701FB50B90B4B1B6864
:10A8D0004FF47A715943204629B0BDE8F04300F0A7
:10A8E0008FBB29B0BDE8F08364050020283C002020
:10A8F00008060020626F0208C03700201C010020FB
:10A90000004870470000C07F00207047002070475B
:10A9100070474FF0FF307047704700207047704716
:10A9200000207047002070470020704700207047CB
:10A9300000207047002070470020704700207047BB
:10A94000002070470020704700487047946F02084D
:10A950000020704700487047946F02084068036801
:10A96000DB681847B0F9180070470177704700207E
:10A970007047002070470020704700797047000042
:10A98000BFF34F8F0549064BCA6802F4E0621343D8
:10A99000CB60BFF34F8F00BFFDE700BF00ED00E0CD
:10A9A0000400FA0500207047436893F8700170476F
:10A9B00010B54FF47A7204460023D0E90401F6F78B
:10A9C00043FCA368184410BD704700207047002066
:10A9D000704700207047002070470020704700003B
:10A9E00000487047A26F02087047F8B507460C464A
:10A9F0008E18B44200D1F8BD78680368D3F8A4304B
:10AA000098474FF480710546002015F00CFD454035
:10AA100004F8015BEDE710B5044620300EF0A4FF0A
:10AA200084F8580010BD08B50023037101211320DC
:10AA300015F01CFE0121132015F082FEBDE8084030
:10AA40000221C12015F012BE0121132015F078BE9D
:10AA50000021132015F074BE08B5F8F735FE72B664
:10AA6000BDE80840F8F738BE07B50023009340F270
:10AA7000762202236FF07F410AF09FFE03B05DF85B
:10AA800004FB10B54FF4EE710446FBF7ECFC2046D6
:10AA900010BD4068002108F003BB10B5044615F056
:10AAA0002FFFD4E90431A269A061821A9B1841F1F9
:10AAB0000001C4E9043110BD10B500220023C0E933
:10AAC00004238160044615F01BFFA06110BDF8B59A
:10AAD000446823682046D3F884309847054615F02B
:10AAE0000FFF15F020070CD023683C21D3F88C30E1
:10AAF000204698470023C4F8D43184F8D831002088
:10AB0000F8BD15F0100394F8D86115D1002EF2D1DC
:10AB100015F004052AD0D4F8D4318BB1C01AD4F87A
:10AB2000CC3198420ED923680421D3F88C302046CA
:10AB30009847C4F8D461E2E736B9012384F8D831E4
:10AB4000C4F8D4010120DBE7D4F8D431C01AD4F81A
:10AB5000D0319842F6D923683C21D3F88C30204676
:10AB60009847C4F8D47184F8D871C8E7C4F8D451B0
:10AB700084F8D851C3E7036810B51B6C04469847A6
:10AB800020B92046BDE8104005F054BC10BD10B4FB
:10AB90004468134694F8702110BC05F079BC00009D
:10ABA00070B590F8586086B01446E6B10F4B039329
:10ABB0000125049305930023CDE9003503AA04ABD6
:10ABC00005A920300FF0DCF8039A294620460CF046
:10ABD00059FF049A294620460CF05BFF059A294646
:10ABE00020460CF064FF304606B070BD0000C07F08
:10ABF00030B5D0E9003485B01B6E9847012120465E
:10AC000009F0A0FB01220021204609F0C0FB7F23B0
:10AC10008DF80F3000220123CDE9003289210DF19A
:10AC20000F02D4F86C0106F050FFD4F86C311868AC
:10AC300003680521DB69984715F062FE0546D4F8E4
:10AC40006C311868D96A02681269904720B115F012
:10AC500057FE401B322806D9D4F86011204608F070
:10AC6000F4FA05B030BDD4F86C31186803685B6D38
:10AC70009847E4E730B51D4887B0002105F0E6FFAE
:10AC80001B4A1C491C480AF02EFB1C4B0493102243
:10AC90001623CDE90232122105230024CDE900312B
:10ACA000174A184914480594082307F061FA054625
:10ACB00058B11549154815F013F814480A222946C9
:10ACC00015F088F8204607B030BD01221146012456
:10ACD00009480AF07DF9009441F2210341F60F5230
:10ACE000214605480AF024FAECE700BF643A002048
:10ACF0002872020888720208083800209A99D93F01
:10AD000000007A428D675944B46F0208283C002045
:10AD100013B5054B00936946044B0193044600F0BC
:10AD20004FFC204602B010BDD86F02080838002042
:10AD300073B5244E244B33604820FBF790FB234D22
:10AD4000044607F09FF82146284607F035FA204BC5
:10AD50002B60422240F65E73C5E973231D4B1E4AE9
:10AD60001A600024C3E90156C5F8D44185F8D841DA
:10AD70001A4D83F82440C3E90344194B2B60194B47
:10AD8000AB6000220023C5E904236C6015F0B8FD18
:10AD9000A861154D002200232846C5E90223C5E914
:10ADA0000423C5E90623114B40F8203B104B4FF01C
:10ADB0000131CDE9001369460FF05AF885F8584083
:10ADC00002B070BDE4390020887102080838002004
:10ADD000E46F0208E037002004710208C037002049
:10ADE00074710208EF93446660370020087202080D
:10ADF00005040076704770477047704700487047F9
:10AE0000CB85020800207047002070470020704763
:10AE10004FF07E507047C82070474FF47A607047FB
:10AE200070B50F481646F5F793FEF5F7EDFA0246B2
:10AE30000B4600200B4916F085FA0B4B0022F5F764
:10AE400083F9044630460D46F5F7BCFA02460B4638
:10AE500020462946F5F730FBF5F7DEFD70BD00BF53
:10AE60009A99593F000024400000F03F002370B53C
:10AE70000446C0E90C33C0E90E33A0F85830406DE9
:10AE800003681B689847236820625B6B20469847DD
:10AE90002368A0649B69204698470646A06CF5F796
:10AEA00009FF4FF07E5105463046F5F753FE014647
:10AEB0004FF07E50F6F70AF801462846F5F752FFA4
:10AEC000F6F752F92064606D03681B689847606468
:10AED000206D03681B689847206D03681B6B9847BB
:10AEE00084F82C0070BD2DE9F0410446406D0368E4
:10AEF0001B689847656C2368451B9B69064620467E
:10AF000098474FF07E51F5F725FE01464FF07E50F1
:10AF1000F5F7DCFF236807465B6B204698478046C1
:10AF20002846F5F7C7FE3946F5F71CFFF6F71CF97A
:10AF3000054670B14046F5F7BDFE3946F5F712FFFC
:10AF4000F6F712F9236C66641D44A84294BF20648E
:10AF50002564BDE8F081F8B51E4613780B701746DE
:10AF60009A090D4601D00020F8BD03F00302092321
:10AF7000D34013F0010319BFB7F80130EB800B8108
:10AF8000CB801BBFB7F803302B81012105217C5CEE
:10AF9000AC80A209032AE6D004F03F0402FB04447B
:10AFA000E2B2402ADFD801315418B442DBDC394424
:10AFB00005F10A0019F0A9FA321B92B2B82A6A8088
:10AFC000D1D8391905F14A0019F09FFA0120CBE7D1
:10AFD00010B50446C06C03681B68984730B9B4F8D4
:10AFE000583043F00103A4F8583010BD002383808B
:10AFF000438080F80231F8E7C06C03685B6818474B
:10B00000406D036810B51B680C469847001B00286C
:10B01000D4BF0020012010BD406D036810B51B682F
:10B020000C469847204410BD03682DE9F0411B6889
:10B0300005460E469847044630B9E86C0368314629
:10B040005B68BDE8F0411847012812D0EF6C3B68FF
:10B0500020F07F412846D3F80880FFF7DDFF220E5D
:10B06000013A034631463846C446D2B2BDE8F04103
:10B070006047BDE8F0812DE9F0410446006D0368AA
:10B08000C2B05B68FF2202A99847061E72DD2368E2
:10B09000206D5F680368DB6B98470546206D036889
:10B0A0009B6B98472946024602AB20460096B8475C
:10B0B000E06C03681B689847054600285AD0014693
:10B0C000334602AA2046FFF746FF00284DD0206DE8
:10B0D0000368DB6B98474FF08141F5F743FEF6F7C5
:10B0E0001DF885F80201276D3B683846D3F80C80BF
:10B0F000DB6B9847324601463846C0470746206D0D
:10B10000036831469B689847636903446361236819
:10B1100006462846D3F8088001F04FF93B46024620
:10B1200029462046C0472B789B0726D4A36B0133C2
:10B13000A36323683946DB693246204698473128A5
:10B1400001461DDDE66CB0F5FA4F3368A8BF4FF439
:10B15000FA4120465F6AFFF75FFF294602463B46F9
:10B16000304642B0BDE8F0411847E06C036829461C
:10B170005B68984742B0BDE8F081E36B0133E3635D
:10B180002946204642B0BDE8F041FFF74DBFF0B57B
:10B19000C56C04462B68406D1E690368C1B01B680E
:10B1A000984701462846B04760B32046FFF79BFE0C
:10B1B000206D0368FF219B689847236CB3EB500F09
:10B1C0004FEA500520D2236820469B6998470646DF
:10B1D000206C281AF5F76EFD4FF07E51054630467B
:10B1E000F5F7B8FC01464FF07E50F5F76FFE0146CB
:10B1F0002846F5F76BFEF5F7B7FF01462046FFF747
:10B200000BFFA06141B0F0BDA1692046FFF7F8FE39
:10B210000028F7D0206D03685B6B9847C0B1E369E5
:10B2200023B9606D03681B689847E061606D03682F
:10B230001B689847E369C51A236820465B6A9847EC
:10B24000854240D9B4F8583043F00203A4F858308E
:10B25000E56C606D0023E3612B68DE6803681B68A2
:10B26000984701462846B04760600028CAD0037856
:10B270008DF80030092203F0030322FA03F3DB0701
:10B2800041BFC388ADF801300389ADF8033054BF26
:10B290000123052382880DF803205D1C027900F14B
:10B2A0000A010DEB050001F073F866687288054429
:10B2B0005319FF2B0CDDE06C036831465B6898473F
:10B2C000002363609EE7236820461B6A984794E743
:10B2D00006F14A010DEB050019F017F9206D76888B
:10B2E00003682E4431469B6898470546606D0368A5
:10B2F0001B689847E060206D036832461B69694609
:10B300009847064678B96568236828461F6901F0A2
:10B3100054F8294602462046B84761682046FFF7A0
:10B320006BFE66606EE705EB450569082046FFF792
:10B3300073FEA06066E7F8B5416A0446FFF760FE59
:10B34000C8B1256D2B685E6A236820469B6A9847C2
:10B3500001462846B047256D2B689E6A2368204623
:10B36000DB6A984701462846B0474FF4FA61204609
:10B37000FFF752FE6062206D0368DB699847206D1D
:10B3800003681B6B984794F82C30834217D084F8DD
:10B390002C00B0B9606D03681B6898472062606D2F
:10B3A00003681B689847236AC01AB0F5FA5F82BF2A
:10B3B000B4F8583043F00403A4F8583001E0002BEF
:10B3C000EDD06368002B64D0206D03685B699847FB
:10B3D000002800F09880606D03681B689847E56856
:10B3E0002369471B3B44236106462046FFF77BFD4C
:10B3F000236C9F427CD900232364236820469B69E9
:10B4000098470646206CC0F16400F5F753FC4FF0F6
:10B410007E5105463046F5F79DFB01464FF07E50C4
:10B42000F5F754FD01462846F5F750FDF5F79CFE6B
:10B4300001462046FFF7F0FDA061206D03689B697F
:10B44000984761688A884888930902F03F0203FBA5
:10B450000222D2B223680232DB68024420469847B7
:10B4600061680B789B0755BF236B636B0133013316
:10B4700054BF236363632046FFF7BEFD0023636070
:10B48000236820461B6B984701462046FFF7C4FD02
:10B49000A062236820461B6B9847002811DDA16A33
:10B4A0002046FFF7ADFD60B1206D0368DB6A984769
:10B4B000236820461B6B984701462046FFF7ACFDEA
:10B4C000A062E56C606D2B689E6A03681B689847F4
:10B4D00001462846B047014610B12046FFF7A4FDBB
:10B4E0002046FFF7C8FD2046BDE8F840FFF74FBEF5
:10B4F0001D44AD1B632D25647FF67FAF606D03682F
:10B500001B68984798E7A1682046FFF779FDA0B12E
:10B51000206D03689B69984761688A884888930909
:10B5200002F03F0203FB0222D2B22368023202443D
:10B530001B692046984761689DE7F8BD2DE9F047F3
:10B54000064608790C461746984600F011FFF56C40
:10B5500088B16388B82B0ED82B6841463046D3F8A3
:10B560000890FFF759FD3A46034621462846CC4647
:10B57000BDE8F04760472B68214628465B68BDE878
:10B58000F04718470368DB69184710B520220446C6
:10B59000002118F07AFE204610BD10B4044608467B
:10B5A000214610BC0BF072B810B50446FFF7EDFF52
:10B5B0004022002104F1200018F067FE204610BD53
:10B5C00030B50D4689B00446FFF7DFFF2B686946AA
:10B5D0001B6828462022984720466A4604F120012D
:10B5E0000EF068FD204609B030BD0000F0B5B1B0E6
:10B5F0000146044668460EF07AFD9DF80030013B96
:10B60000DBB2FD2B30D81B4B20AA03F140071646B6
:10B6100018685968154603C50833BB422A46F7D156
:10B62000154B08AA03F1200C1746186859681546EF
:10B6300003C5083363452A46F7D12246394610A888
:10B640000EF06EFC3246694618A80EF069FC202206
:10B6500018A910A818F0EFFD30B910AB13F8012BA2
:10B660002AB901302028F9D1002031B0F0BD0120E5
:10B67000FBE700BFDC7202081D73020838B50C46F8
:10B680000546014620222046FFF77CFF20280AD1EC
:10B69000402205F120012046FFF774FFA0F140038E
:10B6A0005842584138BD0020FCE738B50B680C46BD
:10B6B0005B680146054620222046984720280BD18A
:10B6C000236840225B6805F1200120469847A0F1DD
:10B6D00040035842584138BD0020FCE73F2A70B56E
:10B6E0001ED95F2A00F1200300F1600407D853F847
:10B6F000042B41F8042BA342F9D1402070BD1A4617
:10B700000D4652F8046B45F8046BA242F9D1403162
:10B7100050F8042B41F8042B9842F9D16020EDE752
:10B720000020EBE7602A30B40B4613D10A4603F140
:10B73000400400F1200152F8045B41F8045BA2428E
:10B74000F9D1603352F8041B40F8041B9A42F9D136
:10B7500030BC7047402AFBD100F120010A4603F1BA
:10B76000400453F8045B42F8045BA342F9D130BCB7
:10B770000EF0BDBC13B50446084611461A4604F146
:10B780002003009323460FF0C1FA02B010BD0B4610
:10B79000114600F1200218460EF0C2BB70477047F8
:10B7A00000207047704770477047002070470020A6
:10B7B000704700207047002070470020704770B528
:10B7C000046D2368054608469E6800F0F6FD0146B4
:10B7D0002046B047052204460021286E00F042FEB4
:10B7E00034235C436423B4FBF3F4604370BD08B5B9
:10B7F00004220121006E00F035FE7823584308BD75
:10B80000FFF734BBFFF797BDF8B58B8803F03F0413
:10B81000013CE4B223F03F031C438C80A4090134B3
:10B820000D46E4B201F10A060027AB8803F03F039E
:10B8300013FB04F3BB4200DCF8BD3046264422462D
:10B840003146274418F061FEEFE7F8B50A788B8897
:10B85000920706460C4601D50020F8BD03F03F07CD
:10B860009B090133DBB207FB0333402B07F10105D2
:10B87000F2DC0368DB6B98470028EDD0A2889209C0
:10B880000132D2B207FB024006F168010A3018F01B
:10B890003CFEA38823F03F031D433368A5801B6C47
:10B8A000214630469847A38803F03F03013340EA1E
:10B8B0000360D2E72DE9F043202B93B080460E467B
:10B8C00017461D4603D8FFF783FB044620B9002422
:10B8D000204613B0BDE8F0830346102203F84A2B3C
:10B8E00006F12009324652F8041B43F8041B4A456E
:10B8F000F9D1D8F85C0003681B6898472A46C4F859
:10B900006A008046394604F1AE0018F0FEFD05F1EC
:10B91000640363800DF1040C33461868596862466D
:10B9200003C208334B459446F7D12A4639460AA844
:10B93000CDF8248018F0E9FD05F1240301AA04F1F3
:10B940006E013046FFF716FFC2E72DE9F04FAFB0AA
:10B9500099469DF8E0A0DDF8EC804FEA9A130AF0D2
:10B960003F0403FB044408F105032344A62B0646C9
:10B970008B46174604D9002528462FB0BDE8F08F26
:10B98000FFF726FB05460028F5D0202303709BF81F
:10B99000003080F84A3096F8683080F84B304946DD
:10B9A00022460DF101008DF800A004F1020918F003
:10B9B000ACFD04F1B9030DEB09006B44B8F1000FC5
:10B9C00012D09DF8E42003F8B82C3A99424618F0BA
:10B9D0009CFD08EB09036A4605F14C01384600F06E
:10B9E00046FE02306880C7E7FF2203F8B82C336EAA
:10B9F0001A680146166818460422B047A31DEAE7F4
:10BA00007FB509788DF814100B9903910A9902916A
:10BA10009DF8241001919DF82010009105A9FFF7D1
:10BA200094FF07B05DF804FB2DE9F8430229DDF827
:10BA3000249007460D4690461E4603D809F111038F
:10BA4000B82B03D900242046BDE8F883FFF7C0FADD
:10BA500004460028F6D0AD00057098F8003080F854
:10BA60004A3097F8683080F84B3000F14C01089A62
:10BA70004B46304600F0FBFD02306080E3E770B5D6
:10BA80000E461546FFF7A4FA044638B10C2300F819
:10BA90004A3B2A46314618F038FD6580204670BD85
:10BAA000F8B50F4616461D46FFF792FA044668B1F0
:10BAB0002D01282345F00305037080F84A503246D3
:10BAC00039464B30013618F020FD66802046F8BD1F
:10BAD0002DE9F0470B78FF2B05460C4690464AD0DF
:10BAE00003689B6C984704F14A09064604F10A0A68
:10BAF000E6B9A27849462846FFF7C1FF0746002865
:10BB000039D0227904F10A010A3000F050FC3B7868
:10BB1000B88023F0030343F002033B7032464346F0
:10BB200039462846BDE8F047FFF708BD2B68214697
:10BB30005B6C2846984700F59670A278804433469F
:10BB400049462846FFF7ACFF074688B1227951469F
:10BB50000A3000F02CFC3B78B88023F0030343F05C
:10BB600002033B700022434639462846FFF7E6FCB5
:10BB7000013EF6B2BCE7BDE8F08770B591F84A60C7
:10BB800006F00F03032BC2B005460C4634D14B8898
:10BB9000042B31D901A800F0E6FB237822798DF837
:10BBA000043004F10A010DF10E0000F000FC62887F
:10BBB000ADF80800013A92B204F14B010DF14E00CC
:10BBC000ADF8062018F0A1FC686E036801A91B6897
:10BBD000984788B9686E036801A95B68984701A90E
:10BBE0002846FFF711FE36094FF4967206FB022233
:10BBF00001A92846FFF76CFF002042B070BDB82AAB
:10BC000070B50E46154603D8FFF7E2F9044610B9A1
:10BC10000024204670BD2C2300F84A3B2A463146BA
:10BC200018F073FC6580F4E72DE9F0410D781746B4
:10BC3000C5F38302092A06460C4620D0013BDAB23E
:10BC4000022A1CD825F0030545F001050D70406E51
:10BC50009B018B8003685B6898472378C3F3830359
:10BC6000082B0AD0042B14BF012203223B46214695
:10BC70003046BDE8F041FFF761BC0222F6E7BDE8BF
:10BC8000F0812DE9F0411F460B789DF818500646CB
:10BC9000C3F3830009280C4622D0013DE8B20228F4
:10BCA0001ED823F003030B701388706ECB8053886B
:10BCB0000B810368AD015B688D8098472278C2F3E1
:10BCC0008302082A0AD0042A14BF012203223B4619
:10BCD00021463046BDE8F041FFF730BC0222F6E7CE
:10BCE000BDE8F0812DE9F0410C46069F257825F04E
:10BCF000030545F002052570C5F38305092D0646A9
:10BD00001146984618D160884A301A46204418F0E7
:10BD1000FCFB6388434463800023A3800525706E89
:10BD2000036821465B6898473B462A4621463046D1
:10BD3000BDE8F041FFF702BC1A4604F10A0000F02A
:10BD400036FB2578A080C5F38305A5F108035D4285
:10BD50005D41E4E72DE9F04F0A7802F00303023B6E
:10BD6000012BF1B005460C466AD8C2F38303092BB8
:10BD70008E8859D13F2E1AD891F852E04F88D1F8C9
:10BD80004A20D1F84E300EF0030C093F06FA0CF6AB
:10BD9000FFB21FFA86F847450BD80A3405680397A7
:10BDA000CDE900E401F153060296AC6DA0470020F6
:10BDB00037E05336012200F1680102FA0CF2A019B3
:10BDC00018F039FA0028F2D12B682146DB6B28469F
:10BDD00098470028EBD0686E036821461B68984797
:10BDE0000028E4D1686E036821465B68984794F99F
:10BDF0000201F4F763FF4FF07A51F4F7B3FF4FF00D
:10BE00008141F4F7AFFFF5F789F9A3885A1C234461
:10BE1000A28098722B6821465B6C2846984740F0B8
:10BE2000C06071B0BDE8F08F0B2B06F03F063DD12E
:10BE300091F94A30002B33DB002E43D1930706D40F
:10BE40002B6821469B6B284698470028AFD1237862
:10BE5000C3F383020F2AAAD801A151F822F000BF30
:10BE6000A5BF0008A5BF0008A5BF000865BF000862
:10BE7000D3C100084FC100084FC10008CBC0000863
:10BE8000A5BF0008AFBD0008B9C20008AFBD0008DB
:10BE9000AFBD0008AFBD0008AFBD000889C20008F3
:10BEA000002E84D10368DB6E984780E7002EC5D052
:10BEB000032B07D14B88032B04D90368D1F84A2000
:10BEC000DB6F9847A28892090132D2B205F168016E
:10BED00004F10A0018F0AFF900287FF468AF2B686E
:10BEE0002146DB6B2846984700283FF460AF237853
:10BEF000C3F383030A2B06D12146284671B0BDE85F
:10BF0000F04FFFF73ABE686E0268032B12682146B5
:10BF100013D19047064600287FF449AF686E036846
:10BF200021465B68984721462846FFF76DFC32465C
:10BF300021462846FFF7CCFD39E7904700287FF4DB
:10BF400036AF686E036821465B68984721462846ED
:10BF5000FFF75AFC2B6821465B6C2846984740F057
:10BF600080705EE76388D4F84A60032B7FF61FAFCA
:10BF7000686E036821461B68984700287FF417AF56
:10BF8000686E036821465B6898472B683246DB6F12
:10BF90002146284698472146284671B0BDE8F04F13
:10BFA000FFF753BC94F84B308DF81830638894F841
:10BFB0004A60042B7FF6FBAE686E036821461B685F
:10BFC0009847814600287FF4F2AE686E03682146E8
:10BFD0005B68984795F86830B34264D12B6806A92E
:10BFE000DB6C2846984704F14C0806460EAF0DF16D
:10BFF000BC0AB14557DA2B684A461B6D39462846BC
:10C00000984763884246023B5146384600F053FB4E
:10C01000B0F1000B56DD2278C2F38302082A47D123
:10C020009AF80080404600F0A3F900283BD04FEA80
:10C03000981308F03F0603FB0666B21CABEB020B3D
:10C04000564452445FFA8BF12B6804910392727844
:10C0500002F00F02CDE901820DF1BD060096D3F882
:10C060005CA04A463B4621462846D047C8B12378C3
:10C0700013F0020315D1CDE9023301932379009324
:10C0800006A904F10A033A462846FFF75EFC01467A
:10C0900038B14FF4FA730093324643462846FFF70F
:10C0A00021FEFF23237021462846FFF7CEFBB8E68A
:10C0B0002B680097CDE901AB21465E6D28464B46C3
:10C0C000B047EEE709F1010993E7638894F84A6005
:10C0D000232B7FF66CAE686E036821461B68984779
:10C0E00000287FF464AE686E036821465B68984759
:10C0F00095F86830B3427FF44EAF04F14B0606AAC0
:10C1000004F16B0730687168134603C30836BE42FA
:10C110001A46F7D106AA0EA905F16800FFF737FB0A
:10C1200063882FAF213B324639460EA800F0C3FA90
:10C1300000287FF730AF2B68CDE900700EAA5E6E45
:10C14000214606AB2846B047FF23237023E794F827
:10C150004A308DF818306388032B7FF628AE686E5E
:10C16000036821461B689847064600287FF41FAEE7
:10C17000686E036821465B6898472B680EAA5F6F5C
:10C1800006A904232846B84704F14B0A80460DF15E
:10C1900039090DF1BC0B464585DA63884846013BF9
:10C1A0005246594600F087FA002809F121090EDDB0
:10C1B0002B682278CDE900B006EB46169F6F0EABD8
:10C1C0003344C2F3830221462846B8476BE7013661
:10C1D000E1E70EA8FFF7D9F90EAE04F14A0304F126
:10C1E0006A0718685968324603C20833BB421646CC
:10C1F000F7D16388D4F86A90632B7FF6D8AD2022FC
:10C200000EA905F1680018F016F800283FF4CFAD2C
:10C21000686E036821461B68984700287FF4C7AD05
:10C22000686E036821465B680EAF98470FCF2FAE4C
:10C230000FC6B4F8028097E80F00A8F16408B8F1BF
:10C24000200FA8BF4FF0200804F1AE0A86E80F00C7
:10C250004246514638A8CDF8DC9018F056F908F15E
:10C2600024032FAA04F16E010EA8FFF796F9002807
:10C270003FF49DAD2B68CDE900A80EAA1E6E2146A5
:10C280004B462846B0470EE703F00303023B012B61
:10C290003FF68DAD686E036821461B6898470028FD
:10C2A0007FF485AD686E036821465B6898472B680C
:10C2B00021461B6F2846F7E56288022A7FF677AD94
:10C2C00094F84A3003F00F03032B7FF470AD042A77
:10C2D0007FF66DAD2FA800F046F8237822798DF80F
:10C2E000BC3004F10A010DF1C60000F060F862886C
:10C2F000ADF8C000013A92B204F14B010DF5837024
:10C30000ADF8BE2018F001F9686E03682FA91B680C
:10C31000984700287FF44BAD686E03682FA95B68CF
:10C3200098472B68DDF80621DB6F2FA92846984730
:10C330003DE500BF2DE9F0410D7825F0030545F0FE
:10C3400002050D700646406E0368002517460C4630
:10C350008D805B6898473B462A4621463046BDE8BB
:10C36000F041FFF7EBB800220270828042807047F4
:10C3700000F03F038009032800F1010206D013FBFF
:10C3800002F04028CCBF00200120704700207047F9
:10C3900010B5930902F03F0403FB0444402C04DC75
:10C3A000224618F0B2F8204610BD0024FBE710B575
:10C3B0001446FFF7EDFF204610BD83889A0903F06D
:10C3C0003F0302FB033342880078DBB2023310F0F4
:10C3D0000300134405D0C21E50425041800018444F
:10C3E00070470420FBE730B50446A1B002A80D4613
:10C3F0000AF028FA23780122C3F383030DF1070121
:10C4000002A88DF807300AF005FB9DF80730092BCC
:10C4100004D10222211D02A80AF0FCFA628804F16C
:10C420004A0102A80AF0F6FA08220DEB020029469A
:10C430000AF022FB02A80AF0EBF921B030BDA0F10E
:10C440004103052B02D83738C0B27047A0F1610311
:10C45000052B01D85738F7E73038C0B20A2828BF73
:10C460000020704737B50368144604220D461B6848
:10C470000DEB020198470198621BB0FBF2F302FB3F
:10C480001300284403B030BDF0B50B4D03468E18A1
:10C49000B14203F1020303D1002300F81230F0BDD2
:10C4A00011F8014B270904F00F04EF5D2C5D03F830
:10C4B000027C03F8014CEBE7C87302082DE9F04158
:10C4C000DFF8308005460C468F18BC4201D1BDE82C
:10C4D000F08114F8016B330906F00F0618F8031009
:10C4E000284613F001FC18F80610284613F0FCFB50
:10C4F000EBE700BFC8730208F8B5064610460D46C4
:10C500001446F4F7C5FEB0EB450F17D1224631466D
:10C510008B1BAB4202F1020201DB0120F8BD12F8D5
:10C52000020C12F8017CFFF78AFF04463846FFF739
:10C5300086FF40EA041001F8010BE9E70020EDE76F
:10C54000F0B504460020074625780DB1904208DB7F
:10C55000214614F8012B1AB19A42F9D100230B702D
:10C56000F0BD41F8204025462E782C4601351EB1FD
:10C570009E42F9D127702C460130E5E7F0B59FB017
:10C580001F461646044668460D460AF05BF93A46D1
:10C59000314668460AF03EFADDE9241268460AF0A0
:10C5A00039FA2A46214668460AF066FA68460AF0D1
:10C5B0002FF91FB0F0BD2DE9F041B0B0064601A83B
:10C5C00015460C461F4609F007FB3146102201A80C
:10C5D00009F0B2FA2E46A6EB0508B84506DB01A81D
:10C5E00009F090FA404630B0BDE8F081324621466D
:10C5F00001A809F0E1FC10341036ECE72DE9F04316
:10C60000B5B0064605A81C460F46154609F0E4FAE3
:10C610003146102205A809F08FFA07EB04092E19FC
:10C620000F2CA9EB0405A6EB040819DC002C0FDD88
:10C630001022002101A817F028FE2246414601A839
:10C6400017F063FF294601AA05A809F0A1FB1035E0
:10C6500005A809F057FAED1B284635B0BDE8F08370
:10C660004246294605A809F093FB103CD8E7F0B5EF
:10C670008F1CA1B00E4639460546FFF7BFFF0446A2
:10C6800002A80AF0DFF8294602A820220AF041FA9F
:10C690002246394602A80AF0BDF90223009320225F
:10C6A0003346294602A80AF04CFA02A80AF0B0F86C
:10C6B000A01C21B0F0BD2DE9F043022BA3B005462C
:10C6C0000F4616461C4603DC002023B0BDE8F0836D
:10C6D00004A80AF0B7F806F102082022294604A8A7
:10C6E000023C0AF016FA4FF002092246414604A81D
:10C6F0000AF090F92022294603AB04A8CDF8009057
:10C700000AF01FFA04A80AF083F84A46314603A843
:10C7100017F091FD0028D7D12346424639462846D6
:10C72000FFF749FFD1E7F0B5044620B30020235CB2
:10C73000261803B31A061FD503F13E02D2B21D2AF2
:10C740001CD903F12002D2B20F2A19D903F1100229
:10C75000D2B2042A0FD8042200EB020C8C450AD86E
:10C76000B6460127BA420DD1032A1BD1E02B7278BD
:10C7700012D19F2A14D8F0BD0122EDE70222EBE787
:10C780000322E9E71EF8015F002DF4D005F0C00593
:10C79000802DF0D10137E5E7ED2B01D19F2AEAD8B2
:10C7A0006046C4E7042AFBD1F02B727801D18F2AAE
:10C7B000E0E7F42BF4D18F2AF1E7F8B503780B709A
:10C7C000427806460C468AB343F010030B70836828
:10C7D000C1F80130C368C1F805300925338A33B187
:10C7E000237843F020032370338A63530235738A1E
:10C7F00033B1237843F040032370738A63530235C7
:10C80000706888B103787BB1C5F12001FFF78BFF19
:10C81000074648B1237863F07F03237002467168AE
:10C82000601917F072FE3D44E8B2F8BD0125D5E766
:10C8300038B50023837004460878E362C4E90933FD
:10C840006370C30641BFD1F801306362D1F805308F
:10C85000A3624CBF09230123850642BFCD5AA5859B
:10C860000233450642BFCD5AE58502339A42207015
:10C870000DDB000609D5D51A07D02A461944A01C9D
:10C8800017F043FE62190023937001236370204662
:10C8900038BD000001480BF039B800BFEC3900206A
:10C8A0002DE9F047074607F5805800243960ADF5BB
:10C8B000027D0846C8F804443E4991460BF057F9FA
:10C8C00000284DD03AA83B4A396823460BF045F979
:10C8D0003AA80BF0AAFA002842D04FF0A00A12A8FA
:10C8E000FEF753FEA022002112A817F0CEFC202252
:10C8F00002A93AA80BF017FA202804462DD10122EC
:10C900001AA93AA80BF00FFA0128054625D10422EE
:10C9100035A93AA80BF007FA04281ED1022201A972
:10C920003AA80BF000FA022817D12A460DF1690146
:10C930003AA80BF0F8F901280FD140220DF16A0155
:10C940003AA80BF0F0F9402807D122460DF1AA01D0
:10C950003AA80BF0E8F9202806D03AA80BF01DFA07
:10C960000DF5027DBDE8F08702AD0FCD0AAC0FC416
:10C9700095E80F0084E80F000AAE0FCE12AD0FC588
:10C9800094E80F0085E80F00484602AA0DF1AA01BD
:10C99000FEF7FDFED8F804041F28DEDC431C0AFB6A
:10C9A0000070C8F80434A02212A9043017F0ADFDBD
:10C9B00095E700BFD97302082DE9F84300F58053CD
:10C9C0000E46D3F804941746041D0025A94504DC3F
:10C9D0004FF000084046BDE8F88321463A4630460D
:10C9E00017F029FCA046A0340028F3D00135EDE76C
:10C9F00000F580532DE9F74F00F59B54D3F80474EC
:10CA00000D46064690460434011D4FF000094FF0D4
:10CA1000FF3A4F4523DC202F06D07A1CC3F80424AC
:10CA2000A02303FB0766341DA0220021204617F037
:10CA30002CFC2B4684F82080254603F1200618683C
:10CA400059682A4603C20833B3421546F7D1FF237B
:10CA500084F82130A346584603B0BDE8F08F202269
:10CA6000284601938B46009117F0E5FB0028F2D091
:10CA70009BF82020019B02F00302032A594605D0AF
:10CA8000DBF8882052453CBF5C46924609F101091B
:10CA9000A031BEE72DE9F04188B015469DF83880F9
:10CAA00018F0030F04460F461A4621D12946FFF716
:10CAB00083FFF8B104F58053A021D3F804546A1E13
:10CAC000C3F80424231DC31A194A581150432A1AC3
:10CAD0004A43A03A03F1A40104338542D8BF00229F
:10CAE0002144E01817F0B7FB012008B0BDE8F08141
:10CAF0001F2B01DC0020F8E76A462B4605F1200ECB
:10CB0000944618685968164603C60833734532467A
:10CB1000F7D1614600222046FFF76AFF2A4680F8D7
:10CB2000208000F162013846FEF731FEDCE700BFED
:10CB3000CDCCCCCC2DE9F0430C46CBB00160054602
:10CB40003249204617460BF01EF802A82F4A01234F
:10CB500021460BF002F802A80BF067F9F0B10026AD
:10CB600005F16604ADF8046005F58055D5F8043488
:10CB7000B34210DD14F8423C13B90136A034F5E796
:10CB8000A4F162086FB94146202202A80BF00FF809
:10CB9000202880460AD002A80BF0FFF84BB0BDE871
:10CBA000F0834046B8470028EDD1E6E70122A4F122
:10CBB000420102A80AF0FBFF01288146EBD10422C2
:10CBC00004F12A0102A80AF0F2FF0428E3D10222AC
:10CBD00001A902A80AF0EBFF0228DCD14A46A4F121
:10CBE000410102A80AF0E3FF0128D4D14022A4F1B8
:10CBF000400102A80AF0DBFF4028CCD14246214682
:10CC000002A80AF0D4FF2028B7D0C4E7D9730208DD
:10CC100010B5421E0A24002012F8013F303BD9B261
:10CC2000092900D910BD04FB0030F5E710B5044612
:10CC3000F4F72EFB00212318A34203D913F8012C8B
:10CC4000202A00D010BD03F8011DF5E770B5CAB069
:10CC50000446002302A80AF080FF02A80BF0E5F8C2
:10CC6000002800F03A82616804220C3102A80BF01F
:10CC70005AF861682022103102A80BF054F80422FF
:10CC8000694602A80BF04FF86168082230310DEBBD
:10CC900002000BF048F86168082238310DEB020001
:10CCA0000BF041F861681022403102A80BF03BF80C
:10CCB00061680422503102A80BF035F86168012246
:10CCC000543102A80BF02FF861680122553102A8F7
:10CCD0000BF029F861680122563102A80BF023F805
:10CCE0000122694602A80BF01EF86168042258313F
:10CCF00002A80BF018F8616804225C3102A80BF05E
:10CD000012F861681022603102A80BF00CF861681B
:10CD10000422703102A80BF006F80422694602A82A
:10CD20000BF001F861680122783102A80AF0FBFFDC
:10CD300061680122793102A80AF0F5FF61680122D9
:10CD40007A3102A80AF0EFFF616801227B3102A864
:10CD50000AF0E9FF616804227C3102A80AF0E3FFCF
:10CD600061680122873102A80AF0DDFF61680122B3
:10CD700001F2331102A80AF0D6FF6168012201F521
:10CD80009A7102A80AF0CFFF0122694602A80AF0B0
:10CD9000CAFF61680122803102A80AF0C4FF6168FD
:10CDA0000122573102A80AF0BEFF616801228631D4
:10CDB00002A80AF0B8FF61680122883102A80AF0CF
:10CDC000B2FF616802228A3102A80AF0ACFF6168F2
:10CDD00001228C3102A80AF0A6FF6168042290317A
:10CDE00002A80AF0A0FF61680122943102A80AF0AB
:10CDF0009AFF61681022953102A80AF094FF6168D9
:10CE00000122A53102A80AF08EFF0322694602A87A
:10CE10000AF089FF61680122A63102A80AF083FFA7
:10CE200061680422A83102A80AF07DFF616801222E
:10CE3000AC3102A80AF077FF61680422B03102A881
:10CE40000AF071FF61680422B43102A80AF06BFF96
:10CE500061687822B83102A80AF065FF6168012292
:10CE600001F5987102A80AF05EFF61680122813124
:10CE700002A80AF058FF61680122823102A80AF074
:10CE800052FF6168012201F2311102A80AF04BFF42
:10CE90006168012201F2351102A80AF044FF6168BD
:10CEA0000122833102A80AF03EFF61680122843129
:10CEB00002A80AF038FF61680122853102A80AF051
:10CEC00032FF6568AE6D00213046F4F7E9F80028BE
:10CED00040F0058189493046F4F700F900B1874EEA
:10CEE000AE65EE6D00213046F4F7DAF8002840F028
:10CEF000F8804FF080413046F4F7F0F808B14FF079
:10CF00008046EE652E6F00213046F4F7C9F8002800
:10CF100040F0E9804FF080413046F4F7DFF808B187
:10CF20004FF080462E67EE6800213046F4F7B8F8DF
:10CF3000002840F0DA8072493046F4F7CFF800B1AB
:10CF40006F4EEE602E6D6F493046F4F7A9F8002859
:10CF500040F0CD806C493046F4F7C0F800B16A4E1D
:10CF60002E65EE6F69493046F4F79AF8002840F0D4
:10CF7000C08067493046F4F7B1F800B1644E95F8C7
:10CF80007830EE670C2B28BF0C23052B38BF052308
:10CF900085F87830626892F87930082B28BF08232A
:10CFA000052B38BF052382F87930626892F9543036
:10CFB0001E2BA8BF1E236FF008018B42B8BF0B4683
:10CFC00082F85430626892F87B30012B28BF01232D
:10CFD00082F87B306668D6F8B45000212846F4F712
:10CFE0005FF8002840F087804A492846F4F776F831
:10CFF00000B1484D96F83331C6F8B450022B28BF23
:10D00000022386F83331626892F88830012B28BFFA
:10D01000012382F888306368B3F88A2042F21071E5
:10D020008A4228BF0A46A3F88A2093F88C20012A56
:10D0300028BF012283F88C206268D2F89030B3F5C3
:10D04000E13F28BF4FF4E133B3F5165F38BF4FF42B
:10D050001653C2F8903092F894300E2B28BF0E234E
:10D0600082F89430626892F8A530012B28BF012322
:10D0700082F8A530626892F8A630012B28BF012300
:10D0800082F8A630626892F8AC30022B28BF0223E7
:10D0900082F8AC30626892F83031012B28BF01234E
:10D0A00082F83031626892F83131012B28BF0123B8
:10D0B00082F83131626892F83231012B28BF0123A6
:10D0C00082F83231626892F83531012B28BF012392
:10D0D00082F8353102A80AF060FE4AB070BD002621
:10D0E000FEE600260DE700261CE7002629E7054E90
:10D0F00036E7064E43E700257CE700BF0000A0416D
:10D10000000010410000164300401C459A99F94068
:10D110000000FA430000204130B50C46C9B00D496B
:10D12000054620460AF02FFD21460A4A012368469B
:10D130000AF013FD68460AF078FE044638B16868C4
:10D14000694601F057FE044668460AF026FE20466E
:10D1500049B030BDE573020830B50C46C9B005468C
:10D16000144920460AF003FD90B16846114A002395
:10D1700021460AF0F2FC68460AF057FE30B16868B2
:10D18000694601F030FF68460AF007FE49B030BD3D
:10D19000094920460AF0EBFC0028F7D02146284632
:10D1A000054AFFF753FD2146284649B0BDE8304007
:10D1B000FFF7B2BFE5730208F1730208426892F804
:10D1C00056305B003B2BDCBF002382F85630806872
:10D1D00003681B68184700002DE9F04314464268B5
:10D1E00092F8AC3087B002F1100563B98DF80410E5
:10D1F0008DF805300295214601A80593FFF7DDFA69
:10D2000007B0BDE8F083012B1FD10269D2E9028982
:10D21000D2E904678DF804108DF80530404610A35C
:10D22000D3E9002349460295F3F746F9F3F7F4FBF7
:10D230000BA3D3E90023039039463046F3F73CF9BA
:10D24000F3F7EAFB00230490D5E7D2E90C89D2E991
:10D250000E6701238DF80410DEE700BFAFF30080F6
:10D260000000000080842E412DE9F043171DA9B075
:10D27000044689461646AD490A2238461D4616F030
:10D28000DAFF00284AD106F10E0015F0A6FDF3F7EB
:10D290000BFC4FF07E510646F3F702FF20B9A4497C
:10D2A0003046F3F71BFF30B1A249284629B0BDE84C
:10D2B000F04317F022B931469D486768F3F706FE40
:10D2C0004FF07E51F3F744FCF8602046FFF776FFFD
:10D2D00063684FF07E51D868F3F73CFC01469448F0
:10D2E000F3F7F4FD0646F3F719FF0446F3F7E6FCFF
:10D2F00001463046F3F72CFC8F49F3F733FD4FF02E
:10D300007C51F3F727FCF3F709FF8C4903462246CB
:10D31000284629B0BDE8F04316F0CCBE8849032268
:10D32000384616F088FF50B9F01D15F056FDF3F79A
:10D33000BBFB6668F0602046FFF740FF62E1814971
:10D340000B22384616F077FF38B906F10F0015F0BA
:10D3500047FD636883F88600EDE77B490422384681
:10D3600016F069FF60B97949022206F1080016F04B
:10D3700062FF6368B0FA80F0400983F83501DAE7AC
:10D3800073491322384616F056FFC0B906F117004C
:10D3900015F026FD00286368B8BF0330801083F8BD
:10D3A00087002046FFF70AFF63686A4993F88720E1
:10D3B0009200284629B0BDE8F04316F07BBE6649CE
:10D3C0000B22384616F037FF38B906F10F0015F07A
:10D3D00007FD636883F87B00ADE76049102238469B
:10D3E00016F029FF60B95949022206F1140016F01F
:10D3F00022FF6368B0FA80F0400983F87A009AE768
:10D4000057491622384616F016FF90B906F11A0051
:10D41000FFF7FEFB431E012B01D9A82801DD51496E
:10D4200043E7636883F85700A0680368DB6998479F
:10D4300081E74D491022384616F0FDFEA8B906F1E5
:10D440001400FFF7E5FB431E3A2B01D9F02802DD5B
:10D4500046493C22ADE7636800EBD070401083F88A
:10D460005600A06803689B69E1E741490F223846EE
:10D4700016F0E1FE38B96068102206F11301603041
:10D4800002F07CFD57E73B490822384616F0D3FEF0
:10D4900038BB06F10C0240216846FFF72DF8F0B1C9
:10D4A0006846FEF7A3F8D0B110A8FEF77DF8402239
:10D4B0000DEB02006946FEF735F9A068036810A974
:10D4C0009B6C98472C49284617F017F8202210A982
:10D4D00005F12100FEF7D8FF29B0BDE8F083274908
:10D4E000E3E627490522384616F0A5FE00284DD16F
:10D4F000244906F1080212F8013F2BB96068202286
:10D5000006F109011030BBE73A2B09D8292BF2D9D3
:10D510002A3BDBB221FA03F3DB07ECD51A49C4E658
:10D520003F2BFBD05B3B022BE5D8F7E729740208C1
:10D530000000C842347402080000204153740208FD
:10D540006074020864740208707402084E7F020856
:10D550007574020889740208A5740208B17402087F
:10D56000C2740208D9740208C8740208FE74020862
:10D5700026750208367502083F75020861750208B3
:10D580007075020805000100707802089A490722A8
:10D59000384616F050FEC0B99849032206F10B0038
:10D5A00016F049FE6368B0FA80F0400983F8550030
:10D5B0002046FFF703FE6368914A93F85510914B9C
:10D5C00000290CBF114619466FE68F490D223846D7
:10D5D00016F031FEC0B98D49022206F1110016F095
:10D5E0002AFE6368B0FA80F6760983F83061204637
:10D5F000FFF7E4FDA068036831469B6E984700285A
:10D6000000F0CF82824950E682491122384616F056
:10D6100012FE002836D1E06803689B6C984700280A
:10D6200000F0BF82153679490222304616F003FE1B
:10D6300080B9E068036801215B6C984740B163687A
:10D64000012283F831212046FFF7B8FD72492CE60C
:10D6500072492AE630466949032216F0ECFD064677
:10D6600070B9E068036831465B6C98470028EFD0DA
:10D670006368204683F83161FFF7A0FD684914E62E
:10D68000684912E668491122384616F0D4FD002890
:10D6900035D1E06803685B6D9847002800F081820F
:10D6A00015365A490222304616F0C5FD80B9E068A9
:10D6B000036801211B6D984740B16368012283F81C
:10D6C00032212046FFF77AFD5849EEE55849ECE54E
:10D6D0004A490322304616F0AEFD01460028CFD15C
:10D6E000E06803681B6D98470028EFD0636800224C
:10D6F00083F832212046FFF761FD4E49D5E54E49BA
:10D700000622384616F097FD8046002857D104F1CE
:10D710001C0306F10A0118461E4616F0EEFE2C23E5
:10D72000042210A93046FEF70BFF071E45DD1098B6
:10D73000414616F0E9FA012F81463ED04146119844
:10D7400016F0E2FA022F804637D0129815F048FB07
:10D75000032F06462FD0139815F042FBC7B2374966
:10D760004846F3F7B1FC40B335494846F3F7A2FC0D
:10D7700018B3F6B2731F072B1FD87B1F032B1CD8BF
:10D7800030494046F3F7A0FCB8B12F494046F3F7C3
:10D7900091FC90B1636883F87860636883F879706E
:10D7A0006368A068C3F85090C3F87C8003681B6866
:10D7B0009847264979E50027D1E7254975E52549A8
:10D7C0000422384616F037FD38B906F108006768BC
:10D7D00015F003FBC7E90C01ADE51F4904223846EB
:10D7E00016F029FD002839D106F10800676815F008
:10D7F000F4FAC7E90E019EE576750208E37902089E
:10D8000013740208FC7302087E7502084E7F02083A
:10D810000A6D02089F750208B1750208CA750208F0
:10D82000F27502080C7602082B7602083D76020893
:10D83000567602087E760208007E02080000164333
:10D8400000401C450000E0400000FA4398760208C2
:10D85000AD760208C9760208CE7602089F490822F2
:10D86000384616F0E8FCA0B906F10C0015F0B5FA40
:10D87000F3F71AF900210646F3F726FC38B1984968
:10D880003046F3F717FC10B163689E6553E5954980
:10D890000BE595490822384616F0CDFCA8B906F1EB
:10D8A0000C0015F09AFAF3F7FFF800210646F3F79B
:10D8B0000BFC40B14FF080413046F3F7FBFB10B159
:10D8C0006368DE6537E58949EFE489491322384604
:10D8D00016F0B1FC60B906F1170015F081FAC0B27C
:10D8E000402803D8636883F8810024E58149DCE49B
:10D8F00081491122384616F09EFC50B906F11500F8
:10D9000015F06EFAC0B24028F0D8636883F8820040
:10D9100011E57A491222384616F08DFC50B906F10D
:10D92000160015F05DFAC0B24028DFD8636883F8AE
:10D93000830000E572491722384616F07CFC50B986
:10D9400006F11B0015F04CFAC0B24028CED863682F
:10D9500083F88400EFE46B491322384616F06BFC21
:10D9600050B906F1160015F03BFAC0B24028BDD8F8
:10D97000636883F88500DEE463490A22384616F0BE
:10D980005AFC50B906F10E0015F02AFAC0B2402830
:10D99000ACD8636883F88000CDE45C490F22384638
:10D9A00016F049FCB0B906F1130015F016FAF3F7BA
:10D9B0007BF800210646F3F787FB002883D04FF061
:10D9C00080413046F3F776FB00283FF47CAF636874
:10D9D0001E67B0E44E490B22384616F02CFC98B96D
:10D9E00063680E36B83316F8011F21B16268B83289
:10D9F0009A1A762A02D900221A709CE47C2908BF60
:10DA00000A2103F8011BEEE742490F22384616F0BF
:10DA100012FC60B906F1130015F0E2F9C0B2022859
:10DA200003D8636883F8330185E43B493DE43B490F
:10DA30000C22384616F0FFFB18BB1036384903227B
:10DA4000304616F0F8FBA0B136490722304616F0F2
:10DA5000F2FB68B134490822304616F0ECFB60B1A5
:10DA600032490622304616F0E6FB40B130491CE44C
:10DA70000120636883F834015DE40220F9E70320A4
:10DA8000F7E72C490322384616F0D5FB80B9F01D84
:10DA900015F0A6F9636883F854002046FFF78EFB63
:10DAA000D4E90120036892F95410DB6A9847A9E58C
:10DAB000B9F1000F42D120490522384616F0BBFBD0
:10DAC00000283BD106F1090015F087F9F2F7ECFFC9
:10DAD000666830652046FFF771FB6AE6D376020878
:10DAE0000000A041DC76020888770208F076020880
:10DAF00003770208177702082577020837770208AC
:10DB00004A7702086277020876770208817702086E
:10DB1000917702089D770208AD770208C677020860
:10DB2000E3790208E9790208F3790208FE7902082C
:10DB3000D3770208057802080978020821490F22E4
:10DB4000384616F078FB78BB06F1130015F045F95E
:10DB5000F2F7AAFF63680146C3F8B400E0680368FF
:10DB60009B689847C8B12046FFF728FB6368D3F845
:10DB7000B44000212046F3F789FA10B11249FFF7AB
:10DB800094BB2046F2F740FC0B461049024628465B
:10DB900029B0BDE8F04316F08DBA63680022C3F8DF
:10DBA000B4200B49FFF781BB0A49284616F0A5FCB3
:10DBB0008F22394605F1100029B0BDE8F04302F08C
:10DBC000DDB900BF0F7802081F7802084378020809
:10DBD0008C7502085F7802082DE9F043161D97B096
:10DBE000054688461746A249092230461C4616F0CB
:10DBF00022FB28BB6B684FF07E51D868F2F7AAFF72
:10DC000001469C48F3F762F90646F3F787FA0546A2
:10DC1000F3F754F801463046F2F79AFF9649F3F7C6
:10DC2000A1F84FF07C51F2F795FFF3F777FA93499B
:10DC300003462A46204617B0BDE8F04316F03ABA2C
:10DC40008F490222304616F0F6FA28B96B68D86878
:10DC500002F0AEF9024618E08A490A22304616F070
:10DC6000EAFA20B96B6893F8862087490EE0874965
:10DC70000322304616F0DFFA70B96B6893F835115D
:10DC8000834A844B002918BF1A468349204617B09F
:10DC9000BDE8F04316F00EBA80491222304616F065
:10DCA000CAFA20B96B6893F887209200DDE77C49B7
:10DCB0000A22304616F0BFFA18B96B6893F87B2039
:10DCC000D3E778490F22304616F0B5FA18B96B68D9
:10DCD00093F87A10D4E774491522304616F0ABFA5F
:10DCE00018B96B6893F85720BFE770490F22304688
:10DCF00016F0A1FA20B96B6893F856205200B4E7E9
:10DD00006B490E22304616F096FA10B96A686032F6
:10DD1000BBE7B8F1000F1BD166490722304616F069
:10DD20008AFAA8B9A86803685B6C9847402206A9DC
:10DD3000FDF7D4FC1C35024606A92846FEF7A4FBD5
:10DD400055492A46204616F0B5F917B0BDE8F083CC
:10DD500059490422304616F06EFA10B96A6810323A
:10DD600093E756490622304616F065FA28B96B68E3
:10DD7000484A93F85510464B84E7514903223046F0
:10DD800016F059FA28B96B68D3E90C01F2F78CFE4A
:10DD90005EE74C490322304616F04DFA18B96B681D
:10DDA000D3E90E01F2E748490C22304616F043FA57
:10DDB00018B96B6893F8301162E744491022304675
:10DDC00016F039FAA8B9E86803689B6C984730B92F
:10DDD0003F49204617B0BDE8F04316F08EBBE86817
:10DDE0000368DB6C98472A4A2A4B002818BF1A465A
:10DDF0004BE738491022304616F01DFA48B9E8685A
:10DE000003685B6D98470028E2D0E86803689B6D63
:10DE1000E8E731490522304616F00DFAE8B96B689B
:10DE2000186D02F0C5F8014602A816F066FB6B6893
:10DE3000D86F02F033F9014606A816F05EFB6B6856
:10DE4000264993F87920019293F87830009302AA3A
:10DE500006AB204616F02EF977E721490722304617
:10DE600016F0E9F900283DD16B68986DF0E600BF27
:10DE7000817802080000C842000020418B78020827
:10DE8000EB6A02089A780208A5780208C66A0208B6
:10DE9000E37902084E7F020895780208AA78020802
:10DEA000BD780208C8780208D8780208DE7802082F
:10DEB000EE780208FD7802083F7B0208956A0208A6
:10DEC000826A0208866A0208057902081279020845
:10DED0008C750208237902089C7F020834790208B5
:10DEE000EE6A020896490722304616F0A4F910B9E6
:10DEF0006B68D86DACE693491022304616F09BF95A
:10DF000018B96B6893F88220AFE68F491222304629
:10DF100016F091F918B96B6893F88120A5E68B4942
:10DF20001122304616F087F918B96B6893F88320F0
:10DF30009BE687491622304616F07DF918B96B68C2
:10DF400093F8842091E683491222304616F073F943
:10DF500018B96B6893F8852087E67F490922304617
:10DF600016F069F918B96B6893F880207DE67B4953
:10DF70000E22304616F05FF910B96B68186F67E62D
:10DF800077490A22304616F056F9B0B923463E22A8
:10DF900003F8022B202262706968B73111F8012F53
:10DFA00012B900221A70D0E6181B9E28F9DC0A2A42
:10DFB00008BF7C2203F8012BF0E76A490E223046A5
:10DFC00016F039F918B96B6893F833214DE66649B4
:10DFD0000B22304616F02FF970B96B6893F8343184
:10DFE0000BB96249F5E6012B01D16149F1E6022B3B
:10DFF0000CBF60496049ECE660490222304616F0E9
:10E000001AF938B9BB7913F0DF0F03D16B6893F9B4
:10E0100054202AE65A490422304616F00CF910B969
:10E020006B68186D14E657490A22304616F003F95A
:10E0300078B95549204616F060FAA86803685B6C09
:10E04000984720220146A01C17B0BDE8F043FEF718
:10E050001BBA4E490422304616F0EDF820B9A868E4
:10E060000368DB689847F5E549490B22304616F00E
:10E07000E2F808B9474A08E647490E22304616F04A
:10E08000DAF800283FF4A4AE44490E22304616F0D8
:10E09000D2F8B0B9E8680368DB6898470021054604
:10E0A000F2F7F4FF00287FF493AE2846F2F7ACF9BC
:10E0B0000B463B490246204617B0BDE8F04315F039
:10E0C000F9BF38490E22304616F0B5F808B936497E
:10E0D0007FE636490D22304616F0ADF808B93449CE
:10E0E00077E634491122304616F0A5F8B0B9EE684B
:10E0F00033683046D3E91937984701463046B84768
:10E10000ED682B680646D3E91B3728469847014639
:10E110002846B8472849034632468BE527490D2251
:10E12000304616F088F80028D9D025490822304614
:10E1300016F081F8074600285FD022493246A5E54F
:10E14000B379020842790208537902086679020815
:10E15000787902088F790208A2790208AC7902085E
:10E16000BB790208C6790208D5790208E17902086C
:10E17000E7790208F1790208FC790208E86A0208E6
:10E18000BB6A0208057A0208656F0208107A020865
:10E19000157A0208217A0208267A0208357A0208DE
:10E1A000447A02084B7A02085A7A0208687A02080E
:10E1B000767A02089C7A0208AE7A0208C87A0208C7
:10E1C000D67A0208FD7A02080F4ADFF84090DFF89D
:10E1D000408026463046494615F06CFF0137032F34
:10E1E000064406D06B683B44424693F83631002B18
:10E1F000F0D1B4427FF4A9AD04E06B6893F83631F6
:10E20000002BE1D10349E4E5CB850208DF7A02085F
:10E21000E47A0208E67A02082DE9F04F0023137031
:10E2200089B005460F4614460B461E460133327828
:10E23000202AFAD096490A22304616F04CF80028D7
:10E2400078D1B37A13F0DF0F74D106F10A031E46BA
:10E2500001333278202AFAD03046FEF7E7FC3378D3
:10E2600033B98C49204609B0BDE8F04F16F045B9E6
:10E270006B694FF0000903F28C483378202BB346CA
:10E2800006F10106F9D0002B4CD05B461A781E46E9
:10E29000013322B1202AF9D186F800901E46D5F824
:10E2A00014A05B461A4613F8017B6FB17C2F01D096
:10E2B0002C2FF7D182F800901F4613F8012B202A4B
:10E2C000FAD03846FEF7B2FC59461BF8013B202B2A
:10E2D000FAD00BB97049C5E71FB13B780BB96F494C
:10E2E000C0E7B8F8002003910023504601F058FA27
:10E2F0000399804640B96A4A0B46A021204609B0DE
:10E30000BDE8F04F15F0A2BE80F80490002FB4D005
:10E310003946504601F092FA80460028ADD1614A54
:10E320003B46EAE76869A022214609B0BDE8F04F04
:10E3300001F070BB38462023042204A9FEF700F93F
:10E340000128074607D16869A022214601F062FB37
:10E3500009B0BDE8F08F40F36481059E5249304614
:10E36000F2F78CFF20B9A86803685B6D9847EFE768
:10E370004E493046F2F782FF98B9D5E900060368A6
:10E380001B689847C6F8B0002846FEF717FFA86834
:10E3900003689B6D9847464A4649002808BF1146C6
:10E3A00060E7022F64D044493046F2F767FF60B956
:10E3B0000699686901F042FA28B1037923F0010354
:10E3C00003713C494EE73D494CE73D493046F2F781
:10E3D00055FF48B90699686901F030FA0028F2D073
:10E3E000037943F00103EBE736493046F2F746FF85
:10E3F00038BB0699686901F021FA06460028E2D088
:10E400004188686901F058FA3379721D70B101884A
:10E4100061B12D4913F0010F2C4B18BF0B4600932F
:10E420002B49431D204615F045FE91E7274913F07F
:10E43000010F2046244B08BF0B46264915F03AFE33
:10E4400086E725493046F2F719FF00284CD1069996
:10E45000686901F0F3F906460028B4D001466869FE
:10E4600001F045FA1D49721D204615F023FE6FE7A5
:10E4700019493046F2F702FF002872D1686901F0AD
:10E4800033FA10B1421D1649EEE7164AFBE700BF0A
:10E49000187B0208237B0208337B0208447B0208B6
:10E4A000557B02086A7B0208817B0208867B020892
:10E4B000047B02080A6D02088B7B0208927B02082B
:10E4C000A77B0208AD7B0208CB8502082011030858
:10E4D000B17B0208BD7B0208C47B0208C97B02082D
:10E4E000D97B0208167B02084F493046F2F7C6FE78
:10E4F000002845D1069F4D493846F2F7BFFE064633
:10E5000068696EB9314601F0FCF9A86803683146C4
:10E51000DB6D9847A86803689B6D98474449A1E65E
:10E52000394601F08BF9064638B90346024606998A
:10E53000686901F035F9064688B1002333716869CE
:10E54000314601F0DEF9A86803683146DB6D984773
:10E55000A86803689B6D98473649721D84E7364961
:10E5600080E631493046F2F789FE002859D16869C2
:10E5700001F0C1F910B1421D304975E72B4AFBE7A4
:10E580002F493046F2F77AFEB8B9032F686905D0F3
:10E59000079901F053F918B92A4963E600F28C4053
:10E5A000028806996869002301F0FAF808B926493B
:10E5B00058E600232549037154E625493046F2F711
:10E5C0005DFE78B90699686901F0BAF8014638B17C
:10E5D000686901F09AF900287FF4F3AE1D4941E61D
:10E5E0001D493FE61D493046F2F748FEC8B9069E70
:10E5F0001B493046F2F742FE38B11A493046F2F76D
:10E600003DFE08B118492DE60120009068690123FC
:10E61000A022214601F018FA00287FF499AE134990
:10E6200020E613491EE600BFE57B0208037C0208D2
:10E63000ED7B02080A7C0208237C02083B7C02086E
:10E64000757C0208507C0208657C0208797C02080F
:10E650008E7C0208957C0208A57C0208CB7E02080D
:10E66000B57C0208BD7C0208C47C02085C6B020811
:10E67000E47C02082DE9F04F14468DB0054688462B
:10E6800008227A4920461E4615F0D5FD28B1784962
:10E690000822204615F0CFFD30B9E86803681B6AF0
:10E6A0000DB0BDE8F04F184772490622204615F01C
:10E6B000C2FD18B9E8680368DB69F1E76E49092211
:10E6C000204615F0B8FD28B928686C4903685B68D6
:10E6D0009847EFE76A490E22204615F0ACFD80B955
:10E6E000A27B12F0DF020CD1A868036840F2DC5173
:10E6F0005B699847634930460DB0BDE8F04F15F0AF
:10E70000FCBE61490622204615F095FD40B9A86877
:10E71000036840F2DC515B69012298475B49EAE7F4
:10E720005B490A22204615F086FD30BB2868036845
:10E730001B68984780451ED9286803685B6808F104
:10E7400001019847286803681B689847014604A898
:10E7500009F092F89DF810309DF813204D4903F50B
:10E76000FA6302939DF8113001939DF812300093E3
:10E770009DF814302FE04849BDE74849092220465A
:10E7800015F059FD48B9E8686968036832461B6CA2
:10E790001031984710BB4249ADE742490522204657
:10E7A00015F049FDE8B9286803681B6898470146D9
:10E7B00004A809F061F89DF810309DF813203A493B
:10E7C00003F5FA6302939DF8113001939DF812301E
:10E7D00000939DF81430304615F06CFC0DB0BDE888
:10E7E000F08F32490522204615F025FD80B9601DC5
:10E7F000FEF70EFA0446286803681B6898478442AF
:10E8000004D92868036821465B689AE7284972E7BB
:10E8100028490922204615F00EFD38B9A86803687A
:10E820001B6B31460DB0BDE8F04F1847224910224E
:10E83000204615F000FD002844D110342046F2F7A0
:10E8400027FD402828BF402047102246394604A80B
:10E85000FDF752FE38B1A868036804A95B6B3A461D
:10E860009847164947E7164945E700BFF67C020876
:10E87000FF7C02080B7D0208087D0208EF934466C6
:10E88000127D0208217D02084C7902083A7D0208B7
:10E890004B7D0208567D02087F7D02089E7D02089E
:10E8A000A87D0208AE7D0208667D0208B47D0208DC
:10E8B000BA7D02084F6D0208DB7D02080A6D02086E
:10E8C000EC7D0208A2490A22204615F0B4FC074656
:10E8D00000286BD105F11C0304F10A0118461C46FF
:10E8E00015F00BFE2C23052204A92046FDF728FE77
:10E8F000B0F1000858DD0498394615F005FAB8F172
:10E90000010F834646D00598002115F0FDF9B8F1B6
:10E91000020F814643D0069814F062FAB8F1030F53
:10E920005FFA80FA3ED0079814F05AFAB8F1040F53
:10E93000C4B203D0089814F053FA074685495846E4
:10E94000F2F7C2FB80B384495846F2F7B3FB58B3E1
:10E95000AAF10503072B27D8631F032B24D87F496F
:10E960004846F2F7B1FBF8B17D494846F2F7A2FB01
:10E97000D0B1002F18DDA8680368CDE900474A46EA
:10E980001C6D59465346A04776493A46304615F025
:10E9900091FB23E70024A2464FF00009CEE70024B4
:10E9A000A246CBE70024C9E76F49A4E66F490922D4
:10E9B000204615F040FCB8B96868102204F109013E
:10E9C000403001F0DBFA2846FEF7F8FB6849304694
:10E9D00015F093FD69689122403106F10E000DB0EB
:10E9E000BDE8F04F01F0CABA62490B22204615F08B
:10E9F00022FC28B9A8680368DB6C98475E497AE670
:10EA00005E490422204615F016FC40B933462246E2
:10EA1000414628460DB0BDE8F04FFFF7DDB8584934
:10EA20000422204615F007FC40B9334622464146F1
:10EA300028460DB0BDE8F04FFEF716BCB8F1000F48
:10EA400014D150492046F2F719FC78B9A868036838
:10EA50001B6998474C4A4D4B4D49002818BF1A4630
:10EA600030460DB0BDE8F04F15F024BB49490322F4
:10EA7000204615F0E0FB88B9A86803685B689847F2
:10EA80000446A86803689B689847434903462246A2
:10EA900030460DB0BDE8F04F15F00CBB3F490522E4
:10EAA000204615F0C8FB28B9E86803681B69984739
:10EAB000014620E63A490B22204615F0BCFB0746EA
:10EAC000F8B904F10B082C6923682046DB689847E5
:10EAD0000546BD420FDD236839461B69204698472D
:10EAE0004146F2F7CBFB40B9236839465B692046C3
:10EAF0009847024618B92B49FDE50137E9E72A494D
:10EB0000AEE72A490B22204615F095FB002855D187
:10EB100005F11C0304F10B0118461C4615F0EDFC31
:10EB20002023022204A92046FDF70AFD00280ADD61
:10EB30000128049908D0059A286903689B699847B9
:10EB400020B11B49D7E51B49164AF5E71A49D2E51A
:10EB5000FC7D02080000164300401C450000E04018
:10EB60000000FA43077E0208247E02082C75020882
:10EB70003A7E0208497E0208557E02089A7E020803
:10EB8000A67E02086D7F0208ED7C02080A6D02086D
:10EB9000687E0208317A02087E7E02088D7E0208B5
:10EBA000937E0208F17C0208957802089F7E020895
:10EBB000AB7E0208CB850208AE7E02086E490B22AE
:10EBC000204615F038FB0746002842D12869036823
:10EBD000DB68984780462046F2F75AFB0B2804D999
:10EBE00004F10C00FEF714F80746474501DB6349C2
:10EBF00081E56349DFF88C914246304615F05AFAB8
:10EC00003046F2F745FB3418A31B852B05DDB845CC
:10EC10001BDD5D493A46204623E7286903683946EB
:10EC20001B69984782462869036839465B6998479B
:10EC3000524603464946204615F03CFA2046F2F774
:10EC400027FB0137B8450444DED1002304F8013C1A
:10EC5000C4E54E490622204615F0EDFA38B9324691
:10EC6000214628460DB0BDE8F04FFFF7D5BA484918
:10EC70000E22204615F0DFFA08B946493BE5464921
:10EC80000F22204615F0D7FA38B96B6883F8A50033
:10EC90002846FEF793FA41492DE541490B222046CB
:10ECA00015F0C9FA30B96B6893F8A530002BF2D093
:10ECB0003C4920E53C490922204615F0BCFA30B910
:10ECC000A868036801211B6A9847384913E5384949
:10ECD0000822204615F0AFFA014628B9A868036853
:10ECE0001B6A9847334906E533490922204615F047
:10ECF000A2FA28B9A86803685B6A98472F49FAE422
:10ED0000B8F1000F35D12E490322204615F093FAB1
:10ED100028B9A86803689B6A98472A49EBE42A49FE
:10ED20000D22204615F087FA38B9637B13F0DF0F08
:10ED300003D1A86803681B6C73E524490B222046A5
:10ED400015F079FA38B9E37A13F0DF0F03D1A86828
:10ED50000368DB6B65E51E490A22204615F06BFA55
:10ED600038B9A37A13F0DF0F03D1A86803689B6B4F
:10ED700057E51849BFE400BFC47E0208D07E0208F0
:10ED8000DE7E0208E77E0208EE7E0208A07B020813
:10ED9000FA7E0208097F02081D7F0208E379020853
:10EDA0002D7F02084E7F0208397F0208437F020848
:10EDB000517F02085A7F0208697F0208737F0208A8
:10EDC0004F6B0208817F0208887F0208967F020845
:10EDD000A27F0208AD7F0208A0F10903DBB2172B66
:10EDE0009DBF0348D84000F001000020704700BFDD
:10EDF000130080002DE9F041C4B001AC05460E4679
:10EE00004FF0010800278460216030460D4984F8E6
:10EE10000881C4F80480277210F062FF2B6885F81F
:10EE200004801B68284698470749304610F058FF71
:10EE3000404518BF84F8087194F80801AF6044B0E9
:10EE4000BDE8F081CD7F0208F36B020810B5C279EE
:10EE5000044652B10023C371A379072B5DD8DFE8C4
:10EE600003F01322429F7DB21D1A006803681B69DC
:10EE7000984708B9002010BD206803685B6998476F
:10EE8000021EF7DBD2B2E7E77B2A40F0A580012320
:10EE9000A3710320EFE77D2A00F09C802C2A02D189
:10EEA0000123A3710FE0617949B13A2A0DD12144C0
:10EEB00000230B7263710223A3710120DBE710466C
:10EEC000FFF78AFF18B10520D5E70E2925D822F0D3
:10EED0002003413B192B01D95F2A1ED14B1C214431
:10EEE00063710A72EFE76179D1B91046FFF774FFD9
:10EEF0000028E8D1222A01D10323D2E77B2AC6D0F9
:10EF0000A2F13003092BE9D9A2F16103192BE5D94C
:10EF10002D2A09D02E2A07D091B94FF0FF30AAE749
:10EF2000A2F13003092B06D87E29D7D91046FFF766
:10EF300053FF48B9F1E7A2F16103192BE8D8F3E7D1
:10EF40002C2A01D07D2AF1D121440023E2710B72D9
:10EF5000002363710523A37102208CE76E2A08D178
:10EF600063797E2BD9D85A1C627123440A221A7203
:10EF7000C2E7722A07D163797E2BCED85A1C627100
:10EF800023440D22F3E7222A03D05C2A01D02F2A42
:10EF9000C3D163797E2BC0D8591C61712344E6E745
:10EFA000222A04D16379234400221A72D0E75C2A12
:10EFB00001D1042375E763797E2BAED8591C234415
:10EFC00061711A727FE72C2A3FF46AAF7D2A03D160
:10EFD0000723A37104204EE71046FFF7FDFE00282B
:10EFE0007FF471AF99E72DE9F041C4B001AD002481
:10EFF0000127064685F808716C602C7285604FF019
:10F00000100829602846FFF721FF031E0CDC0CB90D
:10F01000013302D1002385F8083195F80801002357
:10F02000B36044B0BDE8F081013B032BEAD8DFE8D0
:10F0300003F002090F1408FB045003A9883015F0EF
:10F040005CFADFE7336877711B6830469847D9E789
:10F05000062CDFD80134E4B2D4E7002CDAD0013C2E
:10F06000F9E70000037913B1002303717047836847
:10F070000149186810F034BEE47A02082DE9F04125
:10F08000D0F808801D4698F80430012B04460F463E
:10F0900016462ED1FFF7E6FFA368204D1868DFF86B
:10F0A0008080394610F01CFEA3681E4918681E4F68
:10F0B00010F016FEA36816F8011B186821B9BDE808
:10F0C000F0411A4910F00CBE222903D1184910F062
:10F0D00007FEEFE75C2901D14146F8E70A2901D193
:10F0E0003946F4E70D2901D12946F0E710F0FCFD7F
:10F0F000E0E790F9051008EB011138468831F2F786
:10F10000BDF8074638B9013D2A4608F108013046E6
:10F1100015F0F3F87755BDE8F08100BFC97F02080C
:10F12000C37F0208BD7F0208C67F0208BE7F0208B7
:10F13000C07F0208F8B587683B79012B04460E466C
:10F14000154613D1FFF78EFFA3683146186810F0FB
:10F15000C7FDA3680D49186810F0C2FDA3682968AF
:10F1600018680A22BDE8F84010F03EBE90F905107C
:10F1700007EB011188313046F2F780F820B907F12A
:10F18000080013F031FE2860F8BD00BF3E6D020894
:10F19000F8B587683B79012B04460E46154613D116
:10F1A000FFF760FFA3683146186810F099FDA36867
:10F1B0000D49186810F094FDA368298818680A2280
:10F1C000BDE8F84010F010BE90F9051007EB0111F2
:10F1D00088313046F2F752F820B907F1080013F0F1
:10F1E000FFFD2880F8BD00BF3E6D0208F8B58768B6
:10F1F0003B79012B04460E46154613D1FFF732FF2B
:10F20000A3683146186810F06BFDA3680D491868B3
:10F2100010F066FDA368297818680A22BDE8F84056
:10F2200010F0E2BD90F9051007EB0111883130466E
:10F23000F2F724F820B907F1080013F0D1FD287087
:10F24000F8BD00BF3E6D0208F8B587683B79012B19
:10F2500004460E46154614D1FFF704FFA368314655
:10F26000186810F03DFDA3680D49186810F038FDCE
:10F27000A36895F9001018680A22BDE8F84010F05C
:10F2800087BD90F9051007EB011188313046F1F781
:10F29000F5FF20B907F1080013F0A2FD2870F8BDB2
:10F2A0003E6D0208F7B587683B79012B04460E4690
:10F2B000154625D1FFF7D6FEA3683146186810F031
:10F2C0000FFDA3681749186810F00AFDD5E900671B
:10F2D0000022002330463946F1F756FBA46830B1CE
:10F2E0001149206803B0BDE8F04010F0F9BC0623D6
:10F2F0000093206832463B4610F0D2FE03B0F0BDCA
:10F3000090F9051007EB011188313046F1F7B6FF8F
:10F310000028F3D107F1080013F05FFDC5E90001F3
:10F32000ECE700BF3E6D020851740208F8B587682B
:10F330003B79012B04460E4615461FD1FFF792FE7E
:10F34000A3683146186810F0CBFCA368144918680C
:10F3500010F0C6FC2D6800212846F1F797FEA3683F
:10F3600028B118680F49BDE8F84010F0B9BC18681A
:10F3700029460422BDE8F84010F0D2BD90F90510EE
:10F3800007EB011188313046F1F778FF30B907F10A
:10F39000080013F022FDF1F787FB2860F8BD00BFDD
:10F3A0003E6D0208517402082DE9F041876897F814
:10F3B0000480B8F1010F05460E46144620D1FFF730
:10F3C00051FEAB683146186810F08AFCAB681649EC
:10F3D000186810F085FCAB68A360236884F804808B
:10F3E0001B6820469847AB681049186810F078FCF5
:10F3F000012803D0AB68002283F80821BDE8F08122
:10F4000090F9055007EB051188313046F1F736FFCA
:10F410000028F3D12368A7600135657120461B6879
:10F42000BDE8F041184700BFCC7F0208F36B02082B
:10F4300070B50546D2B00B4616461049426868467C
:10F4400014F038FE2868694608F091FB044690B134
:10F45000296800236A460AA808F07FFB0AA808F07A
:10F46000E4FC044638B10AA93046FCF707F9044623
:10F470000AA808F092FC204652B070BDCF7F020867
:10F4800030B50446D3B00B4615460F49426868466E
:10F4900014F010FE2068694608F075FB216801230E
:10F4A0006A460AA808F059FB0AA808F0BEFC044600
:10F4B00030B10AA92846FCF7F8F80AA808F06DFC54
:10F4C000204653B030BD00BFCF7F020800207047F8
:10F4D000836910B544695A1CA24208D2046982614A
:10F4E000E154026983690021D154012010BD00203C
:10F4F000FCE7F8B505460F4616460024B44201D194
:10F500002046F8BD2B68395D1B68284698470028BF
:10F51000F6D00134F2E7002070474FF0FF3070471B
:10F520004FF0FF307047704710B500230122C0E94B
:10F53000012304460160C0F88C3480F890340349FC
:10F5400000F2914014F0D9FF204610BD167B02084E
:10F55000A0F12303DBB2162B04D8064A42FA03F3C8
:10F56000DB0704D5402894BF00200120704701200C
:10F57000704700BFFC1B80FFF0B5454B0D46002ACD
:10F5800014BF16461E46E9B004463146284608F028
:10F59000EEFA18B90026304669B0F0BD32460023B5
:10F5A000294620A808F0D9FA20A808F03EFC064613
:10F5B0000028EFD000230127C4E901730322694624
:10F5C00020A808F0B0FB032804D0002620A808F0EB
:10F5D000E4FBE0E7022204F1080120A808F0A3FB05
:10F5E00002280246F1D1A11D20A808F09CFB0228A8
:10F5F0000546EAD13A4604F5926120A808F093FB4B
:10F600000128E2D12A46211D20A808F08CFB0228FF
:10F61000DBD1242765891F2DD8D87D4305F10C0146
:10F620000222214420A808F07EFB02460028CDD00B
:10F630000228CAD105F10E01214420A808F073FB6D
:10F640000228C2D105F111011F22214420A808F08F
:10F650006AFB1F28B9D105F110010122214420A81D
:10F6600008F061FB0128B0D1802269460DEB020051
:10F6700008F059FB8028A8D12544A288AB899A427A
:10F680009CBF0133A380638901336381C2E700BF5C
:10F69000D87F020870B50C464979242988B0054600
:10F6A000164606D12188006808B0BDE8704000F019
:10F6B000C3BB232904F1050207D1334628682188FA
:10F6C00000F01FFC012008B070BD232311460DF18E
:10F6D00001008DF8003014F010FF33466A46EDE764
:10F6E0002DE9F04F054691B00F46904600F10C060B
:10F6F0004FF000096B894B4505DC4FF0000A50467E
:10F7000011B0BDE8F08F347918EA0404B24608D18C
:10F7100004236A4631462846FFF7BCFF83465C4512
:10F7200003DB09F101092436E4E739460DEB041047
:10F7300000F0AAFBFB888342E1D00134EFE7000030
:10F740002DE9F0410D46064614492846F1F796FD8D
:10F7500018B906F28C40BDE8F0812B78B6F80A8023
:10F76000232B08BF013506F112070024444501DBB5
:10F770000020F0E717F8013C232B3946284618BF34
:10F7800007F1FF31F1F77AFD243720B9242303FB79
:10F7900004600C30DFE70134E8E700BF167B0208A5
:10F7A0002DE9F8438846054617461E46013911F8EB
:10F7B000019FB9F1000F0AD141462846FFF7C0FF6B
:10F7C000044668B10388BB4235D0478005E048460F
:10F7D000FFF7BEFE04460028E9D12046BDE8F883C5
:10F7E0006889C6B1431C6B812423434303F10C0495
:10F7F0002B4401222C441A742423584305EB00099E
:10F800001130A9F80C601F224146284400F0B6FBD5
:10F81000A9F80E70E1E71F28DFD8431C6B81242371
:10F82000434303F10C042B4401221A74AE88B3182D
:10F830002C44AB80E0E74C46CFE700002DE9F047D1
:10F840000D4604461B492846F1F718FD20B904F27D
:10F850008C442046BDE8F0872B78B4F80AA0232B0F
:10F860004FF0000708BF013504F10C06B846BA4551
:10F8700001DC4446EDE77379232B14BF06F105093B
:10F8800006F10609494628463446F1F7F7FC0028F8
:10F89000DFD02846F1F7FCFC49460246284614F022
:10F8A000CAFC00280CBF3446444601372436A04623
:10F8B000DDE700BF167B0208F0B541B144890023A3
:10F8C000242500F10C06A34204DB002001E000F235
:10F8D0008C40F0BD05FB03F2B75A8F4202D10C32C7
:10F8E0001044F6E70133EEE7C188FFF7E5BF01B149
:10F8F0000988C1807047018909B1FFF7DDBF08465B
:10F90000704701B1098801817047F8B50B8863B170
:10F910004189002200F10E042425914207DC0024D5
:10F9200000F10C022426A14208DC00201DE005FBAA
:10F9300002F6A65B9E42F8D00132EEE706FB04F524
:10F94000575B9F4201D00134EDE74B1E9BB21A1B5F
:10F9500005F1300172430C35438101449C42C8BF1C
:10F960000022284414F077FC0120F8BD2DE9F8436B
:10F970000546884614461E46002747451DDB21796B
:10F980006379208811F0010F04F10502E9881AD08B
:10F99000232B194F194B08BFA21D884218BF3B46A5
:10F9A0001749304610F0C9F905F10C074FF000096E
:10F9B0006B894B4511DCBDE8F8832021304610F0FF
:10F9C00093F90137D9E7232B0B4F0C4B08BFA21D2E
:10F9D000884218BF3B460B49E3E77A8823889A425E
:10F9E00006D133463A4608F101012846FFF7BEFF2B
:10F9F00009F101092437DBE7CB850208E27F020821
:10FA0000F50E0308E47F02080B4600F28C42002149
:10FA1000FFF7ACBF10B588B091B172B100234FF4BD
:10FA20007A74CDE90512CDE902340B70054C0194CE
:10FA300001A90793FFF7E8FF079A104608B010BD29
:10FA40000A46FAE7F47F02082DE9F74F98469DF839
:10FA500030A090F89034009207460D4608EA030360
:10FA6000BAF1000F02D01BB92C4607E0002BFBD1E6
:10FA70002C462A2304F8023B2C236B7007F1120654
:10FA80004FF000094FF02C0B7A894A4509DCAC4253
:10FA900088BF04F1FF340023601B237003B0BDE86E
:10FAA000F08F16F8022C314608EA0202BAF1000F74
:10FAB00004D02AB909F101092436E5E7002AF9D171
:10FAC00016F8012C232A18BF06F1FF3108460191D0
:10FAD000F1F7DEFB0246601B009B019910440230E7
:10FAE0009842E7DA2046019214F00FFD019A14447F
:10FAF00004F801BBDEE70000F0B53B4B0D46002AE1
:10FB000014BF16461E46E9B031460446284608F0A2
:10FB10003AF832460123294620A808F01EF820A80A
:10FB200008F083F9064678B180220021684614F077
:10FB3000ACFB0322694620A808F039F8032806D058
:10FB4000002620A808F029F9304669B0F0BD02224D
:10FB500004F1080120A808F02AF802280246EFD193
:10FB6000A11D20A808F023F802280546E8D10122AB
:10FB700004F5926120A808F01AF80128E0D12A467D
:10FB8000211D20A808F013F80228D9D104F110058E
:10FB900000276389BB42D4DD0222291F20A808F078
:10FBA00006F802280246CBD1A91E20A807F0FFFFC5
:10FBB0000228C5D11F22691C20A807F0F8FF1F28C2
:10FBC000BED10122294620A807F0F1FF0128B7D1B4
:10FBD000802269460DEB020007F0E9FF802805F15D
:10FBE0002405ADD10137D4E7D87F0208806A704779
:10FBF00040697047836953F8210070476FF0604394
:10FC0000994270B534BF8E004FF0FF36044630463F
:10FC10000D46F6F726FC20602846F6F722FC6060C9
:10FC20003046F6F71EFC0023C4E902052361204696
:10FC300070BD4B1C30B5024605690DD00023184637
:10FC4000AB4200DB30BD946854F82340641A002CAA
:10FC5000D8BF01300133F3E72846F3E71830FFF748
:10FC6000E8BF70B5024604694FF0FF330020FF255E
:10FC700084420ADC002B26DB1168013C51F823008A
:10FC80001461116999420EDC70BD966856F82060C7
:10FC9000761A002E05DC5668365CAE423CBF034641
:10FCA00035460130E4E7990014680431655844F89A
:10FCB00023505468E5186D78E5549468615844F809
:10FCC00023100133DDE70020DEE71830FFF7C9BF5E
:10FCD0002C30FFF7C6BF02698A4230B5034618DDF3
:10FCE0000068013A50F821001A611A698A4200DC62
:10FCF00030BD8A001C680432A55844F821505C6865
:10FD000065186D7865549C68A25844F8212001312B
:10FD1000EBE70020ECE700210430FFF7DCBF1830F0
:10FD2000FFF7D9BF30B5D0E90354AC420CD0056819
:10FD300045F8241041680A550269816841F822306B
:10FD400001320261012030BD0020FCE700231A4689
:10FD50000430FFF7E7BF70B5044618300D46FFF7D3
:10FD6000E1FF30B92368294620465B68BDE8704052
:10FD7000184770BD70B51346044600222C300D465E
:10FD8000FFF7D0FF30B92368294620465B68BDE8FD
:10FD90007040184770BD00002DE9F0410646134B36
:10FDA00046F8043B04460D463046FFF727FF294638
:10FDB00004F11800FFF722FF294604F12C00FFF799
:10FDC0001DFF0027AF4202DB2046BDE8F0814FF463
:10FDD0008270F6F744FB8046FCF7C5FA00231A460A
:10FDE00041463046FFF79EFF0137EBE720800208CF
:10FDF000431E0F3013F8012F1AB98342FAD10120A4
:10FE0000704700207047F0B5D0F820510F2D044600
:10FE100011DCAB1C20F8151000EB031302F11007E6
:10FE2000106851681E4603C60832BA423346F7D1FD
:10FE30000135C4F82051F0BD2DE9F04706460025F4
:10FE40008E46284606F12008D6F82011A94201DD89
:10FE5000984201DBBDE8F08736F81510714511D1E5
:10FE600008EB051C00F1010902EB00140CF1100A6B
:10FE7000674603CF574520606160BC4604F1080423
:10FE8000F6D148460135DFE730B5A3B0054604A8F2
:10FE90000C4606F0D7FC10220DEB0200294606F0B6
:10FEA00038FE23780122C3F383030DF10D0104A86A
:10FEB0008DF80D3006F0AEFD628804F14A0104A809
:10FEC00006F0A8FD02231022009329460DF10E032F
:10FED0000DEB020006F035FEBDF80E3053B90123DC
:10FEE000ADF80E3004A8BDF80E4006F091FC204697
:10FEF00023B030BD4FF6FF729342F3D14FF6FE733D
:10FF0000EEE72DE9F0419846D0F820319EB0054645
:10FF10000E4617460024A34218DC684606F092FC01
:10FF20003846F1F7B5F939460246684606F072FDE3
:10FF300041466846102206F09FFD2846424631465B
:10FF4000FFF761FF684606F063FC12E035F8142005
:10FF5000B24211D1023405EB0414424604F11003FD
:10FF6000254603CD9D42106051602C4602F10802E7
:10FF7000F6D11EB0BDE8F0810134CCE7013902446E
:10FF8000131A012B02D800230370704711F8013FA8
:10FF9000002BF8D000F8013BF2E7013810F8013FE0
:10FFA0000BB901207047202BF8D0002070470000CB
:10FFB00070B500210646F1F769F8374C054640B1A7
:10FFC000302323702E22A37000236270E370324826
:10FFD00070BDC6F3C7537F3B1E2B99B257DC13F19C
:10FFE000170F54DBC6F31602162B42F4000216DD7F
:10FFF000173902FA01F0002E40DB0A22214610F0E8
:020000040801F1
:100000001DFA237822460134002BFAD12E231370D7
:10001000EDB93021931C517000221A70D7E7002BE4
:1000200008DBC1F11700013142FA00F08A4022F0EA
:100030007F45E0E7DB43002E42FA03F54FF0300343
:1000400020DA63702D222E232270A3700334E11D69
:1000500023460A2045432A16303203F8012B8B42EF
:1000600025F07F45F6D106342278302A234603D185
:1000700014F8012D2E2AF7D10133CDE72D2304F8F2
:10008000013BBAE723702E2363700234DFE730238D
:100090002370002363709AE7003A002037B52049A7
:1000A0000546F0F75FFE002104462846F1F70CF8FC
:1000B00070B34FF07C512046F0F74CFDF1F72EF86D
:1000C0004FF47A7290FBF2F302FB13000028154CF8
:1000D000154AB8BF404210210090204613F0B6FFE9
:1000E0002046F1F7D5F80021431E2044002B03DD04
:1000F00010F8012C302A0ED00A48F1F7C9F801385F
:10010000235C2E2B04BF00232354064803B030BDCC
:100110004FF03F41CFE700F8011D013BE6E700BF8C
:1001200000007A44F03900204C800208024A13781B
:1001300043F0100313707047103A002038B504469E
:10014000406812490368D3F8B830984723682046BE
:100150005B6D9847034684F8240060680268082BAA
:100160008CBF10212021126E9047094BA0680025FA
:100170001D7003689B6B9847012801D1FFF7D6FFDC
:10018000A5612577E583256238BD00BF2D010108F3
:10019000103A0020C38B41833F2B82BF0023C383CF
:1001A00003627047034B187800F0EF00431E58427B
:1001B00058417047103A00202DE9F041174E34782D
:1001C00014F0100405460F46904616D040680368A8
:1001D0000121DB6E9847041E0DDD68684445036805
:1001E000A8BF44461B6B22463946984790B16B69BD
:1001F00001336B610024002333703378012B06D068
:10020000686803689B69984708B9012333702046E2
:10021000BDE8F081EB680133EB60ECE7103A0020B9
:10022000406808B50368DB6F98474FF47A73B0FBFA
:10023000F3F008BD10B50446406803689B6A984710
:10024000A06803689B699847014B00221A7010BD93
:10025000103A002040680368D3F89C30184700002B
:1002600070B5094E3378DB0604460CD403681B6C6A
:100270009847054638B9236820465B6C9847357027
:100280002583E583256270BD103A002010B5174B19
:100290001A78C38B012A044617D13F2B17D803685D
:1002A0001B6C984780B9236820461B6D9847F0F770
:1002B00035FFB4F918300D33984205DCE38B013378
:1002C000E383236A0344236210BD3F2BFCD9236AD6
:1002D000002BF9D0B8BF3F3343F38F136FF0770291
:1002E0009342B8BF134623830023ECE7103A002063
:1002F00006490B78024613F0100005D000230B705E
:100300001369013313610120704700BF103A0020C8
:100310000739234B2DE9F04153F82180044601466B
:1003200040461546F0F7DAFEC0BB2846F0F75AF80B
:100330001C4B0022F0F7C0F802460B4600201A4979
:10034000EFF702FF06460F4620464146F0F700FC55
:10035000F0F75AF8154B0022F0F7D8F902460B4691
:1003600030463946F0F7A8F80F4B002204460D46F8
:10037000F0F714FB60B10022002320462946F0F775
:100380002BFB40B120462946F0F78EFBBDE8F081FB
:10039000054D0024F6E700240025F3E70020F5E7EB
:1003A000548002080000703F0000F03F000024402D
:1003B00040686FF0004105F04CBA406803685B6D1F
:1003C00018470000406808B503681B699847024B4E
:1003D00000221A7008BD00BF103A0020F8B504468C
:1003E000806803685B690D46164698476068036835
:1003F00032465F6A29460023B84720B9064B0322DC
:100400001A700120F8BD2046FFF7DCFFA0680368E2
:100410009B6998470020F5E7103A0020406808B52E
:1004200003689B69984710B9014B01221A7008BDF7
:10043000103A002038B5B0F91A30044613B9207FBD
:1004400098B938BD03681B6D9847B4F91A30054652
:10045000B4F918001844F0F731FC01462846F0F7CB
:100460003DFE0028EBD00120EBE7236820469B6D82
:100470009847064B0546002220461A70FFF7CEFF2C
:1004800015F10F0018BF0120DBE700BF103A002074
:100490000846114606291A4601DDFFF739BF00203C
:1004A000704700002DE9F843054642F21070904075
:1004B000164699468846F0F7FDFB1D499DF82070C9
:1004C00004464846F0F74EFC01462046F0F7FEFC95
:1004D000F0F74AFE053E9DF82430012E8CBF112412
:1004E0001924083304EB83044443D8F80400036858
:1004F000FF21DB6F9847A4088442A7F1050234BFAF
:10050000031BC4F57A63022A98BFDB004FF47A72AA
:1005100098BFB3FBF7F304F2E73403F2E733B4FB1D
:10052000F2F4B3FBF2F32C606B602846BDE8F8836D
:100530000000204100207047F0B51D4F1D4CD7F83A
:10054000E03585B0002200921B4A04EA832303EBC6
:10055000C12307CA01AD85E80700D7F8E02504EA02
:10056000822203F1FF6602F1FF6106F5F02601F534
:10057000F021B14218D802F10062013AB24213D31D
:10058000A3F50043DB0A0293F1F758FD69462846BC
:10059000F1F7E6FD0446F1F763FD002C14BF6FF0A0
:1005A0000400002005B0F0BD6FF01500FAE700BFB1
:1005B0000070FF1F00FCFF03E46202082DE9F04712
:1005C000204E214FD6F8E04507EA842404F1FF6469
:1005D00004F5F02414441D4604EBC124F1F72EFD6C
:1005E000804678B9089B23F0070303EB04096FF0FA
:1005F000784AA1450AD1F1F733FD40EA080010F02E
:10060000FF0001D06FF00400BDE8F087D6F8E035B8
:1006100007EA832303F1FF6202F5F022A24202D827
:100620005344A34204D2F1F71BFD6FF01500EBE732
:100630002146F5E802230120F1F74CFD08348046FD
:10064000D7E700BF0070FF1F00FCFF0338B5184656
:100650001546049A8BB182B1094B0A4CD3F8E035A8
:1006600004EA83242C4404F1FF6404F5F02404EB31
:10067000C12113F04AFF002038BD6FF01500FBE7E1
:100680000070FF1F00FCFF0310B5034B036004461E
:1006900007F014FA204610BD7480020810B5044615
:1006A000FFF7F2FF20465021F5F7DDFE204610BD92
:1006B00010B50449044607F009FA034B23602046AD
:1006C00010BD00BF240100207480020813B5002370
:1006D0008DF807309DF80730044603F0FF014BB159
:1006E000204607F016FA0021204602B0BDE810406F
:1006F00007F0FEB907F0FCF90028F1D002B010BDF8
:100700000148FFF7D5BF00BF143A002008B50248E2
:10071000FFF7BAFF08BD00BF143A0020028BC08A61
:10072000101A7047C28A018B914288BF0169034643
:1007300083BF885C0132DA824FF0FF307047028B52
:10074000C38A9A4286BF0269D05C4FF0FF3070477F
:10075000806DD0F8DC302BB100234384D0F8E0303A
:10076000D43018477047000070B54FF47A730E46C6
:100770000021C0E90113034615462B4A43F8C42B58
:100780000446C0F8C4109C22C3E90111C0E9341129
:10079000C0E93611C0F8E010283013F076FDF3B24E
:1007A0001A2B19D8214A52F8233006F4E0661E436A
:1007B000EBB21A2BC4F8846022D81C4A52F82330BA
:1007C00005F4E0651D430023C4F88850E3612384E9
:1007D0002361A382204670BD06F0C002C02A0CD15E
:1007E000C72B0AD8124B06F03F0206F4E06653F816
:1007F00022200E4B53F82230D9E74FF0FF36D7E7CF
:1008000005F0C002C02A0CD1C72B0AD8084B05F04E
:100810003F0205F4E06553F82220044B53F82230E0
:10082000D0E74FF0FF35CEE7848002088C670208DE
:100830006C67020838B50446283000F081FCE06996
:1008400018B112F0DDFA0023E36120690025258448
:1008500010B112F0D5FA2561A58238BD38B505462C
:10086000074B45F8D43B0446FFF7E4FF2846F5F76D
:1008700006FB04F1C400F5F702FB204638BD00BFBB
:10088000848002080123994080F824300023817677
:100890004384704738B5838A8B4205460C4609D29B
:1008A000202938BF20240069214612F0CBFB10B16B
:1008B0002861AC8238BDFEE773B5846D866ED4F8CE
:1008C000CC300546E3B1E28A238B9A4218D33146F5
:1008D0002046FFF7DFFF2069324605F1740113F06F
:1008E00014FE0023E382D4F8CC30268301960BB9A2
:1008F00010F09AF9D4F8D03001A904F1C400984757
:1009000002B070BDB1F5806F70B505460C4610D8C9
:10091000038C99420AD920290E4638BF2026C06987
:10092000314612F08FFB18B1E8612E84204670BD6D
:10093000FEE70024FAE713B590F824308DF807108D
:1009400004467BB1418C0131FFF7DCFF40B1638C81
:10095000E2699DF80710D154638C01336384012050
:1009600002B010BD01220DF10701283000F038FC63
:10097000B0FA80F04009F3E770B590F824300446EF
:100980000E46154693B1418C1144FFF7BBFF10B9D9
:100990000025284670BD638CE0692A46184431461C
:1009A00013F0B3FD638C2B446384F2E792B22830DA
:1009B00000F016FC0028EBD1EBE70346006918B104
:1009C0009A8A002113F061BC70470346C06918B1D0
:1009D0001A8C002113F059BC704738B50446C9B9C8
:1009E000AA23A36594F8BE30012B16D1638CE2696B
:1009F000A17E04F1280000F074FC042828BF042024
:100A000045B22046FFF7E1FF0023638484F82430D9
:100A1000E8B238BD4FF42A43E3E70425F8E72DE9AF
:100A2000F04790F8BEA09DF820509DF82490BAF1B0
:100A3000010F04460F461646984637D111467F00EF
:100A4000FFF728FFFFB2CDB1032D28BF0325013DDD
:100A50000023EDB284F824A0A7766384ED00236818
:100A600028FA05F11B68C9B22046083D984715F1E0
:100A7000080FF4D100212046FFF7AFFFB9F1000FB6
:100A800011D1AA23A36522693346394604F128000F
:100A900000F0C0FB002818BF00260023E382268355
:100AA0003046BDE8F0874FF42A43EBE70026F7E72E
:100AB00007B5019300230093FFF7B1FF03B05DF882
:100AC00004FB0123FFF7F4BF0121FFF786BF38B510
:100AD00004460025C5820583FFF76FFF6584204625
:100AE000FFF773FF38BD0000F8B50446D0F8840066
:100AF0000FF0F6FC00210FF0B9FDD4F884201309A3
:100B000013F00C0645D103F00F03254D254F55F882
:100B1000231002F00F0257F822300A6993433DD0A8
:100B2000D4F888000FF0DCFC01210FF09FFDD4F811
:100B300088001D4B010911F00C0F1B682CD100F02F
:100B40000F021A4C57F82270B3FBF4F3184A0A2428
:100B500001F00F016343142655F821C0CCF828702A
:100B6000D2F804E05468A4EB0E04A342FADCCCF8FB
:100B70001870D2F804C05468A4EB0C04A342FADC49
:100B8000013EE9D10FF0ACFC3146BDE8F8400FF072
:100B90006DBD00231B69FFDEB662FCE7F8BD00BF38
:100BA00008000020B46802084000002040420F0006
:100BB000001000E02DE9F04104460026C6820683BD
:100BC0001F460D469046FFF7F8FE6684A67620463F
:100BD000FFF7FBFED4F8DC30C4F8804033B104F1F9
:100BE000D401032208469847C4E93766002384F8F5
:100BF00024306B0084F825306B1E5D425D4184F823
:100C0000BE50204684F8BF8084F8C07004F12805E7
:100C1000FFF76AFF94F825200949284600F0DCF91F
:100C200094F8BE304BB92846064900F0B2FB28467E
:100C30000549BDE8F04100F0A5BBBDE8F08100BF6B
:100C4000A086010051070108B90801080A460023DF
:100C50000121FFF7AFBF000002480822C021FFF7C3
:100C600083BD00BF643A00200148FFF7F7BD00BF15
:100C7000643A00204FF0B04382B09A6D02439A6507
:100C80009B6D03400193019B02B070472DE9F04F2B
:100C9000874B53F8312082429FB00F4607D103EBB8
:100CA000C102D2F80480B8F1000F40F0FD801C2290
:100CB0008049814C43F837007A4301EB5003B3FB82
:100CC000F0F0A318A2589D7E01EB5204B4FBF2FA97
:100CD000DC8A0594059E1C8A1A8B0E923444149467
:100CE0000E9E9C89CDF83CA03444EA1C4243323C21
:100CF000A41A24EAE474059E0694DC89A41BA4F5D6
:100D000082740244A21A22EAE272079200FB05F200
:100D100008925A68B1FBF2F215929A68B1FBF2F2AE
:100D20001692089A02EB4002323212924242049228
:100D3000129A00261021821810910B964FF0FF385E
:100D400034070E9D1C94059CF1B22C44139112990A
:100D500011946FF00105AAEB0404511A05FB02443B
:100D600018940D914FF00009149C0D9DAC4200F2B7
:100D70008A801C9C49EA04041B940024CDE90244A7
:100D80004B4C04EBC7041D94069C029DAC4270D8EA
:100D9000079CAC426DD3109C139DAC4269D00B9C58
:100DA0000134072C0B947FD85C8A039D17941B9CFD
:100DB0002C431A94089C141B0094119C14440C940A
:100DC000189C0A9400240194089D009C2C44179DB3
:100DD000A5423DD2009C323CB0EB940F38D21A9D14
:100DE000019C2C430C9D1994A2EB0A042C440A9DEF
:100DF000099596464FF0000C169D0AEB040B5D45D5
:100E00001AD8159D5D4517D3B3F814B0F34513D820
:100E1000704511D2DDF824B00F9D1BEA240B38BFBA
:100E2000A346AB4508D2199D4CEA05081D9DC5F89F
:100E30000480139DCDE90FB5099DDDF810B00CF5C8
:100E4000807C5D44BCF5803F0C4409958E44D3D131
:100E5000019C049D01340194009C0C4400940A9C64
:100E60002C440A940C9C0C440C94019CB4F5807F97
:100E7000AAD1029C0C440294039C04F58034B4F57E
:100E8000801F039480D10D9C09F580190C44B9F1A1
:100E9000807F0D947FF468AF04990136091A102EF3
:100EA000049102447FF44CAF40461FB0BDE8F08F80
:100EB000543B002000CA9A3BA880020808B52C4B7E
:100EC000984216D14020F3F74FF9002846D14FF051
:100ED000B0432849D3F888301B0903F4407343F426
:100EE00040328A4238D001F580718A423BD0B3B398
:100EF000FEE7214B984215D18020F3F735F968BB06
:100F00004FF0B0431D49D3F888301B0903F4406308
:100F100043F440228A421FD001F580618A4222D0E8
:100F2000EBB1FEE7164B98421FD14FF48070F3F7F8
:100F30001BF998B94FF0B0431249D3F888301B0918
:100F400003F4405343F440128A4205D001F5805126
:100F50008A4208D01BB1FEE70B4B186808BDBDE8FC
:100F60000840F3F75BB80948F8E70020F6E700BF50
:100F700000540040000103000058004000040C0031
:100F8000005C004000103000400000200024F4000D
:100F900008B50E4B994212D90D4B994207D80068FB
:100FA000FFF78CFF0121BDE80840FFF76FBE094B3A
:100FB000994209D80068FFF781FF0221F3E7006832
:100FC000FFF77CFF0021EEE7002008BDA0860100AE
:100FD000801A060040420F00F8B50F461546044639
:100FE000002800F09F805049C06DF5F735FF4F494C
:100FF0000646206EF5F730FF0146002E00F0928085
:10100000002800F08F803046F5F74DFF2060002863
:1010100000F08880464B984204F1040650D14FF40A
:101020000010FFF727FE4FF0B0439A6B02439A631C
:101030009A6B22F400129A6341F61E73A4F864308E
:101040003C4B1E603949206EF5F7EEFE3649E06DE7
:10105000F5F7EAFE2368636039462046FFF798FFFC
:101060000123C4E902050025C4E9043594F897304A
:1010700094F96400A5615B1B18BF0123DB042362A4
:1010800094F8983084F845505B1B18BF01235B042B
:1010900063622A460221F0F741FE94F96400F0F7FA
:1010A0006FFE94F965002A460221F0F737FE94F9A5
:1010B0006500F0F765FE3046F1F7C1FA70B3FEE760
:1010C0001D4B984213D14FF48000FFF7D3FD4FF032
:1010D000B0439A6B02439A639A6B22F480029A633C
:1010E00042F22013A4F86430124B5E60AAE7134B5F
:1010F0009842A7D14FF40000FFF7BCFD4FF0B0437A
:101100009A6B02439A639A6B22F400029A6343F249
:101110003013A4F86430074B9E6093E70223A06667
:1011200084F89530F8BD00BF88660208346602086E
:1011300000540040483B002000580040005C004044
:1011400010B5044690F96400F0F728FE94F96500A4
:10115000F0F724FE201DF1F7C8FA206E0321F5F701
:10116000D5FDE06D0321F5F7D1FD2368194A9342BF
:101170000ED14FF0B0439A6B42F400129A639A6B0F
:1011800022F400129A639A6D22F400129A6510BD3F
:10119000114A93420DD14FF0B0439A6B42F4800252
:1011A0009A639A6B22F480029A639A6D22F4800209
:1011B000ECE70A4A9342EAD14FF0B0439A6B42F40B
:1011C00000029A639A6B22F400029A639A6D22F4E9
:1011D0000002DBE70054004000580040005C004083
:1011E000202A30B514D800239CB2A24207D890F828
:1011F00094301344DBB280F89430002030BD90F876
:101200009440CD5C1C440444013384F87450EBE7F3
:101210000120F3E72DE9F34705460F46904699462E
:10122000F0F73CF90024D5F830A006460435CDF897
:1012300000A04B46424639462846F1F765FB022896
:1012400006D1F0F72BF9841B642CF0D906201FE09F
:1012500008BBF0F723F906462846F2F720FA2028C3
:1012600009D0632C07D8F0F719F9841B2846F2F748
:1012700019FA0028F0D02846F2F714FA632C0CD89B
:1012800082060AD443070AD4003818BF0120800020
:1012900002B0BDE8F0870420FAE70520F8E7032054
:1012A000F6E710B5642304460430F1F737FA022854
:1012B0000AD0032801D068B910BD94F84530202B1E
:1012C0000CBF02200520F7E794F84530202B18BF0B
:1012D0000620F1E794F84530202B0CBF02200420B3
:1012E000EAE72DE9F34704460E4691461F46F0F71C
:1012F000D5F880463FB901223146204602B0BDE80C
:10130000F047FFF7CEBFD4F830A000250434CDF865
:1013100000A03B464A4631462046F1F781FA0228B2
:1013200007D1F0F7BBF8A0EB0805642DEFD9062034
:101330001FE008BBF0F7B2F806462046F2F7AFF917
:10134000202809D0632D07D8F0F7A8F8851B204680
:10135000F2F7A8F90028F0D02046F2F7A3F9632DA0
:101360000CD882060AD443070AD4003818BF0120DB
:10137000800002B0BDE8F0870420FAE70520F8E716
:101380000320F6E720B119B1C1660430F1F7D2BBF2
:10139000704720B119B101670430F1F7CBBB70473A
:1013A00070B590F89130012B04460E46A0F104056B
:1013B00009D1436E3BB1836E28469847022384F8D7
:1013C000913000236366012E4FF0000312D1E26ECC
:1013D00084F891301AB184F890302846904794F8F8
:1013E000902004F1700120464FF00073BDE870407A
:1013F000F1F7DCBA0122636684F89120616E7431E2
:10140000294420464FF08073BDE87040F1F730BBAF
:1014100010B590F89130012B044604D1436E13B1FE
:10142000836E04389847022384F891300023636662
:101430002046BDE81040F1F77DBB436E1F2BDEBF99
:10144000436E0133436690F89130012BDAB206D136
:10145000416E70314FF080730144F1F709BB704762
:10146000002380F89030704790F892300BB9F1F774
:1014700061BB7047014B1868F1F770BB483B002017
:10148000014B1868F1F701BF483B0020014B586839
:10149000F1F764BB483B0020014B5868F1F7F5BEFB
:1014A000483B0020014B9868F1F758BB483B0020AF
:1014B000014B9868F1F7E9BE483B00202DE9F04167
:1014C000104D2F4604468C4690469E46061D0FCF73
:1014D0000FC697E80700069B86E807001C35A36245
:1014E000079BE3620FCD04F13006C4E9088E0FC6F6
:1014F0002B683360002363642046C4F800C0BDE855
:10150000F08100BFF062020810B50446006803686D
:101510005B6C98472068216A036882689B689847DB
:101520002068216A03680269DB689847004B10BD98
:101530005C010020006803689B6C18472DE9F041AE
:101540000D461946037C0446407CADF5067DDE0859
:10155000082B5FFA85FC06EBD00663898D9FD0B21D
:1015600095BF40EA0C004CEA122C8DF800008DF873
:10157000010092BF0DF101008DF800C00DF10200D5
:10158000AB423E443A462CD112F0BFFF20680368BC
:101590005B6B98472068216A0368C268DB689847DC
:1015A000206803683246D3F83880694643ABC047A9
:1015B0002068216A03680269DB689847206803682D
:1015C000DB6B98472389AB4207D1217C8C9843ABD6
:1015D0003A4603EBD10112F098FF0DF5067DBDE808
:1015E000F081A18912F051FED0E72DE9F04FADF561
:1015F000077D0446929F9DF84CA21646D519994640
:10160000002B55D0684612F080FF90993A460DEBBA
:10161000060012F07AFF20680368BAF1000F05D0C7
:10162000E26A013254D1DB693221984720680368AD
:101630005B6B98472068216A0368C268DB6898473B
:10164000206803680DF58678D3F838B02A464346FB
:101650006946D8472068216A03680269DB689847B1
:1016600020680368DB6B9847BAF1000F07D0E26A85
:1016700020680132036845D1DB690121984765691B
:1016800035B1002F5CD0E37C18F80300A84705466D
:10169000B9F1000F07D1A37C919806EBD3013A462C
:1016A000414412F032FF28460DF5077DBDE8F08F6A
:1016B000837C68464FEAD30805EBD30512F025FF7B
:1016C000A18908EB07020DEB060012F0DEFDA2E790
:1016D0005B6A984780462068E16A03681B699847FF
:1016E0000028A3D0206803685B6D984720680368D2
:1016F0005B6A9847E369A0EB08009842EBD36FF46C
:101700003075D0E71B6A01219847206803685B6A3F
:10171000984705462068E16A03681B6998470028D6
:10172000ADD0206803685B6D9847206803685B6AEA
:101730009847E369401B9842ECD36FF43075A7E7F4
:101740003D46A5E7F0B51E46037987B005460F462E
:101750003BB9CDE900620A460189FFF7EFFE07B009
:10176000F0BD90F9114090F811C0002CB8BF0734BB
:10177000E410013C64B204ABE0001946002C12DA1C
:101780002C7CE408601E40B2B0F1FF3F15D101236C
:10179000CDE9022300230196009304EBDC022846E6
:1017A000FFF723FFDBE7B5F808E0013C4EFA00FE47
:1017B00003F801EB64B20838E0E74FEAC00E27FAFD
:1017C0000EFE03F801EB0138DDE7F0B589B0002328
:1017D0008DF81730037904460A465BB9012101915F
:1017E0000DF1170100910189FFF7A8FE9DF8170080
:1017F00009B0F0BD90F91130467C002BB8BF07331B
:10180000DB10013B5BB206A8DD000146002B13DABA
:10181000257CED086B1E5BB25F1C15D10123CDE961
:1018200002330DF1170301930023009305EBD60259
:101830002046FFF7DAFED9E72789013B2F4100F860
:10184000017B5BB2083DE1E7DF0022FA07F700F811
:10185000017B013BDFE7F0B516461A46037987B0F6
:1018600005460F4643B9CDE900320A463346418961
:10187000FFF764FE07B0F0BD90F9114090F811C079
:10188000002CB8BF0734E410013C64B204ABE000A4
:101890001946002C12DA2C7CE408601E40B2B0F12C
:1018A000FF3F15D10123CDE902230022CDE90062DB
:1018B000284604EBDC02FFF798FEDBE7B5F80AE008
:1018C000013C4EFA00FE03F801EB64B20838E0E791
:1018D0004FEAC00E27FA0EFE03F801EB0138DDE7F0
:1018E000F0B5037989B004460D468DF8172053B939
:1018F0000122CDE900320A460DF117034189FFF7B5
:101900001DFE09B0F0BD90F91130467C002BB8BF28
:101910000733DB10013B5BB206A8DA000146002B5F
:1019200013DA227CD208531E5BB25F1C15D1002053
:10193000012301900DF117000090CDE9023302EB75
:10194000D6022046FFF751FEDBE76789013B1741CE
:1019500000F8017B5BB2083AE1E7DF0025FA07F700
:1019600000F8017B013BDFE72DE9F0479DF820A05F
:101970009DF828709DF82C901C4643EA0A03072B1B
:1019800005460E46904642D8544540D3FFF71DFF0A
:10199000631CFF22DBB2CAF1080A02FA03F342FA1F
:1019A0000AF21343DB43DBB280EA0802134205D19B
:1019B000B9F1000F02D10020BDE8F08720EA03044E
:1019C00003EA08031C43E4B2224631462846FFF7E7
:1019D00087FF286803689B6A98479DF824804FF426
:1019E0007A73814603FB08F8286803689B6A984766
:1019F000A0EB0903434502D36FF00F00DCE731464B
:101A00002846FFF7E2FE60400742EDD1D3E76FF0D2
:101A10000A00D1E77FB59DF824600396089E9DF8E3
:101A20002850CDE90136002300930446FFF7DDFD81
:101A300038B935B1A36923B1204604B0BDE8704080
:101A4000184704B070BDF0B590F9114090F811C07E
:101A5000002CB8BF0734E41087B0013C64B205AD78
:101A60000F46E6002946002C0DDA9DF8344002941A
:101A70009DF83040CDE9003413464FEADC02FFF711
:101A8000C9FF07B0F0BD47FA06FE013C05F801EBBF
:101A900064B2083EE7E77FB59DF824600396089E90
:101AA00002960026CDE9003601239DF82850044611
:101AB000FFF79BFD38B935B1A36923B1204604B0C7
:101AC000BDE87040184704B070BDF0B590F9114002
:101AD00090F811C0002CB8BF0734E41087B0013C67
:101AE00064B205AD0F46E6002946002C0DDA9DF8DC
:101AF000344002949DF83040CDE9003413464FEA5B
:101B0000DC02FFF7C8FF07B0F0BD47FA06FE013C54
:101B100005F801EB64B2083EE7E770B586B0002334
:101B20008DF8133090F91130427C002BB8BF073389
:101B3000DB10013B04465BB205A8DD000146002B2B
:101B400016DA0123CDE902330DF1130301930023CB
:101B50000093D2082046FFF748FD054628B963697F
:101B60001BB19DF813009847E080284606B070BD71
:101B7000E689013B2E4100F8016B5BB2083DDEE7D0
:101B800070B50B46054601F11404303053F8046B70
:101B900040F8046BA342F9D16A640E1F01F11004EE
:101BA000286856F8041F036882689B689847A64215
:101BB000F6D170BD406C18B970478B4204D0183014
:101BC0000378002BF9D118467047F8B50546FFF7A2
:101BD000F1FF88B1041D05F12C0605F1400756F808
:101BE000041F002904DB286822680368DB68984723
:101BF000BE4204F10404F2D1F8BD00000648074BD0
:101C0000074A1B68B3FBF2F310B544684B434268C4
